:020000040000FA
:10000000021F3F022003FFFFFFFFFF02200BFFFF45
:10001000FFFFFF022013FFFFFFFFFF02201BFFFF78
:10002000FFFFFF022023FFFFFFFFFF02202BFFFF48
:10003000FFFFFF022033FFFFFFFFFF02203BFFFF18
:10004000FFFFFF022043FFFFFFFFFF02204BFFFFE8
:10005000FFFFFF022053FFFFFFFFFF02205BFFFFB8
:10006000FFFFFF022063FFFFFFFFFF02206BFFFF88
:10007000FFFFFF022073FFFFFFFFFF02207BFFFF58
:10008000FFFFFF022083FFFFFFFFFF02208BFFFF28
:10009000FFFF70DFFFFF040000000002000000C847
:1000A000030002030369A5020269A532730000017F
:1000B00000000000000400FFFFFFFFFFFFFFFF0440
:1000C00003090424035400650078006100730020D4
:1000D0000049006E0073007400720075006D0065C9
:1000E000006E007400730024035400490020004394
:1000F000004300320035003300310020005500532A
:10010000004200200043004400430000035F005F02
:100110000030005800000000000000000000000057
:1001200000000000000000000000000000000000CF
:100130000000000000303132333435363738394171
:100140004243444546331C881C881C881C881C90EC
:100150001C74F8121BCD900391E06015900302749B
:10016000FEF0900304744DF0A37405F07A011207B9
:100170001C7F01021D6C74F8121BCD74FF121EB699
:100180007E00801F851882851983E064FE700690CA
:1001900003877401F0851882851983E0F890038441
:1001A000E068F07901AA18AB191210E9E9700302AE
:1001B0000287851882851983E064EF70027E07E06C
:1001C000C0E0900387E0FA900385E0F8EA28F8E4BD
:1001D0003400F9740228F582740339F583D0E0F015
:1001E000900387E0609E14600E14602B14603B1433
:1001F0006051146067809E900384E4F085188285C6
:100200001983E0900386F0C394809003874003E451
:1002100080827402020194851882851983E090031C
:1002200082F09003877403020194851882851983F4
:10023000E0900383F0900386E060199003877404D4
:10024000020194900385E004F0F8900386E0686072
:10025000030201959003877405020194900385E4DD
:10026000F0900387F0900384E0F885188285198365
:10027000E0686003020195900382E0644D60030230
:1002800001951203BF8002EEF97401121E370201BC
:100290007174F7121BCD74FB121EB6EAFEEBFF75EC
:1002A00008047509007808121ED07402121F377AEC
:1002B000907B0079041218EB7402121E3712070E9D
:1002C000121F88E0687003A3E069701285188285A8
:1002D0001983E0F47003A3E0F4600302039A74044A
:1002E000121F2F1207708A088B09A808A909740227
:1002F000121F88E8F0A3E9F07404121F88E0600878
:1003000079011201510203B3851882851983E068CF
:100310007003A3E0697076851882851983E0F47014
:1003200003A3E0F470197402121F887410F0A37410
:1003300020F08518828519837410F0A37420F0755D
:1003400008017509007808121ED07402121F377A4E
:10035000247B0812196F7402121E3775080478087E
:10036000121ED07402121F377A907B007904121883
:10037000EB7402121E3712070E121F88E06870031A
:10038000A3E069700479028006790480027903127F
:1003900001518E828F83741E80058E828F83E4F0DC
:1003A00012070E121F88E0687003A3E069700479D9
:1003B00001800279007405121E377F02021D6C74E1
:1003C000ED121BCD74F8121EB6900307E0FD9003EA
:1003D00006E0FCFAEDF8E4C8F9EA28FEE93408FF83
:1003E000751001750B00750A068E088F0974027866
:1003F00008121F1CC39508F8E49509F9740228F542
:100400000E740339F50F8E088F0974097808121FCE
:100410004EE508F511EE2410F508E43FF509EEF578
:100420000CEF5401F50D900383E014605914700330
:100430000204FB14700302057614601024FE70039E
:100440000206311470030206E10206F1750A03790F
:100450004E1213BD9003071207047402F0A37440F8
:100460001207027408120702F0A3F07418C394076D
:1004700004F510AA10A90B12071CA90A7408121E71
:10048000377F0C021D6C750A04794E1213BDEE45C0
:100490000D7005A9111219D5C3EE9425EF940850DB
:1004A0003CC3E5089424E50994084031E50E249600
:1004B000F8E50F3420F988828983E0701BA3AA82B3
:1004C000AB83E070139003887401F0888289837491
:1004D000A5F08A828B838004900388E4F07508106D
:1004E0007509007808121ED07C087D03EEFAEFFB38
:1004F00012196F7402121E37020473750A05E51192
:10050000C394794006750B0102047375124075138C
:10051000007812121ED07C097D037402780C121F21
:100520001CAA0CAB0DA9111218EB7402121E379005
:100530000307E0A3F0900306E0A3F0751043C3EEB9
:100540009425EF94084003020473C3E5089424E55E
:100550000994085003020473900388E070030204B6
:1005600073E50E2497F8E50F3420F988828983E437
:10057000F0A3F00204737508047509007808121ED0
:10058000D07402121F377A907B0079041218EB7432
:1005900002121E377402121F88E0F8A3E0F98518D2
:1005A00082851983E0687003A3E069851882851944
:1005B00083700BE0F47003A3E0F470578009E0F45B
:1005C0007003A3E0F4700D8518828519837410F010
:1005D000A37420F012070E121F88E8F0A3E9F0754B
:1005E00008017808121ED07402121F377A247B0883
:1005F00012196F7402121E377508047808121ED083
:100600007402121F377A907B0079041218EB74027F
:10061000121E3712070E121F88E0687003A3E069EC
:100620007006750A01020473750A02750B0702044D
:10063000739003D6E0600764026003020473EDFF69
:100640007A01790012071CE060030206D5800312CC
:10065000118512116CE970F77404121F881206F6E6
:100660007404121F887808121F6C85080C85090D08
:10067000850A0E850B0F9003C2780C121EF67404C7
:10068000121F88780C121F5DE5084509450A450BC5
:1006900070CE8EC2E5C554E04FF5C57404121F88B4
:1006A0001206F67404121F887808121F6C85080C55
:1006B00085090D850A0E850B0F9003C2780C121E5A
:1006C000F67404121F88780C121F5DE50845094571
:1006D0000A450B70CE7A01790012071C79080204D2
:1006E0007CEC900391F07003020473750A09020414
:1006F00073790602047CE4F0A37426F0A3E4F0A36B
:10070000F022F0A3E4F0A3F0A3F0A3F0A322851855
:1007100082851983E0F8A3E0F974022274F8121BB1
:10072000CDEAFE900305E0D2E7F0E9A3F0EE9003F6
:1007300003F08E0874042AFE7C028004E062080C38
:10074000ECFA3395E0FB74022AF58274033BF583DF
:10075000EEF8C3EA98EB9400A2D265D03340DDE511
:1007600008F074012AF97A027B0312112702017141
:1007700074E9121BCD7582007583FE121E198A164C
:100780008B177514007515008A828B83E4F0900333
:10079000D6E07006D2AAD2AF800464027005790058
:1007A000120151750C00750D20750E00750F00902B
:1007B00003D6E0600464027015121185120176E917
:1007C000F874096860030208AC7900120151E06412
:1007D000027007A29240030208877508007509029B
:1007E0007808121ED07402121F37850C08850D0977
:1007F000AA08E5095407FB850E0A850F0B740B78D0
:1008000008121E87A9081218EB7402121E377E0008
:100810007F009003CAC0828E10EFF5113395E0F58A
:1008200012F513850C08850D09850E0A850F0B78C6
:10083000087910121F099003C67808121EF67583F6
:1008400003D0827808121DFA501D851882851983FD
:10085000E5822EF582E5833FF583E0F9AA14AB1516
:100860001208DB8A148B150EEE70010FC3EF940291
:1008700040A09003CE780C121EF69003D2780C1292
:100880001DFA40030207AF7900AA14AB151208DB6A
:1008900079001208DB8B159003D6E07004C2AFC25A
:1008A000AAEA451570277AA57BA58021E870030286
:1008B00007CE74066870030207CE740768700302DF
:1008C00007CE8516828517837401F080BA75820081
:1008D000758302121E197F10021D6CC008C0097CAE
:1008E000088A088B09740F7808121F4EE508F8EA89
:1008F00025E0FAEB33FBE9A2E7500474014AFAE879
:10090000A2E0500874216AFA74106BFBE9C333F952
:100910001CEC70CDD009D00822C082C083120F33E6
:1009200060030209F0A3E0F8A3E060030209F0A36A
:10093000E064027002A3E060030209F09003B8E0F3
:100940002480600914604F14605C0209F0E86003C1
:100950000209F09003B2E060047801800278009010
:1009600003C0E8F0A3E4F09003B1E0600A9003C094
:10097000E04402F0A3E4F09003A6E0640460149065
:1009800003B374C0F0A37403F0A3E4F0A3740212E1
:100990000F95F0020E6E90039FE064047052900376
:1009A000C0E4F0A380D0E8547FFA90039FE0640491
:1009B000703EEAC394065038749F2AF582E43403EB
:1009C000F583E854806018A3A3A3A3A3A3A3E064C2
:1009D0000370047801800278009003C0E88094E5F9
:1009E00082240CF58250020583E0640370E980E301
:1009F0009003A67404809B74F8121BCDE9FE90034B
:100A0000BE120F366003020AD990039FE0640460AF
:100A10000B9003BC120F366003020AD99003B8E0B2
:100A2000541F6009146030146020020AD99003BA80
:100A3000E064017022EE9003B1F060047905800259
:100A400079067A00121BCB020ADF9003BCE0547FC8
:100A5000FA9003BAE060057900020AE1EAC394065D
:100A60005077EA90620EF0749F2AF8E43403F9900C
:100A700003BCE05480602EEE600474108002744069
:100A8000906211F0EE60047B0380027B00EB8882B1
:100A90008983A3A3A3A3A3A3A3F0EE600479088092
:100AA0002F7907802BEE60047B2080027B80EB9007
:100AB0006214F0EE60047B0380027B00E8240CF5F6
:100AC00082E439F583EBF0EE6004790A800279095B
:100AD000121BCB90620EE480059003A67404F0799B
:100AE000017F01021D6C79001209F7E97003121BE6
:100AF000BA2279011209F7E97003121BC922C082D8
:100B0000C0839003BC120F367015A3120F36700FFE
:100B10009003BA120CD95480FAE9FBEA4B600790B3
:100B200003A67404801AE8906200F090039F6009A5
:100B3000E06402700C74038007E0640370037402C5
:100B4000F0020E6E74F5121BCD9003BAE0FAA3E02A
:100B50001460081460101460398057121754120C76
:100B6000B6A37B8080417900121776120CB67B8089
:100B7000E92402F9E43AFA121E6DFC1919E0FAA30D
:100B8000E92403F9E43AFA121E6DF9ECA3F0A3E9A3
:100B9000801CEAF91217E49003B3EAF0A3EBF0A388
:100BA000E4120CC5A37B00121E6DA3F0A3E4F002B7
:100BB0000C709003B3E4F0A3F0A3F0750B00900465
:100BC0007DE0FAA3E0FB020C4E850B08750900746A
:100BD000037808121F1CEA2508F8EB3509F9900381
:100BE000BA120CCFE493C0E0EFFCD0E06C705DA3D0
:100BF000E4936E70579003BC120CCFA3A3E493C090
:100C0000E0EFFCD0E06C704488828983A3A3A3E466
:100C1000936E703888828983A3A3A3A3E493F50815
:100C2000740193F5099003B3E508F0A3E509F0A377
:100C30007480F088828983A3A3A3A3A3A3E493F879
:100C4000740193F99003B6E8F0A3E9F0050B900462
:100C50007F120CD9C39AF508E99BF509740378084B
:100C6000121F4EC3E50B9508E495095003020BC90A
:100C70009003B3E0FCA3E0FDA3E0FEEC4D4E900337
:100C8000A6700474048029E0640460259003BEE02B
:100C9000FAA3E0FB9003B6E0F8A3E0F9C3EA98EB0F
:100CA0009950089003B6EAF0A3EBF09003A6740104
:100CB000F07F04021D6C9003B3EAF0A3EBF0A37481
:100CC00080120CC522F09003B3E0F9A3E0FA22E011
:100CD000FEA3E0FF8882898322E0F8A3E0F9E822FE
:100CE00074EE121BCDEA2404F8E43BF98808890964
:100CF0008882F583E4936025900481120CD9FEE983
:100D0000FF8007EE2404FE50010F8E828F83E49350
:100D1000F8740193F9EA687002EB6970E6750B00EC
:100D2000803F9062147490F07410120E3570037549
:100D30000A408E828F83A3A3A3E493550E6006E539
:100D40000AD2E0F50AE50A906215F0EA906213F023
:100D5000EC240CF582E43DF583E4F090620EF0059E
:100D60000B850882850983E493F8E50BC39840035B
:100D7000020E307A0079051216E78A0C8B0DEA45CF
:100D80000D60DCEA2402F8E4350DF9881089118839
:100D900082F583E493540FF51290620EF0750A0009
:100DA0008A828B83A3A3A3A3E4932407F50EA3E471
:100DB000933400F50F7403780E121F4EAA0EA8127A
:100DC000749F28F8E43403F9E8FCE9FD750E017519
:100DD0000F00E512780E121F1CE50EF50EE50C242F
:100DE00003F8E4350DF9851082851183E493A2E7B9
:100DF0004003020D229062117448F07408120E35FF
:100E00007003750A408E828F83A3A3E493550E600E
:100E100006E50AD2E0F50AE50A906212F0EA90626D
:100E200010F08C828D83A3A3A3A3A3A3A3020D59C7
:100E30007F0B021D6CF088828983E4935403640164
:100E400022C082C083120F337010A3120F36700AB3
:100E5000A3E064017002A3E060079003A67404801D
:100E60000C9003B374A0F0A37403120F8BF0D08323
:100E7000D0822274F3121BCD90039FE064026014B1
:100E80009003BC120F36700CA3120F36700690033D
:100E9000BBE060099003A67404F0020F2E7A00797B
:100EA00001121BCB9003BAE0606F7A00F91217763B
:100EB0008A0A8B0BEA450B605890039F7404F090EC
:100EC00003BAE09003A0F0750800850A82850B83C1
:100ED000A3A3A3A3E493F8E508C398504AA8087411
:100EE000A128F8E43403F9E8FEE9FF8E828F83E459
:100EF000F07A0079041216E78A828B83A3A3A3E415
:100F000093F88E828F83E06870E7120CE00508800A
:100F1000B99003A67404F0800E9003A0F090039F94
:100F20007403F0F91216677A007902121BCB7F0660
:100F3000021D6C9003BAE0F8A3E0F9E8492274F6C8
:100F4000121BCD90039FE0640470199003B8E06415
:100F5000817011120F33700C9003BEE064017002B7
:100F6000A3E060079003A67404801A9003BCE024F9
:100F7000A1F508A3E03403F5099003B3E508F0A355
:100F8000E509120F8BF07F03021D6CF0A3E4F0A3C0
:100F900004120F9522F0A3E4F09003A6042274F744
:100FA000121BCD90039FE0640470649003B8E0646A
:100FB00001705C9003BE120F3670549003BAE0FBD0
:100FC0009003BCE0FA9003A0E0F91217AE8A088BF8
:100FD00009AE08AF09EE4F60369003BCE0FA790322
:100FE000121BCB9003BAE0C0E09003BCE024A1F850
:100FF000A3E03403F988828983D0E0F0EEFAEFFBB6
:10100000120CE09003BCE0FA7904121BCB8006902E
:1010100003A67404F07F02021D6CC082C0838003AB
:10102000121A31A2E840F9A823E854046009782391
:10103000E654FBF612140EA823E854106009782336
:10104000E654EFF612142FA823E8A2E05005782307
:1010500054FCF690620EE0FA7404F0906214E0A280
:10106000E05039A9A8C2AF906216E0F8A3E0E8FB0F
:10107000E9A2E792AF8017906228E0C0E090039366
:10108000E0F812111CD0E0F0900393E004F0EBFDC7
:1010900074FF2DFB0470E0906214E4F0EA90620E9D
:1010A000F0E0FC7404F0906211E0A2E040319003A3
:1010B00095E0F8900394E06860257A4090039412DC
:1010C000115FE0906228F0900394E004F008900330
:1010D00095E06860041AEA70E39062117401F0EC24
:1010E00090620EF0D083D0822274F8121BCDE9FEFC
:1010F0007900801212111CE08A828B83F090039297
:10110000E00412115409900392E0F8900393E06810
:101110006005E9C39E40DD7F01021D6C748528F5E2
:1011200082E43404F58322C082C083E9FC80188AFB
:10113000828B83E0C0E090039512115FD0E0121122
:1011400054900395E004F0ECF874FF28FC0470DF81
:1011500079018090F08A828B83A3AA82AB8322E0FC
:10116000F8748528F582E43405F58322C082C083B3
:10117000900395E0F8900394E068600479018002A0
:1011800079000210E402101A74FB121EB67E009061
:1011900006857808121F6C794A1213BD9006857473
:1011A00001F0A3F0A37469F0A374A5F09003D778BD
:1011B00008121EE170047E0180159003DB7808128E
:1011C0001EE16008E59D541864107003022000EED3
:1011D000F9121334C280D291EEA2E050030212E75A
:1011E000AA18AB19120291E970030212E7C29185A5
:1011F0001882851983E0C3943C500EE0F8743CC318
:1012000098F50895E0F5098006750800750900E471
:10121000F50AF50B9003DF780C121F6C7808790C37
:10122000121AD1790612015112101A120176E9F838
:101230007409687007790612015180277407686085
:1012400016A2935012E8600874066860030212E761
:10125000A292400F0212E7750800750900750A0096
:10126000750B0085080C85090D850A0E850B0F90FE
:1012700003C27808121EF6E50C450D450E450F70A9
:10128000A7D2807907120151800312101A12116C33
:10129000E970F77E007F007401121F88E4F0A374E8
:1012A00026F0A3E4F0A3F07401121F887808121F3F
:1012B0006C85080C85090D850A0E850B0F9003C2FD
:1012C000780C121EF67401121F88780C121F5DE54F
:1012D000084509450A450B70CEA29250FCA29350D6
:1012E000F81213B8022000D280D291794E1213BDA9
:1012F000750800750900750A00750B007905120163
:101300005112101A120176E9F874096860EE74013E
:101310006870EE12101A9003E37808121EF690031C
:10132000E77808121DFA50EB1213B802200074057A
:10133000121E372274F8121BCDE9FE53BEFBE59D49
:10134000A2E650FA0078F8790100E824FF18E934A1
:10135000FFF9E84970F375C6807480659E70FA43A2
:10136000BE049062707408F01213ADEE700853F46E
:10137000FEC29043FE017403F5D575D4899003969F
:10138000E4F0A374C2F0A37401F0A3E4F0A3F0A30B
:10139000F0A37408F01213D37AFF7BFF1219EC53F9
:1013A000F4FED29043FE011213AD021117D2804316
:1013B000FD01C29143FE0222D280C29122781075B3
:1013C000B60FE5B4A2E750FAE5BBC39940F118E8BF
:1013D00070ED2274F7121BCD7A0079011217768A0C
:1013E000828B83A3A3A3A3A3A3A3E493A2E6900366
:1013F000B2500474018001E4F09003B1E4F0906213
:101400000F7403F0E0A2E750FB7F02021D6CC08264
:10141000C08390039F7402F0A3E4F09003A6F079D8
:1014200003121667752100752200D083D0822274C2
:10143000F6121BCD90620EE0FEE4F0906211E0FF28
:10144000A2E4501D7480F09003A67407F0E52145D6
:10145000226009852182852283121F979003A6E4CA
:10146000F0EFA2E2500B906211E4F09003A6F0803E
:10147000679003A6E0F87402687046906216E0FF79
:101480009003B3121DACEFF97A207B6212168174BF
:1014900003121E37EFF89003B612164512164F2F9F
:1014A000121657A3E0F8A3E0F9E8496004744080FD
:1014B000027448906211F0E849600302163B02167C
:1014C000177406687009852182852283121F979000
:1014D00003A6E060030215C2EFA2E0400302163B40
:1014E0007508B8750903750A007808121ECC7908CA
:1014F0007A207B621216817403121E3775210075E3
:1015000022009003B8E054E0601D24E0700302154F
:101510009D24E0607224C0604824E070030215A896
:1015200024E0606E0215B3A3E014602624FE601D63
:1015300024FE600A24FC601F24FE60208075120ACD
:10154000FE9003A6E06404707278608070120AF264
:1015500080EF120AE680EA120E7380E5120F9E8079
:10156000E0A3E0600E24FA600F24FE601024FE6009
:1015700011804012091980C9120B4480C4120E4117
:1015800080BF120F3E80BA7521B675221B121BB6A2
:1015900080AF7521B875221B121BB880A47521512C
:1015A00075221B121B51809975218175221B121BFC
:1015B00081808E9003A67404F0808E7840E890625B
:1015C00011F09003A6E0F874016870617F02900347
:1015D000B6E0F8A3E0F9C3E89420E994005007E8E6
:1015E000F5087F0A80037508209003B3121DACA98B
:1015F000087A207B621216AC7403121E37AC0812F4
:10160000164F2C121657A808A3121645EF90621118
:10161000F0E8C394205024E5214522600985218209
:10162000852283121F979003A6E4F0800E7405684C
:101630007009852182852283121F97EE90620EF039
:101640007F03021D6CC3E098F0A3E09400F02290A9
:1016500003B31216D9E922F9E43AFA9003B3E9F098
:10166000A3EAF0A3EBF022C082C083E99003A7783D
:1016700005F0A3D8FC9003AC7805F0A3D8FC0214C5
:101680002A74F8121BCDEAFCEBFDE9F87408121F6E
:10169000881216D460118C828D83E0121EA0E9247A
:1016A0000109E43AFAD8EF7F01021D6C74F8121BAD
:1016B000CDEAFCEBFDE9F87408121F881216D4601D
:1016C00011121E6D8C828D83F0E9240109E43AFA2F
:1016D000D8EF80D31216D9E822E0F9A3E0FAA3E00C
:1016E000FB22D083D08222C082C083E9FCEAFD7A4B
:1016F000007B00800312173290039DE0F8A3E0F90D
:1017000090047BE0687003A3E069602490039EE08E
:10171000F5838882A3E493F8EC68700D90039DE054
:10172000FAA3E0FB1217328007ED6870C8ED60C5C0
:1017300080B090039DE0F8A3E0F5838882E493F8FD
:1017400090039DE028F8A3E03400F990039DE8F0B1
:10175000A3E9F022C082C0831217657A00790112D2
:1017600016E70216E2900479E0F8A3E0F990039DF1
:10177000E8F0A3E9F02274F7121BCDE9FFEAFE12AC
:1017800017657A0079021216E7EA4B601CEF6010C9
:101790008A828B83A3A3A3A3A3E4936F70E480093D
:1017A000EEF874FF28FE0470D97F02021D6C74F5F8
:1017B000121BCDEAFF8B087A001217767A027904A1
:1017C0001216E7EA4B60188A828B83A3A3E4936F17
:1017D00070EA8A828B83A3A3A3E493650870DD7FFC
:1017E00004021D6C74F7121BCD74F0121EB6E97A58
:1017F000007B00600C146010146014146018021850
:10180000D47AF37B030218D47AF77B030218D47AD4
:101810001B7B040218D490043FE060030218D090B0
:1018200003EB7408121F377408121DD9750808F5E8
:10183000097808121ED07402121F377AE87B0779E4
:101840007F1218EB7402121E377808121ED0740A29
:10185000121F377402121F2F121C907402121E37AF
:101860008B09EA450970197509007808121ED07CA9
:101870000C7D787402121F2F121D267402121E375F
:101880007C287D00EDF8851882851983E58228F58E
:1018900082E43583F583E0FFECF8743F28F8E43404
:1018A00004F9EF1218DC88828983F0EFC41218DC87
:1018B000C0E0E824FEF582E934FFF583D0E0F00DC6
:1018C00074FC2CFCEDC3940840BA90043F742AF0D9
:1018D0007A3F7B047410121E370217A9540FFA7452
:1018E000692AF582E43404F583E02274F6121BCDF4
:1018F000890A740F550AF508750900740B780812E7
:101900001F1CEA2400F8EB3480F9E82400E93509CB
:10191000F985C709A2AFE433F508C2AFE50AC4549C
:101920000FFAE5C754F84AF5C7740A121F88E0FA9F
:10193000A3E0FB801C88828983E08C828D83F08801
:10194000828983A3A882A9838C828D83A3AC82AD74
:1019500083EAFEEBFFEE24FF1AEF34FFFBEE4F703D
:10196000D48509C7E508A2E092AF7F03021D6C741D
:10197000F7121BCDED900389F0ECA3F0A37462F095
:10198000A37473F0A3E0541FF07409121F88E0F5EC
:1019900008A3E0F509E508333354FC90038EF07496
:1019A000067808121F4EE50890038DF090038F749F
:1019B00012F0A37442F075D1FE75D601EA906271FF
:1019C000F0EBA3F0906270E0D2E1F0E0A2E740FB20
:1019D0007F02021D6CC082C083E9C333906272F043
:1019E000906270E0D2E0F0D083D0822274F7121BB4
:1019F000CD7523007524007525008A268B27EA9073
:101A0000620BF08A088B0974047808121F4EE508EF
:101A1000906207F08A088B0974097808121F4EE556
:101A200008543E906209F0758B00C2E87F02021DE7
:101A30006C74F7121BCDE59DA2E650FA906206E0A9
:101A4000F9A2E25034AA26EA90620BF0F508852745
:101A50000974047808121F4EE508906207F08A089E
:101A600085270974097808121F4EE508543E9062D4
:101A700009F0906201E0D2E0F0E9782346F6906246
:101A800002E0F50875090074047808121F1C782319
:101A9000E50846F608E50946F6906204E0F50875A3
:101AA000090074097808121F1C7824E50946F6E934
:101AB000A2E050037525017406596003752500E501
:101AC0008BA2E55006758BDF752500121BCC021A20
:101AD00027080808EAC0E0EBC0E086F0E7A4FA189F
:101AE0000986F0E7A42AFA180986F0E7A42AFA186A
:101AF0000986F0E7A42AFA1986F0E7A4FBE5F02AA4
:101B0000FA190886F0E7A42BFBE5F03AFA190886E3
:101B1000F0E7A42BFBE5F03AFA18180986F0E7A4E1
:101B2000C5F02BFBE43AFA1908E7C5F0C6A426F67F
:101B3000E5F03BFBE43AFA1886F0E7A4F6E5F00896
:101B400026F6E43B08F6E43A08F6D0E0FBD0E0FAEB
:101B500022C082C0839003B9E0F8742268700890B4
:101B600003A6E0701A80117420689003A6700DE03F
:101B7000700D121BA89003A6740280027404F080FA
:101B800043C082C0839003B9E064219003A6701320
:101B9000E07013121BA8A37407F0A3E4F09003A64F
:101BA0000480027404F0801C9003B37496F0A37454
:101BB00003F0A3E4F02280028000C082C08390037F
:101BC000A67404F0D083D0822280EF22222518C58B
:101BD00082C0E0E51934FFC583C0E0E518C39582F3
:101BE00024F910AF08858319858218800885831928
:101BF000858218D2AFCEF0A3E520F0A37808E608DE
:101C0000F0A3DEFAEFF0A3E58124FBF8E608F0A3E9
:101C1000E608F0A30808E608F0A3E608F0A315819B
:101C20001581D0E0FED0E0F815811581E8C0E0EE26
:101C3000C0E02212010002020000205104A816098F
:101C40000001020301090243000201008019090496
:101C50000000010202010005240010010424020218
:101C60000524060001052401000107058203400048
:101C70004009040100020A00000007058402400038
:101C800000070504024000004E1C0000711C00000B
:101C900074F8121BCD7408121F88E0FEA3E08015B3
:101CA000A3AA82AB838C828D83A3AC82AD83EE2406
:101CB000FF1EEF34FFFFEE4F60198C828D83E0F83A
:101CC0008A828B83E0F9E86960D6E9C398FA95E0E7
:101CD000FB80047A007B007F01021D6CE47921788F
:101CE00007B800028004F709D8FCE490030278C129
:101CF00079018002F0A3D8FCD9FA7AC27B03900064
:101D00008E78C479018015E493A3AD82AE838A8274
:101D10008B83F0A3AA82AB838D828E83D8E9D9E727
:101D2000121188121F9274F7121BCDEAF8EBF974A6
:101D300009121F88E0FEA3E0FF80188C828D83E0EB
:101D400088828983F0A3A882A9838C828D83A3AC27
:101D500082AD838E088F09E50824FF1EE50934FF54
:101D6000FFE508450970D47F02021D6C8519838543
:101D70001882E0A3FEE0A3F5207808E0A3F608DFD0
:101D8000FAE0A3FFE0A3C0E0E0A3C0E0E0A3C0E06E
:101D9000E0A3C0E010AF088582188583198008850C
:101DA0008218858319D2AFD083D082227403800039
:101DB000CCC0E0EDC0E0E518C39CCCAD1950011DCE
:101DC00010AF068C188D1980068C188D19D2AF12A1
:101DD0001DD9D0E0FDD0E0FC22CAC0E0E0A3C5825E
:101DE000CCC582C583CDC583F0A3C582CCC582C5D1
:101DF00083CDC583DAE6D0E0CA22C008C3E096F5F9
:101E00000808A3E096420808A3E096420808A3E069
:101E10009645087001D3D00822C5822518C582C511
:101E200083351910AF07F5198582188007F51985D4
:101E30008218D2AFC5832200C0D0251810AF08F594
:101E400018500C05198008F51850020519D2AFD0AA
:101E5000D0222518F58210AF08F518400C1519800E
:101E600008F51840021519D2AF85198322BB01026B
:101E7000E722C082C08389828A83BB0003E080029C
:101E8000E493D083D082226016080808C6C313C624
:101E900018C613C618C613C618C613C6D5E0EA225C
:101EA000BB000EC082C0838A838982F0D083D08237
:101EB00022BB0101F722251810AF08F518400C15B8
:101EC000198008F51840021519D2AF227403800456
:101ED00074028000C0E0F404121E52D0E0121F7B96
:101EE00022E066701008A3E066700A08A3E066703E
:101EF0000408A3E06622E026F608A3E036F608A36D
:101F0000E036F608A3E036F622E627F60809E637BB
:101F1000F60809E637F60809E637F622700422606B
:101F20000D18C6C333C608C633C6D5E0F41822253B
:101F300018FAE43519FB222518FCE43519FD227541
:101F4000D00075813F751802751903021CDC600C06
:101F500008C6C313C618C613C6D5E0F422E6F008B7
:101F6000A3E6F008A3E6F008A3E6F022E0F608A353
:101F7000E0F608A3E0F608A3E0F622CAC0E0E6F027
:101F8000A308DAFAD0E0FA222518F582E43519F52B
:101F9000832200000080FBE473FFFFFFFFFFFFFFD1
:101FA000FFFFFFFFFFFFFFFFFFFFFFFFFFFFFFFF41
:101FB000FFFFFFFFFFFFFFFFFFFFFFFFFFFFFFFF31
:101FC000FFFFFFFFFFFFFFFFFFFFFFFFFFFFFFFF21
:101FD000FFFFFFFFFFFFFFFFFFFFFFFFFFFFFFFF11
:101FE000FFFFFFFFFFFFFFFFFFFFFFFFFFFFFFFF01
:0A1FF600850609433886000000004C
:020000040003F7
:01FFF000F020
:020000040000FA
:10200000022DC4022233FFFFFFFFFFFFFFFFFFFF90
:10201000FFFFFFFFFFFFFFFFFFFFFFFFFFFFFFFFD0
:10202000FFFFFFFFFFFFFFFFFFFFFF022B3AFFFF56
:10203000FFFFFF022255FFFFFFFFFFFFFFFFFFFF34
:10204000FFFFFFFFFFFFFFFFFFFFFFFFFFFFFFFFA0
:10205000FFFFFF02216DFFFFFFFFFFFFFFFFFFFFFD
:10206000FFFFFFFFFFFFFFFFFFFFFF022A54FFFFFD
:10207000FFFFFFFFFFFFFFFFFFFFFF0228A5FFFF9E
:10208000FFFFFF0221C401FFFFFFFFFFFFFFFFFF74
:1020900010201020010020FD000200000D32000081
:1020A0000000A7319132DD314F320000D131000004
:1020B0000000000000000000000000000000000020
:1020C00000000000000006FFFFFF00035F005F004C
:1020D0003000580000000000000000000000000078
:1020E00000000000000000000000000000000000F0
:1020F00000000000C5261A271A271A271A272227A8
:10210000010104006D18000000E8030000FFFF3C1F
:102110001903E803000064006400B801A0BB0D00CF
:10212000A0BB0D0002020008000005020704010523
:102130001E02051E020A0A01080803B80B02803EAF
:102140000102FEFFE8030A050001FFFF0A1401E097
:10215000010105030101FF0F10FEFF004F00000009
:1021600000724D00000000FF000000FF00C0E0749E
:10217000F2122666A2AFE433F508D2AFAFA7AEA144
:10218000EE5F54106006122F2B75A1EFEE5F54081E
:102190006008122F3175A1F78023EEA2E092F0EFD4
:1021A000A2E082F05017906198E0F890054EE0C3ED
:1021B00098A2D265D0335002E8F075A1FE751A00DE
:1021C000E5088066C0E074F2122666A2AFE433FE32
:1021D000D2AF9061A4E0F8759B00E5915854086077
:1021E000087591F7122F798023E5915854106008F3
:1021F0007591EF122F7F8014E591A2E092F0E8A292
:10220000E082F05007E0C2E0F01230D59061A3E028
:10221000F8E5E9585404600E1230AB75E9FB9061A3
:1022200093E0A2E640F2751A00EEA2E092AF7F01C1
:10223000022722C0E074F2122666A2AFE433FED277
:10224000AF9061A5E0F8E5BF585404600675BFFB88
:102250001230ED80D1C0E074F1122666E59DA2E651
:1022600050FA906206E0F9A2E25034AA2CEA906299
:102270000BF0F508852D0974047808122DE3E508A4
:10228000906207F08A08852D0974097808122DE3F9
:10229000E508543E906209F0906201E0D2E0F0E976
:1022A000782946F6906202E0F50875090074047812
:1022B00008122D147829E50846F608E50946F69037
:1022C0006204E0F50875090074097808122D147885
:1022D0002AE50946F6E9A2E05003752B0174065978
:1022E0006003752B00E58BA2E55006758BDF752B1F
:1022F0000012361B758B00C2E87F02022722C3E45E
:1023000098F8E499F912233F8026C3E49AFAE49BF3
:10231000FBE920E7E912233FE498F8E499F922C3A6
:10232000E498F8E499F912233FE498F8E499F9C3A2
:10233000E49AFAE49BFB22EB20E7CFE920E7E0B93F
:102340000010BB0008E88AF084F8AAF022E4FBC879
:10235000FA22EB70227B10C833C8C933C933500747
:10236000C39AC3DBF280069A50012ADBEAC833F431
:10237000C8C933F4C9FA2275F008E4C833C8C933B0
:10238000C933C99AC99B5004C92AC93BD5F0ECFB93
:10239000C833F4C8E4C9FA2274F512260074FA129C
:1023A0002C0B7508047509007808122B7A74041236
:1023B0002BEB7AF87B0779031249DD7402122B8D1F
:1023C0009081227808122DD47402122E617808129E
:1023D0002C6270497508027509007808122B7A740E
:1023E00002122BEB7AF67B0779031249DD74021295
:1023F0002B8D851882851983E0F47003A3E0F460C7
:102400001C851882851983E0F8A3E0F98882898306
:102410007402F0A3F0A37469F0A374A5F0C2AF75C1
:10242000D69F0200007406122B8D7F040228E80854
:102430000808EAC0E0EBC0E086F0E7A4FA180986D5
:10244000F0E7A42AFA180986F0E7A42AFA18098600
:10245000F0E7A42AFA1986F0E7A4FBE5F02AFA19B6
:102460000886F0E7A42BFBE5F03AFA190886F0E7B6
:10247000A42BFBE5F03AFA18180986F0E7A4C5F09A
:102480002BFBE43AFA1908E7C5F0C6A426F6E5F0F6
:102490003BFBE43AFA1886F0E7A4F6E5F00826F6E6
:1024A000E43B08F6E43A08F6D0E0FBD0E0FA22126A
:1024B0002E56B9000302250FE47921780DB80002E9
:1024C0008004F709D8FCE49004D1784B7918800295
:1024D000F0A3D8FCD9FA781A9020867A01BA0002C3
:1024E0008007E493A3F608DAF97A1B7B1C9020940A
:1024F00078DA79018015E493A3AD82AE838A828B6A
:1025000083F0A3AA82AB838D828E83D8E9D9E77545
:1025100082F27583BE7406122B1C75826F75834B15
:102520007400122B1CE4CFC0E0E4CEC0E0E4CDC0C8
:10253000E0E4CCC0E075F020E626F608E633F608C5
:10254000E633F608E633F6181818EC33FCED33FDE5
:10255000EE33FEEF33FFC3EC9709ED9709EE9709D1
:10256000EF97191919400FFFEC97FC09ED97FD093A
:10257000EE97FE191906D5F0BFECF709EDF709EE55
:10258000F709EFF7191919D0E0FCD0E0FDD0E0FE13
:10259000D0E0FF222518C582C0E0E51934FFC583CD
:1025A000C0E0E518C3958224F810AF08858319852B
:1025B00082188008858319858218D2AFCEF0A3E5F2
:1025C00020F0A37808E608F0A3DEFAEFF0A3E58197
:1025D00024FAF8E608F0A3E608F0A3E608F0A3085A
:1025E00008E608F0A3E608F0A315811581D0E0FE07
:1025F000D0E0F8158115811581E8C0E0EEC0E02239
:102600002518C582C0E0E51934FFC583C0E0E51890
:10261000C3958224F910AF08858319858218800834
:10262000858319858218D2AFCEF0A3E520F0A37878
:1026300008E608F0A3DEFAEFF0A3E58124FBF8E654
:1026400008F0A3E608F0A30808E608F0A3E608F0FF
:10265000A315811581D0E0FED0E0F815811581E841
:10266000C0E0EEC0E022C0D02518C582C0E0E51968
:1026700034FFC583C0E0E518C3958224F310AF088A
:102680008583198582188008858319858218D2AFC1
:10269000C8F0A3E9F0A3EAF0A3EBF0A37908E709F7
:1026A000F0A3D8FAECF0A3EDF0A3EEF0A3EFF0A3C3
:1026B000D0E0F0A3D0E0F0A3D0E0F0A3E520F0A3B9
:1026C000E5F0F0A32212010002020000205104A84C
:1026D00016090001020301090243000201008019EA
:1026E0000904000001020201000524001001042475
:1026F00002020524060001052401000107058203EA
:1027000040004009040100020A000000070584029D
:1027100040000007050402400000E02600000327F7
:102720000000851983851882E0C0E0A3E0F9A3E0EA
:10273000FAA3E0FBA37808E0F608A3DFFAE0FCA325
:10274000E0FDA3E0FEA3E0FFA3E0C0E0A3E0C0E063
:10275000A3E0F5D0A3E0F520A3E0A3F5F010AF08C7
:102760008583198582188008858319858218D2AFE0
:10277000D082D083D0E0F8D0E032E47375F0108ED0
:10278000218F22858226858325851882851983E0FD
:10279000CEA3E0CF852682852583EBC9EAC8EDCBA1
:1027A000ECCAC3E833C8E933C9EA33CAEB33CBC355
:1027B000EA9EF524EB9FF523B35004AB23AA24EC47
:1027C00033CCED33CDD5F0DAAE21AF2222D083D099
:1027D00082ECC0E0EDC0E0E493A3FCE493A3FDED44
:1027E0004C600D122928EC24FFFCED34FFFD80EF36
:1027F000E493A3FCE493A3FDED4C600D1229FFECE0
:1028000024FFFCED34FFFD80EFD0E0FDD0E0FCE4E0
:1028100093A3C0E0E493C0E022851983851882E089
:10282000A3FEE0A3F5207808E0A3F608DFFAE0A312
:10283000FFE0A3C0E0E0A3C0E0E0A3C0E0E0A3C0ED
:10284000E0E0A3C0E010AF088582188583198008F6
:10285000858218858319D2AFD083D082022B22D0F3
:1028600083D082E9C0E0E493A3C386F0C5F095F07D
:10287000F908E493A386F0C5F095F0700BE493A3F8
:10288000C3994005E9048002A3E475F002A42582FF
:10289000F582E5F03583F583D0E0F9E493A3C0E059
:1028A000E493C0E022C0E074F2122666A2AFE433E3
:1028B000FED2AFE58AA2E2500790050FE0D2E0F029
:1028C000E58AA2E3500790050FE0D2E1F0758A0097
:1028D000C2EB7A107B0090050BE0F91233BDEEA23B
:1028E000E092AF7F01022722851983851882E0A339
:1028F000FEE0A3F5207808E0A3F608DFFAE0A3FFE6
:10290000E0A3C0E0E0A3C0E0E0A3C0E0E0A3C0E03B
:1029100010AF088582188583198008858218858301
:1029200019D2AFD083D08222C0E0C3E4939608745A
:1029300001939618400FE49366700808740193663B
:102940001870007019A3A3C3E493960874019396BA
:1029500018A3A3400DD0E0D0E0D0E0022809A3A343
:10296000A3A3A3A3D0E022D083D082C5F0E493A395
:10297000C5F0C395F0F5F0E493A3C395F04005E5E9
:10298000F0048001E475F002A42582F582E5F035BB
:1029900083F583E493A3C0E0E493C0E02274048051
:1029A000087403800474028000CCC0E0EDC0E0E550
:1029B00018C39CCCAD1950011D10AF068C188D1991
:1029C00080068C188D19D2AF122A9ED0E0FDD0E07F
:1029D000FC2274028000CCC0E0EDC0E0E518C39C8E
:1029E000CCAD1950011D10AF068C188D1980068CC6
:1029F000188D19D2AF122A7CD0E0FDD0E0FC22C0A5
:102A0000E0C0F088F0E493667008087401936618DB
:102A10007000A8F0A3A3700BD0F0D0E0D0E0D0E01D
:102A2000022809A3A3D0F0D0E022D083D082CCC06A
:102A3000E0E493A36006122ABF1470FAE493A36043
:102A400006122C371470FAD0E0FCE493A3C0E0E443
:102A500093C0E022C0E074F2122666758900C2C5F8
:102A60009019E9E0700E7A007B109005E4E0F9120D
:102A700033BD8003123CC97F01022722CAC0E0E4B3
:102A800093A3C582CCC582C583CDC583F0A3C5827F
:102A9000CCC582C583CDC583DAE5D0E0CA22CAC0E1
:102AA000E0E0A3C582CCC582C583CDC583F0A3C5B4
:102AB00082CCC582C583CDC583DAE6D0E0CA22C008
:102AC000E0E493A3D39C5010E493A3C39C400AD0AA
:102AD000E0D0E0D0E0022A47A3A3A3D0E02270090F
:102AE000080808226016181818C6C333C608C6336B
:102AF000C608C633C608C633C6D5E0EA22C008C336
:102B0000E096F50808A3E096420808A3E09642087C
:102B100008A3E09645087001D3D00822C09FF59F16
:102B2000E473D09F22D083D082C09FE493C0E0742E
:102B30000193C0E0740293F59F22C0E0C0D0E8C0CA
:102B4000E0A8A8D2AFC2C7751A00E8A2E792AFD03A
:102B5000E0F8D0D0D0E0322518F58210AF08F51893
:102B6000400C15198008F51840021519D2AF8519C7
:102B700083227404800A7403800674028002740144
:102B8000C0E0F404122B57D0E0122E012200C0D076
:102B9000251810AF08F518500C05198008F51850C5
:102BA000020519D2AFD0D022BB0102E722C082C0F9
:102BB0008389828A83BB0003E08002E493D083D0C0
:102BC00082226016080808C6C313C618C613C618A2
:102BD000C613C618C613C6D5E0EA222518F8E43590
:102BE00019F9222518FAE43519FB222518FCE435D9
:102BF00019FD22C3E0C696F608A3E0C696F608A320
:102C0000E0C696F608A3E0C696F622251810AF088F
:102C1000F518400C15198008F51840021519D2AFA7
:102C200022BB000EC082C0838A838982F0D083D009
:102C30008222BB0101F722C0E0E493A36C7009D0AB
:102C4000E0D0E0D0E0022A47A3A3D0E022E76670FC
:102C5000100809E766700A0809E76670040809E7C2
:102C60006622E066701008A3E066700A08A3E066BA
:102C7000700408A3E06622C3E09608A3E09608A3C8
:102C8000E09608A3E096A2D265D03322C3E697F679
:102C90000809E697F60809E697F60809E697F62286
:102CA000C3E493960874019396087402939608748B
:102CB00003939622C3E096F008A3E096F008A3E001
:102CC00096F008A3E096F022E026F008A3E036F0A4
:102CD00008A3E036F008A3E036F022E647F608093C
:102CE000E647F60809E647F60809E647F622E6272A
:102CF000F60809E637F60809E637F60809E637F672
:102D000022E056F608A3E056F608A3E056F608A31C
:102D1000E056F622700422600D18C6C333C608C6FA
:102D200033C6D5E0F41822E056F008A3E056F008C8
:102D3000A3E056F008A3E056F022E493F6087401ED
:102D400093F608740293F608740393F622E026F6CD
:102D500008A3E036F608A3E036F608A3E036F6222C
:102D6000E657F60809E657F60809E657F60809E6B1
:102D700057F622E4C396F608E496F608E496F608B9
:102D8000E496F622C3E09608A3E09608A3E096082E
:102D9000A3E09622C6F4C608C6F4C608C6F4C60860
:102DA000C6F4C622600D08C6A2E713C618C613C62D
:102DB000D5E0F322C3E7960809E7960809E79608E5
:102DC00009E7962275D00075813F7518D1751904F1
:102DD000000224AFE0F608A3E0F608A3E0F608A39B
:102DE000E0F622600C08C6C313C618C613C6D5E0A9
:102DF000F422E6F008A3E6F008A3E6F008A3E6F064
:102E000022CAC0E0E6F0A308DAFAD0E0FA22E0F83D
:102E1000A3E0F9A3E0FAA3E0FB22E0FCA3E0FDA31A
:102E2000E0FEA3E0FF22EAF0A3EBF0A3ECF0A3EDB9
:102E3000F022E0FAA3E0FBA3E0FCA3E0FD22ECF02B
:102E4000A3EDF0A3EEF0A3EFF022E8F0A3E9F0A3E6
:102E5000EAF0A3EBF022E5C754F84401F5C7790185
:102E6000222518F582E43519F58322122B25E5BCBD
:102E700006122B251DBD06122B256BBE06122B2517
:102E8000EFBE06122B251CB306122B25C6B3061265
:102E90002B25FFB306122B2546B406122B2509B5A8
:102EA00006122B2531B506122B2557B506122B25F8
:102EB0006BB506122B2580B506122B2589B5061297
:102EC0002B255FFA03122B258BFA03122B2533FDDA
:102ED00003122B258AFD03122B25C6FD03122B2579
:102EE000DAFD03122B25F3FD03122B25E4FE03125A
:102EF0002B25C0FF03122B25D4FF03122B25ECC377
:102F000006122B2510C406122B2529C406122B25C8
:102F100067C406122B2597C406122B25C4C40612BB
:102F20002B25CEC406122B2534C506122B2537C5FA
:102F300006122B2541C506122B254EC506122B2540
:102F4000CAB506122B25EAB506122B2529B606129C
:102F50002B2547B606122B2562B606122B25C8B6BE
:102F600006122B25D4B606122B2531B706122B25B7
:102F700055B706122B2516B806122B2523B80612B4
:102F80002B2534B806122B251BD206122B2533D243
:102F900006122B255FD206122B25918A06122B25AD
:102FA000EB8B06122B25F98B06122B250C8C0612A7
:102FB0002B25218C06122B25368C06122B25498CAD
:102FC00006122B25C58C06122B252A8D06122B25C1
:102FD000B28D06122B252A8E06122B25038F061280
:102FE0002B25138F06122B25228F06122B25E4D0BA
:102FF00006122B2508D106122B2530D106122B25BF
:1030000058D106122B2581FD02122B25A8FD021294
:103010002B25C7FD02122B252BFE02122B2552B0A9
:1030200006122B256BB006122B2577B006122B2526
:103030008BB006122B25A9B006122B25B3B00612B1
:103040002B25BDB006122B25D0B006122B255DB165
:1030500006122B25CCB106122B25FBB106122B250F
:1030600049B206122B2598B206122B25B3B20612CE
:103070002B25BDB206122B25CEB206122B2511B37D
:1030800006122B259FFF04122B25EAFF04122B2585
:1030900056D505122B2582D505122B259FD5051255
:1030A0002B25B2D505122B25CDD505122B2527D6DC
:1030B00005122B2555D605122B255BDA05122B257B
:1030C000ACDB05122B25DEDB05122B2540DC0512BF
:1030D0002B25BADD05122B25E2DD05122B25F7DDA8
:1030E00005122B2507DE05122B2547DE05122B25A1
:1030F00089DE05122B2599DE05122B25B3C6061293
:103100002B25CDC606122B25F5C606122B250EC77C
:1031100006122B2532C706122B2550C706122B2567
:1031200067C706122B2595C706122B25B0C70612B6
:103130002B25D7CE06122B251DCF06122B2549FC99
:1031400005122B2559FC05122B2560FD05122B2598
:1031500094FD05122B25B6FD05122B25D9FD051270
:103160002B25F7FD05122B2531FE05122B259AFE86
:1031700005122B25DCFE05122B2523FF05122B251E
:1031800050FF05122B2587FF05122B25649D061283
:103190002B25C69D06122B256D9E06122B25A49E5F
:1031A00006122B25C5A205122B2574A305122B256B
:1031B000A6A505122B257DA805122B250FAA051201
:1031C0002B2571AA05122B25F1AD05122B2539AF40
:1031D00005122B25E3C706122B252EC806122B2518
:1031E000288506122B25E78706122B2584880612D0
:1031F0002B25B08806122B25DE8806122B25138975
:1032000006122B253B8906122B259B8906122B259E
:103210009AF404122B259FF804122B2596FA041217
:103220002B25C4FB04122B25A4FC04122B2559FECC
:1032300004122B2525FF04122B2579FF04122B25C0
:103240006AB806122B2574B806122B2595B80612FB
:103250002B25289405122B253E9905122B25A39A80
:1032600005122B257F9C05122B25039D05122B256E
:10327000A29D05122B259B9E05122B25CD9F051285
:103280002B25E5A005122B2500A205122B25E9BA56
:1032900004122B2521BB04122B25CFC504122B258C
:1032A000CCC604122B251EC804122B257BC9041280
:1032B0002B2554CA04122B2522CB04122B2509CC12
:1032C00004122B25F8CC04122B25A0CD04122B259B
:1032D000D0CD04122B2582CF04122B25F8CF041257
:1032E0002B2511D004122B2572D104122B2530D29C
:1032F00004122B25CFD204122B2578D304122B25B0
:10330000E6D304122B2584D404122B2507D50412EE
:103310002B2525D504122B253CD604122B250AD7A4
:1033200004122B25BBD704122B257EC206122B2597
:10333000A8C206122B25BCC306122B25BFC306123A
:103340002B257DD106122B25BFD106122B2501D2AC
:1033500006122B2511D206122B25BBF505122B25A3
:10336000F9F505122B2562F605122B2581F60512BB
:103370002B259AF605122B254CF705122B2555F710
:1033800005122B25A6F705122B25DCF705122B2598
:10339000F3F705122B255FF805122B25EFF8051220
:1033A0002B2525F905122B2569F905122B25CAF9BC
:1033B00005122B25FCF905122B256FFA05122B257A
:1033C000C3FA05122B2500FB05122B2537FB05122E
:1033D0002B2549FB05122B255BFB05122B2593FBA7
:1033E00005122B25DFFB05122B251DFC05122B25B5
:1033F000538F06122B25939006122B25B69006129A
:103400002B25C79006122B25DF9206122B25FF9243
:1034100006122B25AABA06122B25DEBA06122B2578
:1034200026BB06122B2582BC06122B250080051216
:103430002B253E8105122B257A8105122B254983E8
:1034400005122B25738305122B250A8605122B25C1
:103450004A8605122B25DF8705122B257488051255
:103460002B25D28805122B25658905122B259F89CE
:1034700005122B25E18905122B25548B05122B25CE
:10348000D88C05122B25FD8E05122B252B8F0512AE
:103490002B25578F05122B25608F05122B25B68FF4
:1034A00005122B25469005122B25499305122B2535
:1034B000CB9305122B2536D006122B254CD00612A5
:1034C0002B2556D006122B25B2D006122B25079994
:1034D00006122B251D9906122B25C29906122B25A3
:1034E000019A06122B251E9A06122B254F9A0612B8
:1034F0002B259C9A06122B25D09A06122B250B9B66
:1035000006122B25E79C06122B25529D06122B2511
:1035100005C906122B255AC906122B25B4C9061255
:103520002B2522CA06122B2594CA06122B25D2CA95
:1035300006122B2513CB06122B25EAF701122B2599
:10354000F0F701122B2537F801122B2543FA01124F
:103550002B2573FA01122B25DFFA01122B259CFB78
:1035600001122B25DDFB01122B250FFC01122B254F
:1035700099FC01122B25B0FC01122B25BDFC011278
:103580002B25C7FC01122B2567FE01122B2559FFA5
:1035900001122B25B7FF01122B25C9DE05122B25A1
:1035A000DFDE05122B2591DF05122B25BBE005126E
:1035B0002B25B0E105122B254DE205122B2588E2C3
:1035C00005122B25FAE205122B2558E305122B25AF
:1035D00068E305122B258FE305122B25E1E3051285
:1035E0002B254AE505122B254FE505122B2571E504
:1035F00005122B25A0D206122B25CED206122B2582
:1036000003D306122B2505D306122B2507D306124A
:103610002B2518D306122B251AD306122B251DD3C2
:1036200006122B25EFC006122B255DC106122B2595
:103630007FC106122B25B7C106122B25EDC106123C
:103640002B253AAD06122B2581AD06122B25A4ADF4
:1036500006122B25D7AF06122B25F1AF06122B250C
:103660001CB006122B2520D306122B2546E7051287
:103670002B251FE805122B2505E905122B2516E938
:1036800005122B2527E905122B2573E905122B2599
:1036900067EB05122B25C1EC05122B25F1EC051269
:1036A0002B25B5ED05122B2513EE05122B25FFDA80
:1036B00002122B255ADB02122B25FADB02122B25D4
:1036C00077DD02122B2563DE02122B2520DF02128A
:1036D0002B2537DF02122B2586DF02122B25FADF7E
:1036E00002122B2555E002122B2568E002122B2531
:1036F000CCE002122B253BE102122B2553E10212F2
:103700002B25FEE302122B250CE502122B2567E583
:1037100002122B25BBE502122B256FE802122B2586
:10372000BFE802122B2540E902122B2582E9021282
:103730002B255CEA02122B2595EA02122B25B4EA0E
:1037400002122B25FFEA02122B251FEB02122B255A
:10375000DAEB02122B25C1EC02122B25CCEC021263
:103760002B251AED02122B256FED02122B25BBED36
:1037700002122B251FEF02122B2552EF02122B25CE
:10378000D7F102122B250AF202122B2516F3021290
:103790002B2543F302122B25BBF302122B2596F4A3
:1037A00002122B25D8F402122B254CF502122B25E0
:1037B00066F602122B25B3F602122B25BDF6021275
:1037C0002B25C0F602122B25CAF602122B25E6F68F
:1037D00002122B255EF702122B2597F702122B25DA
:1037E000B3F702122B25DFF702122B2506F802127F
:1037F0002B252AF802122B25A3F802122B2516F9E5
:1038000002122B2559F902122B2563F902122B25DE
:1038100092F902122B25A8F902122B25C4F90212E3
:103820002B25F3F902122B2513FA02122B255CFA31
:1038300002122B2597FA02122B25A3FB02122B252D
:1038400006FD02122B2525FD02122B253CFD02123E
:103850002B254EFD02122B253ACC06122B254BCCE4
:1038600006122B25D4CC06122B25008006122B2500
:103870003E8006122B25D78006122B25E2810612E8
:103880002B252A8406122B25A78406122B258FEEC2
:1038900005122B25DEEE05122B259CF005122B259B
:1038A0006FF205122B25ADF205122B2583F30512BD
:1038B0002B258CF405122B25AEF405122B250AF5C9
:1038C00005122B258BF505122B255A5100122B259D
:1038D0007C5100122B25E65200122B252F5300128B
:1038E0002B25A15300122B251F5400122B25845485
:1038F00000122B25CB5400122B253A5500122B25F4
:10390000E05500122B25555600122B259A56001211
:103910002B25AE5A00122B25C75C00122B25055D06
:1039200000122B25445D00122B255E6000122B2512
:10393000E56000122B25856200122B25BC63001266
:103940002B25CC6400122B253D6500122B251A6611
:1039500000122B259E6600122B25B26600122B2525
:103960007A6700122B25A46800122B25D16A001259
:103970002B25E46C00122B25C06D00122B255170F5
:1039800000122B25267100122B25447200122B25C4
:10399000977500122B25A77500122B25277700128B
:1039A0002B25C47700122B25E37800122B2575797F
:1039B00000122B25CC7A00122B25137B00122B250D
:1039C000C27B00122B256ED804122B250ED90412AF
:1039D0002B257AD904122B2595D904122B2538DAF8
:1039E00004122B2580DA04122B25ACDB04122B25C4
:1039F000EBDB04122B2562DC04122B25B3DC041252
:103A00002B251ADD04122B25C6DD04122B25A9E077
:103A100004122B25C2E104122B2545E204122B25AA
:103A200008E404122B25ADE404122B2557E50412FB
:103A30002B25BCE504122B252BE604122B254AE787
:103A400004122B2543E804122B258DE804122B25A4
:103A5000A4E804122B2563E904122B25A2E9041221
:103A60002B251DEA04122B25A1EB04122B2539ED81
:103A700004122B25A7EE04122B2509F004122B2586
:103A80001BF104122B25AEF104122B251CF204129B
:103A90002B252EF304122B25ACDA03122B2515DB74
:103AA00003122B255DDB03122B25A1DB03122B2533
:103AB00014DC03122B256EDC03122B25A9DC031268
:103AC0002B2543DD03122B259DDD03122B2509DF5A
:103AD00003122B2582DF03122B25ACDF03122B25CB
:103AE000C0E003122B25D4E103122B25FCE10312C5
:103AF0002B25FAE203122B250BE303122B2523E3DC
:103B000003122B2529E403122B254CE403122B2549
:103B10001BE503122B2545E503122B255CE503125B
:103B20002B2582E503122B25C1E503122B25E1E5A8
:103B300003122B2508E603122B2520E603122B2562
:103B400003E703122B255DE703122B25C4E80312BC
:103B50002B2542E903122B2566E903122B257DE96B
:103B600003122B2551EA03122B25EAEA03122B2517
:103B700010EB03122B2560EC03122B257FEC0312B4
:103B80002B25FEEC03122B2535ED03122B2573EDAF
:103B900003122B2509EE03122B257EEE03122B2593
:103BA00062EF03122B2540F103122B2515F20312AD
:103BB0002B2561F203122B256CF303122B258AF4BB
:103BC00003122B25A8F503122B25B6F503122B257E
:103BD000B2F603122B2554F703122B259AF7031282
:103BE0002B25AFF703122B25C1F803122B2562F901
:103BF00003122B25BEF903122B2559A506122B25DE
:103C000014A706122B25DCA706122B2531A80612B5
:103C10002B25B7A806122B258ECF06122B2583A1A4
:103C200006122B25C7A106122B25EDA106122B2566
:103C300014A206122B252CA206122B2544A2061232
:103C40002B255CA206122B2506A306122B2548A3C2
:103C500006122B255DA306122B2564A406122B2524
:103C60007FA406122B2588A406122B2591A40612E8
:103C70002B259AA406122B25A4A406122B2521A5D8
:103C800006122B25F87F00122B257F9806122B2574
:103C90009B9806122B25A09806122B256EBF0612A4
:103CA0002B25817C00122B25977C00122B25187E5A
:103CB00000122B25427E00122B25887E00122B2518
:103CC000917F00122B2558C506122B258ED3061284
:103CD0002B25C07F00122B25008002122B25578038
:103CE00002122B25C38002122B254F8102122B2595
:103CF000058202122B254D8202122B2566820212AA
:103D00002B25898202122B25AB8202122B25E982F8
:103D100002122B25388302122B25638302122B25D6
:103D2000C18302122B25688402122B2510850212F2
:103D30002B258C8502122B25598602122B25A08655
:103D400002122B25EC8602122B25748702122B25DA
:103D5000AD8702122B25038802122B251F88021221
:103D60002B254E8802122B255A8A02122B25888B6E
:103D700002122B25B48B02122B25E88B02122B2565
:103D8000098C02122B25188C02122B25238C02126F
:103D90002B25D28C02122B25428D02122B25CD8D84
:103DA00002122B25D58D02122B25428E02122B25B5
:103DB0007E8E02122B25448F02122B2517900212A1
:103DC0002B256C9002122B250B9102122B2565914D
:103DD00002122B25AA9102122B25439402122B25A5
:103DE000869502122B25709802122B2554990212E7
:103DF0002B25389A02122B255D9A02122B256E9ADA
:103E000002122B25E09A02122B25779B02122B25FA
:103E1000EB9B02122B25DB9C02122B25009D02122C
:103E20002B25189E02122B25369E02122B25529E00
:103E300002122B25C59E02122B25D49E02122B2581
:103E40005C9F02122B2559A002122B2566A002129C
:103E50002B256FA002122B2551A202122B257DA328
:103E600002122B258DA302122B25C8A402122B258A
:103E700047A502122B2578A602122B25B4A6021202
:103E80002B258EA802122B254BAC02122B255FACE2
:103E900002122B2569AC02122B2573AC02122B25C2
:103EA0007DAC02122B2587AC02122B25A0AC02128E
:103EB0002B25AAAC02122B2521AD02122B252CADED
:103EC00002122B255BAD02122B2583AD02122B258E
:103ED0008EAD02122B25F3AD02122B25FDAD021281
:103EE0002B2508AE02122B252CAE02122B2550AE2C
:103EF00002122B25C2AE02122B250BAF02122B256C
:103F000027AF02122B2598AF02122B25E4AF021225
:103F10002B252DB002122B256BB002122B25ECB0F5
:103F200002122B2593B102122B2558B302122B2516
:103F3000BDB302122B25EBB402122B2511B50212D0
:103F40002B2559B602122B2593B902122B2591BBB2
:103F500002122B255CBD02122B25F5BD02122B256A
:103F6000F6BF02122B25ABC002122B25E4C00212B1
:103F70002B2554C102122B255EC102122B2587C3AB
:103F800002122B258AC402122B25C7C502122B252B
:103F90001EC602122B25C9C602122B2579C8021291
:103FA0002B25C6C902122B25E6C902122B253BCAB6
:103FB00002122B253CCB02122B2564CB02122B259F
:103FC000C3CB02122B25BBCC02122B2532CD021201
:103FD0002B2545CE02122B25B3CE02122B25B2CFB4
:103FE00002122B250CD202122B2535D202122B25C0
:103FF0009BD302122B251DD502122B2574D502123C
:104000002B2522D602122B25C7D602122B252AD702
:1040100002122B25E8D702122B257AD802122B2563
:10402000D9D802122B251BD902122B254CD90212EA
:104030002B25A3DA02122B25008003122B253280B8
:1040400003122B256B8003122B25348203122B25A0
:10405000788203122B254E8303122B25AD83031286
:104060002B25C38403122B250F8503122B259D8737
:1040700003122B25818A03122B25C88B03122B25B3
:10408000608C03122B256C8C03122B25B58C03122C
:104090002B25F78D03122B25ED8E03122B25178F61
:1040A00003122B256D8F03122B25C68F03122B2590
:1040B000399003122B256F9203122B25F1930312D3
:1040C0002B25DC9403122B25269603122B255E98B4
:1040D00003122B255B9B03122B256A9B03122B25B6
:1040E000FE9B03122B25A99C03122B25EC9C03128B
:1040F0002B25359D03122B25859D03122B25E99D2C
:1041000003122B255B9E03122B25779E03122B2572
:10411000A69E03122B25E59E03122B25E09F03127A
:104120002B258FA003122B250CA303122B253EA4B5
:1041300003122B2516A503122B2598A503122B2558
:10414000CDA903122B25FCA903122B2557AA031274
:104150002B258AAA03122B2502AB03122B2535AB84
:1041600003122B2596AB03122B25E6AB03122B254E
:10417000B3AC03122B256CAD03122B2530AE03120A
:104180002B25AAB003122B250CB203122B255DB3ED
:1041900003122B2581B403122B2584B403122B2583
:1041A000B3B403122B25ABB603122B256AB7031247
:1041B0002B2599B703122B25B7B803122B257FB9EE
:1041C00003122B2540BB03122B25B0BB03122B255A
:1041D000E2BB03122B2502BC03122B2571BC031278
:1041E0002B256ABD03122B258EBD03122B2501BE84
:1041F00003122B252AC003122B2589C003122B255D
:10420000DDC003122B250CC303122B25EFC30312B1
:104210002B2577C403122B255BC503122B25E5C57F
:1042200003122B25F9C503122B250DC603122B25CE
:1042300021C603122B2535C603122B2562C6031295
:104240002B2592C603122B254DC803122B2523C9FB
:1042500003122B25C7C903122B251CCA03122B25B9
:104260007FCA03122B25C8CA03122B25EFCA0312DB
:104270002B25B7CB03122B255DCC03122B25E3CDC9
:1042800003122B256ECE03122B25B5CE03122B2540
:1042900027CF03122B257CD003122B2525D1031207
:1042A0002B2559D103122B2571D103122B2514D2A2
:1042B00003122B2590D403122B2538D603122B255D
:1042C00056D603122B2574D603122B2540D7031282
:1042D0002B258EDA03122B25A78101122B25E981CC
:1042E00001122B25568701122B25A28701122B259F
:1042F000E88701122B25398901122B259E8901128D
:104300002B25E28901122B25488B01122B25A38E28
:1043100001122B25D68F01122B25659B01122B250F
:10432000F59B01122B25DF9E01122B2544A00112C3
:104330002B25A7A001122B25C3A101122B252DA3EC
:1043400001122B250CA401122B257AA601122B2574
:104350000CA801122B259DA801122B25BCA9011226
:104360002B2549AA01122B2553AA01122B257BAA22
:1043700001122B251EAB01122B2509AC01122B2596
:10438000D1AC01122B255EAD01122B2574AD0112AB
:104390002B2591AD01122B25BAAD01122B25E7ADCE
:1043A00001122B252BB001122B25FEB001122B255B
:1043B00042B101122B25C4B101122B2565B20112A5
:1043C0002B2597B201122B25DEB201122B2511B33A
:1043D00001122B2555B301122B25A4B301122B2555
:1043E000A9B301122B2505B401122B2549B40112E2
:1043F0002B2533B501122B2598B501122B25F6B5C7
:1044000001122B2575B601122B25EDB901122B25B2
:10441000F0BA01122B2586BC01122B25C9BF01124F
:104420002B256BC001122B25B4C201122B256FC3A3
:1044300001122B25AEC301122B2572C501122B25AB
:104440008FC501122B2598C501122B25A1C501127C
:104450002B25ACC501122B25CBC501122B25EFC78F
:1044600001122B254CC801122B2556C801122B25F1
:1044700060C801122B25C3C801122B251FC90112C8
:104480002B252CCA01122B258DCA01122B259ECB60
:1044900001122B25E7CB01122B25B1CC01122B25C4
:1044A000C8CD01122B258CCE01122B25D8CF01129D
:1044B0002B25DCD001122B25D5D101122B25EDD1D6
:1044C00001122B2524D201122B252ED201122B25CD
:1044D00038D201122B2543D201122B2561D20112B1
:1044E0002B25A9D201122B2507D301122B252ED360
:1044F00001122B2540D301122B25E9D301122B25C4
:1045000022D401122B2553D501122B25B0D501122F
:104510002B25A1D601122B25D7D601122B2547D743
:1045200001122B25C3D701122B2544D901122B25AB
:104530006BDA01122B252DDB01122B25FBDB01127F
:104540002B2580DC01122B252FDD01122B2517DEF8
:1045500001122B25B0DE01122B258CDF01122B2539
:10456000F4DF01122B25B3E001122B250FE101121C
:104570002B2573E101122B2539E201122B255CE278
:1045800001122B2516E301122B2538E301122B25EE
:1045900099E301122B25C9E501122B25C2E6011270
:1045A0002B256EE701122B258BE901122B25D4E96F
:1045B00001122B251FEA01122B257BEA01122B2564
:1045C000D9EA01122B25FDEA01122B2521EB01125C
:1045D0002B2556EB01122B257EEB01122B25C3EB6D
:1045E00001122B2521EC01122B257AEC01122B252F
:1045F00074ED01122B2520EF01122B2565EF01121E
:104600002B258EEF01122B2517F001122B258AF096
:1046100001122B2598F001122B25BCF001122B253D
:1046200012F101122B252DF101122B25E8F10112B7
:104630002B2514F201122B2557F201122B25BAF269
:1046400001122B25CAF401122B25F6F401122B2599
:10465000B1F501122B2595F601122B2529F7011230
:104660002B25D6CA05122B250ECB05122B252FCBB9
:1046700005122B2571CB05122B25D5CB05122B2529
:10468000DFCB05122B25EFCB05122B2526CC0512EF
:104690002B25CFCF05122B2597D105122B257BD3A8
:1046A00005122B251DD405122B25A7D405122B2569
:1046B000508004122B25F98004122B25D881041276
:1046C0002B25E48204122B25048304122B25268437
:1046D00004122B25D68504122B25438604122B2584
:1046E000148704122B251A8804122B259288041291
:1046F0002B25CD8804122B25268904122B256189B0
:1047000004122B25AA8904122B253E8A04122B257C
:10471000D48A04122B25A98B04122B257C8C04121D
:104720002B250A8D04122B25308D04122B255D8D2F
:1047300004122B258E8D04122B255B8E04122B2543
:104740006B8E04122B25BE8E04122B25CB8E0412E9
:104750002B25D88E04122B25E18E04122B25458F94
:1047600004122B25A38F04122B25EE8F04122B2568
:10477000099004122B25309004122B254D90041221
:104780002B25599004122B25EA9104122B25039214
:1047900004122B257F9204122B25929204122B25B2
:1047A000A29204122B25469304122B25B2940412D4
:1047B0002B25C59504122B25659604122B256F9683
:1047C00004122B25EE9604122B25FF9604122B259E
:1047D0003E9704122B256C9704122B25399804124E
:1047E0002B25909804122B25C99804122B251F996C
:1047F00004122B253D9904122B258B9904122B258D
:10480000569A04122B25A49A04122B25F19A04120D
:104810002B25749B04122B259E9B04122B25D49BC5
:1048200004122B25E39B04122B25429C04122B25FA
:10483000BA9C04122B25FB9C04122B254B9D0412C1
:104840002B25769D04122B25909D04122B25AA9DC5
:1048500004122B257F9E04122B25899E04122B25E2
:10486000C49E04122B25D49E04122B25DD9E041217
:104870002B252E9F04122B25429F04122B2564A06A
:1048800004122B2577A004122B258EA004122B25B1
:10489000A3A004122B2536A104122B25AAA10412D1
:1048A0002B254FA204122B255AA204122B25BDA39F
:1048B00004122B25D9A304122B2525A404122B2581
:1048C00093A404122B25C5A404122B25DFA40412E3
:1048D0002B253FA504122B25DEA504122B2529A686
:1048E00004122B257CA804122B2514A904122B25B5
:1048F0008BA904122B25E8AB04122B2500AC041263
:104900002B2503AC04122B250FAC04122B2523AC52
:1049100004122B252BAC04122B2562AC04122B2580
:1049200056AD04122B25E0AD04122B2562AE041205
:104930002B25E2AE04122B25B9AF04122B25DBAFD9
:1049400004122B2574B004122B25D1B004122B2590
:10495000D4B004122B2501B104122B2516B1041278
:104960002B2585B104122B25D1B204122B25E4B3DB
:1049700004122B256FB404122B2582B504122B25AB
:1049800049B604122B257AB604122B25A0B60412C0
:104990002B25A9B604122B25D8B604122B2588B7CF
:1049A00004122B2538B804122B25ABB804122B2582
:1049B0004EB904122B25C1B904122B2500BA0412DA
:1049C0002B2549BA04122B257EBA04122B258BCF36
:1049D00006122B2521CC06122B25B9CB06122B252E
:1049E00035CB06122B2501CE06122B254DCD0612F6
:1049F0002B2535CD06122B2525CD06122B25E8FFBC
:104A000003122B25EC7F00122B25BDCE06122B2581
:104A10001FCE06122B250ECE06122B25DBBC05124F
:104A20002B252ABC05122B2546BB05122B2599B92F
:104A300005122B2558B905122B252FB905122B2548
:104A4000DCB805122B2535B805122B259DB70512AC
:104A50002B257BB705122B2523B705122B25E9B68D
:104A600005122B2567B605122B2526AD06122B2520
:104A700006B605122B25CBAC06122B2566AC06120A
:104A80002B25A7AA06122B25D2A906122B2559A938
:104A900006122B254BA906122B252DD006122B25ED
:104AA0002AD006122B25C1B505122B25DCB4051220
:104AB0002B2500B405122B25A8B305122B2517D0E2
:104AC00006122B2518B305122B25D3B205122B2560
:104AD000B7B205122B255CB105122B255394061293
:104AE0002B251EB105122B25C7CF06122B25F8B09A
:104AF00005122B257CB005122B259FCA05122B25EC
:104B000054CA05122B25FBC905122B25CEC9051247
:104B10002B259DC905122B256DC905122B2545C9CD
:104B200005122B25E5C805122B25C7C805122B2514
:104B30008CC805122B250CC805122B252FC4051275
:104B40002B250DC205122B25C9BF05122B2543BFEE
:104B500005122B25C8BD05122B25F1BE05122B25EC
:104B60007CBE05122B2535BE05122B2565A106003E
:104B7000000080FB8F000100DD1987000100DC19B7
:104B800035000400991C250002009D1C260002002F
:104B90009F1C27000200A11C28000100AB1C29005B
:104BA0000100AC1C84000400AD1C86000100B11C97
:104BB0002A000100B21C2B000100B31C2C000100D4
:104BC000B71C2D000800BE192E000100B81C2F00D4
:104BD0000100B91C30000100BA1C31000100BB1CEF
:104BE00032000100C61933000100C719340001006A
:104BF000BC1C36000100C81938000100BD1C39007A
:104C00000100B61C83000200D11C63000100D91909
:104C100064000100B41C65000100B51C6D000100BA
:104C2000DA1971000800B61966000100D01C4300B3
:104C30000100C11C44000200C21C45000100C41C4C
:104C400046000200C51C47000800D11948000100B9
:104C5000C71C4B000100C81C04000100D31CA100AC
:104C60000100D61C37000100D51C88000100D41CAF
:104C70003C000100C9193D000100BE1C49000200B2
:104C8000C91C67000100DB194D000200CB1C4E005F
:104C90000100CD1C4F000200CE1C3E000100D019C7
:104CA00051000100CA1952000100BF1C530001004D
:104CB000C01C54000100CB190000000000000001DE
:104CC0003636010100010201000103010001040167
:104CD000060605020000070100340801000F090460
:104CE00001010D0100FF0E0800001702000019016C
:104CF00000FF1A0100011B0100FE1C0100081D023B
:104D000000001F0100012001000121020000230119
:104D1000000F2402000026010001270100082802DC
:104D200000FF2A0100072B0102402C0100002D0189
:104D300000012E0100012F0100FF30010B1D310881
:104D400000003A0100083B01000F3C0100013D0159
:104D500000FF3E04000042040000460400004A0434
:104D600000004E04000052040000560400005A04E3
:104D700000000103710301030103010301030103A7
:104D800022030203010310030003000300030003D6
:104D9000000300030003420300032403060300038F
:104DA0000003040312032503230325032303040341
:104DB0000403000300030003440300030003230370
:104DC000000365032100350381030003050300038D
:104DD0000003000300032503230301017101010106
:104DE00001011101010131010101010180011001E5
:104DF00061013B0014006301730172016201430110
:104E00000001130106013D013500040112010001FA
:104E100000010001000104010401330133013C01E0
:104E20004401320136000001000165010001350036
:104E30008101000105018201830100010302710269
:104E400030016002110270020102020202028002BD
:104E5000100261023A0041006302730272026202B0
:104E60004302000213023800000200020402120290
:104E700000020002000200020402040237003700B0
:104E80003C024402000239000002000265020002F6
:104E9000350281020002050282028302000203043D
:104EA0007104020460041104700402040204010489
:104EB0000204100461040004140463047304720403
:104EC0006204430400041304060400040004040400
:104ED00012040004000400040004510464000004EF
:104EE00000040004440400040004000400046504F9
:104EF00000043504810464000504000483040004F4
:104F000003007100300160001100700031022003C5
:104F10005004800010006100000014006300730062
:104F20007200620043000000130006000000000051
:104F30000400120000000000000000000400040053
:104F4000370037003C024400000000000000000071
:104F500065000000350081000000050000008300AE
:104F6000000036000100060000000F0000000000F5
:104F7000000000000000000003FFFF00000403FF2A
:104F8000FF0000FFFF0FF4010005C404032000012F
:104F900000000B000000000000000003010F0000F3
:104FA0000000000000000000000000000000000001
:104FB00000000000000000000000000000000000F1
:104FC0000000053A130063391F0069391F806F39EB
:104FD0000100053A0200EB380300F1380400F7380D
:104FE0000500FD3806000939300027393100213924
:104FF000320033393300393935003F39340045390F
:1050000036004B391100573914005D3915001B3932
:10501000FFFF00000A000000020000000400000082
:105020000800000010000000200000004000000008
:1050300080000000000100000002000000040000E9
:1050400000080000001000000020000000400000E8
:10505000011D43065343084D430B6B4310E73F0AC2
:105060007D430223430541430729430C05430D11AA
:105070004364BF3DFF000007ECFDFDFDECDCDCCC34
:10508000BCACAC9C9C8C7C7C6C6C5C5C5C4C4C3C90
:105090003C2C2C1C1C03EAF5E5D5D5C5B5A595958A
:1050A0008585757565655555454535352525151530
:1050B0000500160F00000B150B020002220F330033
:1050C000000E5A6967426565416C6C69616E636583
:1050D000303901030507090B0D0F00020406080A09
:1050E0000C0D00011916181616182303003030177E
:1050F000181921301B1D1F30303016181920231AA3
:105100001C1E3000393D3F373C3C362C442D0003FB
:105110004A49434E181A2505020C0E020B040B0ACD
:105120000708000F020402010101010902E803005F
:105130000000BE040A0000E8030E0000007F001E0D
:105140001E050303000404100A0C10080C280009B3
:10515000040903010C05083108FFC082C0839019BF
:1051600034E4F0A3F07C0D7D1A7A4D7B18123531B2
:10517000123DEF124035123DF50266AB74F5122573
:105180009474F5122C0BE9FF8A08EBFE8C09EF7082
:105190005D74026508703E790812383D750A007822
:1051A0000A122B7EE509F50A780A122B7EEEF50A23
:1051B000780A122B7E90186912299D901CB1E0F993
:1051C0007CD17D19901CD11270DB123E197407122C
:1051D0002B8D0252AE7401650860030252B3790848
:1051E00012383D7B00EEFAF9123E5B0252AE7401BA
:1051F0006F600874026F60030252B3EA60067403C2
:1052000065087047790212383D901CB1E0F990189A
:1052100069122E32123E07E9F8901878E0A2E340B6
:1052200010E8700D901938E004F064047003125215
:10523000D4740365087079901939E0F9740129F084
:10524000E9C39405406A1252D48065740165087000
:105250006274016F790A702E12383D7401122E614A
:10526000E4F07402122E617403F004122E61E4F073
:10527000A3F0A3F0A3F07408122E61E4F0AA18AB17
:105280001912432F804412383D901CA712299D7A91
:10529000007B2090186DE0F91234E37404122B8D1A
:1052A000901CB1E0F9901869122E32123E3DE9F8D7
:1052B000E8601790810612299D7A017B0090186D95
:1052C000E0F91234E37404122B8D740B122B8D7FD2
:1052D00003022819901869E4F0A374F8F0A374FF8E
:1052E000F0A37407F02274F6122594E9FFEAFE7A1F
:1052F000D1F91233998A828B83E5824583702A7AA9
:10530000027B0012337BEA4B700E7A107B00901800
:105310006DE0F91233BD80148A828B8374D1F0EF73
:10532000A3F0EEF91233878003EFA3F00255357432
:10533000F712259489089004D11278C7FF901C9425
:10534000E0F47003A3E0F4702D9005E4E0901C9469
:10535000F0A3E4F080208E828F83A31263B6600FE7
:105360008E828F83A3A31263B3FAA9081238D38E57
:10537000828F83127B01EE4F70DC901C94E0F470FE
:1053800003A3E0F4600A901C94E0FAA9081238D351
:1053900012443D901837125CFF1244377F010228F7
:1053A0001974F0122594890B8C0C7509007508008E
:1053B0007410122E61126AB07412122E61126AA554
:1053C000FD804712546BF50EA3E0F50FAE08EE2EEC
:1053D000FEE433FFEA2EF582EB1276E5650E7004EB
:1053E000A3E0650F7019AE09EE2EFEE433FFEC2E3C
:1053F000F582ED3FF583E50EF0A3E50FF005090515
:105400000AE50AC3950C40BB0508E508C3950B5097
:1054100005750A0080EBA90980007F08022819742D
:10542000F4122594890B7D00740C122E61126AB05F
:1054300080010DEDC3950B502E750A008002050A00
:10544000E50AC39C50ECED25E0FEE433FFEA2EF5BF
:1054500082EB3F126CCD12546B65087004A3E065BB
:105460000970DB7901800279008014AE0AEE2EFE0D
:10547000E433FFE82EF582E9125CC222122B8D7F05
:105480000402281974F612259412551F7003A3E024
:105490006D70177508767509187808122B7AEEFA70
:1054A000123A0B7402122B8D801F75080275098049
:1054B0007808122B7A8C088D097808122B7A1255ED
:1054C00012123A2F7404122B8D806A74F6122594EE
:1054D00012551F7003A3E06D7017750883750918C6
:1054E0007808122B7AEEFA123A117402122B8D8080
:1054F0001F7508037509807808122B7A8C088D09AE
:105500007808122B7A125512123A2F7404122B8D2E
:105510008023EE240E125CBFFD7C8012675322EACA
:10552000FEEBFF12676AFCE439FD901837E06C224D
:105530007402122B8D7F0202281974F612259474BE
:10554000FE122C0BEAFEEBFF851882851983E4F02E
:10555000A3125CB7126695126AA5FBECFA888289E1
:1055600083A3A3E0F9750900750800600574FF695D
:105570007005750882803E901837E06A7003A3E0DA
:105580006B701BAA18AB19124B21E9FA851882859A
:105590001983126ABA70037508838A0980179019F3
:1055A000DCE06004640170057508818008E0640235
:1055B0007003750880851882851983126AA5FDA974
:1055C00008EEFAEFFB123A17E5096011851882859B
:1055D0001983126ABA60061270D51234230255304C
:1055E00074F2122594EAFEEBFF75080075090012AB
:1055F0006766F50AE439F50B12443DEA650A700363
:10560000EB650B7012124B0FE914F50879017A0063
:105610007B19124B0980037509801276DFF50C782F
:105620000C122B7E750C00750D19780C122B7A78E4
:1056300008122B7E780A122B7AE509F508780812F1
:105640002B7E1265321276E2F97A057B80123A1DC2
:105650007407027A3674F6122594E9FF7E008032D0
:105660008A828B83E0F508A3E0F8E4C8F9E508280E
:10567000E439F509EE25E0F8E433F9EC28F582ED9C
:1056800039F583E508F0A3E509F0EA2402FA5001B0
:105690000B0EEEC39F40C902553574E81225947471
:1056A000FC122C0B8A168B177511007402122E61D6
:1056B000E4F0A312689CF0A3F0125FFC3517125CB3
:1056C00089F50B850A82F583127BACFEE439FF85F0
:1056D0000A82850B83A3A3E0FA850A82850B83A344
:1056E000A3A3E0F9EAF508E439F509EEFAEFFB12B5
:1056F00044D9E964016016EEFAEFFB1244D9E9706F
:105700003D901837E06E7003A3E06F60311274EDC6
:10571000122B7EE4F508F5097808122B7A78081226
:105720002B7E9018371229A57508807808122B7ED9
:10573000125A6F123A1D7407122B8D025A65850A90
:1057400082850B83A3A3A3A3E0F510E50A2405F546
:105750000A5002050BE510602B127A9F12341D745B
:1057600002122E61125CFF7402122E61126ABA607C
:10577000137402122E61125A97A9101239038A0A61
:105780008B0B8003751000850A82850B83127A5477
:105790006027127A9F12341D851882851983EAF0DA
:1057A000A3EB126AC0E8496010851882851983123C
:1057B0005A97A90F1239038003750F009004D18006
:1057C00052850A82850B83A3A3A3A3A3A3A3A3E467
:1057D000F0A3F0AA0AAB0B851482851583A3A3E07E
:1057E000F81263B3F9123387851282851383E0C000
:1057F000E0A811740028F582E43419F583D0E0F0B4
:105800000511A2005007AA12AB131234238514828B
:10581000851583E0F514A3E0F515E514451570032F
:105820000259DD851482851583A31263B660DE8577
:105830001482851583A3A3A3A3A3A3A3A3E0A2E03B
:1058400050CB851482851583A3A3A3A3126ABA85BE
:105850001482851583A3A3601E1263B7FA790185AC
:105860001482851583A3A3A3A3125A8A12277A8AC6
:10587000128B13D200800F125A8AA3A3A3E0F51251
:10588000A3E0F513C200E512451370030258028528
:105890001282851383A3E065087004A3E0650960A4
:1058A0000F74FF6508700474FF65096003025802F5
:1058B000851282851383A3A3A3A3A3A3A31229A55F
:1058C000851282851383A3A3A3A3A3A3E0FC74047E
:1058D000122E611270DBA9101238E57402122B8DA2
:1058E000E9703C851282851383A3A3A3A3A3A3A37A
:1058F000A3A3A31229A5851282851383A3A3A3A31F
:10590000A3A3A3A3A3E0FC7402122E611270DBA96F
:105910000F1238E57402122B8DE97003025802E56C
:105920000F2510C333240AFA7B0012337B8A0A8BBB
:105930000BEA450B70030257E88A828B8374D212FC
:105940006CD78A828B83A3A3E8F0A3E9127A10A311
:10595000E510127BBAE50FF0E510602C1279B43532
:105960000BFB850A82850B83125CFA7402122E618E
:10597000125AA1122B76AC10EC2CFCE433FD12333E
:10598000577403122B8D800D8A828B83A3A3A3A34C
:10599000A3E4F0A3F0E50F70030257C1A810E828B4
:1059A000F8E433F9E50A28F8E50B39F9E81279B596
:1059B00039FB850A82850B83A3A3A3125CFA8518A1
:1059C00082851983125AA1122B76AC0FEC2CFCE4C1
:1059D00033FD1233577403122B8D0257D3E5116038
:1059E000251274ED122B7E750800750919780812BE
:1059F0002B7AE511F5087808122B7E9018371229BA
:105A0000A57508008029EEFAEFFB1244D9E9702F42
:105A10001274ED122B7E7508007509197808122B87
:105A20007A7508007808122B7E9018371229A5780D
:105A300008122B7E125A6F123A1D7407122B8D74A6
:105A400002122E61126ABA600B7402122E61127079
:105A5000DB123423851882851983126ABA60061214
:105A600070D51234237404122B8D7F10022819E58F
:105A7000162402FCE43517FDE516240FF582E43503
:105A800017F583E0F97A067B8022125A8E22E0F81D
:105A9000A3E0F583888222E0FCA3E0FDAA0AAB0B19
:105AA00022E0F50CA3E0F50D750E00780C2274F1E0
:105AB00012259474F4122C0B8A088B09ECFEEDFF6E
:105AC000740B122E617403F0122BE3123531124461
:105AD000378A0A8B0BAC0AAD0B7403122BE3123519
:105AE0002BE9600FEE24131276E264036010E06489
:105AF00001600B8518828519837484025C388E825C
:105B00008F83A3A3A3A3A3A3A3A3E06018F46015AA
:105B1000EE24131276E264037016EE24141276E279
:105B20006003F4700B8518828519837482025C38D7
:105B300012789BE064217002A3E06003025C0F8591
:105B40001882851983748C125CB764036003025B4E
:105B5000F97401122BEB1277A7124161E96003027D
:105B60005BF912382B8A0A8B0BEA450B7003025C37
:105B7000398E0C8F0D750E00780C122B767C157DEE
:105B8000001233577403122B8D850882850983A375
:105B9000A3E50A2415FCE4350BFD7409122A9E12B4
:105BA00074B6C0E0E50A241E125C76D0E01260DC18
:105BB000C0E0E50A241F125C76D0E0F0E50A24205C
:105BC000125C767405F0EE240BFE50010FFAEFFB29
:105BD000124A437D007C007900EEFAEFFB1239D5C2
:105BE00090810612299D7A007B1090186DE0F912C1
:105BF00034E37404122B8D8078125C7E122B7E129B
:105C00005C911241437401122B8DE9702C801412A7
:105C10005C7E122B7E125C911241497401122B8D15
:105C2000E9700D851882851983E4F01237FB80092D
:105C30008518828519837488F01274B6F50A780A7B
:105C4000122B7E7401122BDB880A890B780A122B27
:105C50007AE508240CF582E43509125C894480F564
:105C60000B780A122B7A1266051239C97405122BA9
:105C70008D740C027004F582E4350BF58322EE245A
:105C800014125CBFF50A780A22F583E0F50AA3E056
:105C900022EE240BFCE43FFD8E828F83A3A3A3A3FB
:105CA000A3A3A3A3A31271188E828F83A3A3A3A37C
:105CB000A3A3A3A3E0F922F0EE2413125CBF22F504
:105CC00082E43FF583E022C082C08374F3122C0B80
:105CD000851882851983E4F004122E61125CFF742A
:105CE00003122E61AA82AB83123CF3AA18AB1912DD
:105CF0003D2F740D122B8D0266ABA3A3A3A3A3EAC1
:105D0000F0A3EBF02274F6122594126682FAA3E057
:105D1000F9EAF890187EE058F508A3E059F509E58E
:105D2000084509601C7808122B7A9018371229A5AB
:105D30001276DFFD7C0012674F123A297404122B91
:105D40008D02553574EA12259474DB122C0B8A14DB
:105D50008B15751200751300125FFC3515F5831253
:105D600063B7F50EAC18AD197A007B00799C123E32
:105D70006D7A047900123D59EAF50C85188285196F
:105D800083E02AF0F8E50EC3984003025F6EE0C39B
:105D9000950EF509C394044003750903E50975F0F0
:105DA0001AA4FAABF012341D8A128B13EA45137051
:105DB00003025F71750D00AE12AF13850E08025E0F
:105DC000457C087D0079FF125FF1123363850A82FA
:105DD000850B83A3A3A3A3E0702D850A82850B8383
:105DE000126ABA700C1276D4F0EE24181276D780AC
:105DF00010126001F0901A7FE014C0E0125FD1D061
:105E0000E012603AE48034901A7FE004C0E0125F50
:105E1000D1D0E012602DC39403EE4003025ED11294
:105E200076C5740212602D64017003025EDEEE24FA
:105E300015126004F0EE2416126004F0EE241AFE2F
:105E400050010F050DE50DC395094003025F09E5FB
:105E500008C3950C4003025EE7AA087B00123DA729
:105E60008A0A8B0B0508901A6C126019123531855D
:105E70000A82850B83126AB0125FDFE8F0A3E91291
:105E8000604A850A82850B83A3A3A3A3A3A3A3A32C
:105E9000A3A3E0C0E0125FC7D0E0F07401122E614E
:105EA000E4F0850A82850B83126AB07402122E61B7
:105EB0001260137401122BE3123D1DE964016003AB
:105EC000025DC17404122E61125FED123531025D64
:105ED000CD12600212602D64036003025E2EEE2478
:105EE000151276D7025E34E50CC3950E4005750891
:105EF00000801DE50EC3950CF5088014126001F0BA
:105F0000EE241AFE50010F050DE50DC395095061F1
:105F1000740E122BEBAA087B007987123E6D0508E0
:105F20007418122E611260191235317410122E611C
:105F3000125FED123531EE2412F8E43FF9740E12BF
:105F40002E611270DB88828983EAF0A3EB12603A3B
:105F5000740312604A741D122E61E0C0E0125FC724
:105F6000D0E01279A7E84970931276D48091750930
:105F700000750A00780A122B7E7812122B7A7809A3
:105F8000122B7EE50EF5097809122B7E7405122E70
:105F900061E0FD7C00E5141278B33515FBE51412C1
:105FA00076CE3515F583E0F9123A657405122B8D1E
:105FB000E51245136007AA12AB131234237425129D
:105FC0002B8D7F0E022819EE2419F582E43FF5830C
:105FD00022125FD522EE2418F582E43FF58322EEEB
:105FE000125FE4222412F582E43FF58322AC82ADF5
:105FF00083EE1279B53FFB228A088B09EA127A4EAA
:1060000022EE2414F582E43FF583740122F582E444
:106010003FF583E8F0A3E9F0221276F2E8F0A3E975
:10602000F07C807D1AEE2402FAE43FFB22F0850A20
:1060300082850B83A3A3A3A3E0221277187402F036
:10604000EE2416F582E43FF58322F0EE2417F58264
:10605000E43FF5837402F0125FD574FFF02274F60A
:1060600012259474F9122C0B125FF83509127C4535
:1060700012336FEAF8EBF9ECFAEDFB85188285191B
:1060800083122E4A8E828F83A3A3A3A3E0C0E07461
:1060900004122E61D0E01279DFF87405122E6174BB
:1060A00001F07406122E617401F0901841F09018FE
:1060B0004A041277BEFAA3E0FB901842125CFFE894
:1060C00090184B1260DC901840F0AA18AB19123EE1
:1060D0000DE96003123E137407025532F0E50824FF
:1060E0000F1274BE2274F212259474FF122C0B75D9
:1060F00008007E007F0012435F8A0A8B0B12435F09
:106100008A0C8B0DA80CA90D8008050812627B1261
:106110006AB0E84970F49019DCE06007640160033C
:106120000261F112435F8A0C8B0DA80CA90D800649
:1061300012627B126AB0E8496033888289831270E8
:10614000DB901A6CE06A7003A3E06B600A12627B5A
:106150001270DBEA4B70D988828983126AB0901A78
:106160006CE0687003A3E06970030261F17A167B4A
:106170000012341D8A0C8B0DAE0CAF0DEE4F60710A
:10618000901A6C1276EE126013901A611276E9A3DF
:10619000F01244C1E98E828F83A3A3A3A3A3F0903E
:1061A0001CB21276E9A3A3A3A3A3F07C807D1A12EC
:1061B00077A7123531AA18AB197941123C218518FD
:1061C00082851983E06008901837126AB0800478DD
:1061D000FE79FF8E828F83A3A3A3A3A3A3A3126040
:1061E000131276C4E50AF0A3E50BF08E0A8F0B05B7
:1061F0000890184BE0F8E508C3985004790080290E
:10620000E508C398F9C39406400279057800800F29
:10621000E50A2414F582E4350B125C89F50B08902D
:10622000184BE0FAE8C39A40E77509007809122B89
:106230007E780A122B7AE9F5097809122B7E9018DC
:106240004BE0F5097809122B7EAD087C007A427B81
:1062500018901840E0F9123A5F7405122B8D9019CE
:10626000DCE060046401700BEE4F6007EEFAEFFBB8
:10627000123423123E137401027A36E82414F58294
:10628000E439F5832274F012259474FF122C0B8AE2
:106290000A8B0B7E008E0E8E0F125FFC125C791241
:1062A00063B7FFAC18AD197A007B00799D123E6D83
:1062B000851882851983E0F8EFC398400302635E76
:1062C000E0C39FFEC3940B40027E0AEE75F007A464
:1062D000FAABF012341D8A088B098A0E8B0FEA453F
:1062E0000F6079750C00801A850882850983A3A345
:1062F000A3A3A37403F0E5082407F50850020509D9
:10630000050CE50CC39E5056AC08AD09E50C2FFA00
:10631000E43400FB798B123E6D850882850983A3E6
:10632000A3A3A3A3E014600814601314601F80B833
:10633000850882850983A3A3A3A3A3E480B7850866
:1063400082850983A3A3A3A3A3740180A8850882DF
:10635000850983A3A3A3A3A3740280997E00750873
:10636000007808122B7E780E122B7AEEF50878084A
:10637000122B7EEFF5087808122B7E7405122E6121
:10638000E0FD7C00E50A1278B3350BFBE50A1276D6
:10639000CE125C79E0F9123A6B7405122B8DE50E82
:1063A000450F6007AA0EAB0F1234237401122B8D18
:1063B00002541A125A90A3125A8EE02274EE122539
:1063C0009474FE122C0B8A0C8B0D75100075110045
:1063D000125FFC350DF5831263B7F50AAC18AD19E1
:1063E0007A007B0079A312414F126AAAC3E50A988A
:1063F000E499507A851882851983A80AE0C398FE2B
:10640000A3E09400FFC3EE9404EF940040067E03E3
:106410007F008004EE4F6056EEFAEFFBEA75F01550
:10642000A4FAA8F075F015EBA428FB12341D8A0815
:106430008B098A108B11EA45116033750B00750EBC
:1064400000801FAC08AD09A80AE50E28FAE4340064
:10645000FB79A212414FE5082415F5085002050901
:10646000050EC3E50E9EE49F40D9EEF98005750B3D
:106470008B79007508007808122B7E7810122B7A21
:10648000E9F5087808122B7EE50AF5087808122B42
:106490007E7405122E61E0FDAC0BE50C1278B3356D
:1064A0000DFBE50C1276CE350DF583E0F9123A714D
:1064B0007405122B8DE51045116007AA10AB11125F
:1064C00034237402122B8D7F0A02281974F61225C8
:1064D0009474FF122C0BEAFEEBFFEE125FFD3F12ED
:1064E00078CCA3A3A3A3A3A3A3A3E0F9123E31E90D
:1064F000851882851983F07508007808122B7E7440
:1065000001122BDB880889097808122B7A75083567
:106510007509807808122B7A1265281239C974051A
:10652000122B8D74010255327901126532FAE43F63
:10653000FB22EE2402FCE43FFDEE240F2274F41251
:10654000259474FA122C0B125FF81272171278C786
:10655000FFEEFAEFFB123CF9E960171244378A0AA2
:106560008B0BAC0AAD0BEEFAEFFB12352BE9640195
:10657000700A7401122E61E4F0A380097401122ED6
:1065800061EEF0A3EF1279D4A3A3A3A3E0F8A2E6EF
:1065900050087403122E617401F0E8A2E7500874E9
:1065A00004122E617401F07405122E61E4F00412DD
:1065B0002BE3123E61E9851882851983F090810AE8
:1065C000122E3212445B7A007B001244677A007B01
:1065D00000124461750A00780A122B7E7401122B96
:1065E000DB880A890B780A122B7A750A34750B80BE
:1065F000780A122B7A1266051239C97405122B8D8E
:10660000740602547C7901E5082402FCE43509FD96
:10661000E508240FFAE43509FB2274F61225947478
:10662000FF122C0B126682F509A3E0F508A90912E6
:106630003E1FE9851882851983F09019DCE0700B04
:10664000740165087005A909123B2BEE240B127624
:10665000E2702C7508007808122B7E7401122BDB77
:10666000880889097808122B7A75083675098078A8
:1066700008122B7A1265281239C97405122B8D0263
:106680006523EAFEEBFF12677412668D2212669292
:10669000E022F583E0F8A3E0F98882898322C082B2
:1066A000C0839019DCE07003123B31D083D08202AA
:1066B0002B2274F412259474EF122C0BEAFEEBFFDC
:1066C000126766F508E439F509901837E065087037
:1066D00004A3E065097052A818A919880A890B78E3
:1066E0000A122B7A750A11750B00780A122B7A7C24
:1066F000007D007A817B001234A77404122B8DE98F
:106700007027750A00780A122B7E7401122BDB8821
:106710000A890B780A122B7AAC08AD0912674F125E
:106720003A237403122B8D8021750A11750B807822
:106730000A122B7A7808122B7A1276DFFD7C8412EB
:10674000674F123A2F7404122B8D741102547C126D
:10675000675322EE2402FAE43FFBEE240FF582E4B5
:106760003FF583E0F92212676A221267741266927B
:10677000127BB022EE127A4E3F2274F112259474ED
:10678000EB122C0B126682FCA3E0FAE4CAFBEC2AA3
:10679000F508E43BF509901837E065087004A3E0BC
:1067A0006509600302684388828983A3A3E094108B
:1067B000500F88828983A3A3E0851882851983807E
:1067C000088518828519837410F0E0C0E074041203
:1067D0002E61D0E01278B8A982AA83890C8A0D753F
:1067E0000E00780C122B767407122E61E0FC7D00EF
:1067F0007408122E61AA82AB831233577403122BD2
:106800008D7404122BDB880A890B780A122B7A7597
:106810000A11750B00780A122B7A7C007D007A81B0
:106820007B001234A17404122B8D7404122E61E0CB
:106830009018766005E0D2E48003E0C2E412689C20
:10684000E480088518828519837484F0E0C0E074C0
:1068500001122E61D0E0F07402122E61E508F0748E
:1068600003122E61E508F01279EC3F1274F6122B38
:106870007E7402122BDB880889097808122B7A753E
:1068800008147509807808122B7A790312652A1288
:1068900039C97405122B8D7415027004F0851882A5
:1068A0008519832274F612259474E0122C0BEAFEEB
:1068B000EBFF901A6EE064086008E0640460030275
:1068C0006A99AC18AD191239B19019DCE064027004
:1068D0002F1244377402122E61AC82AD8312352B15
:1068E000E9601D12443D8A088B09A808A90985188A
:1068F00082851983E0687003A3E0697003026A99D6
:1069000012460B7402122E61AC82AD831270D51246
:106910004509E964017003026A997418122BE312A5
:1069200044497402122E61AC82AD837418122BE3B9
:1069300012352BE9602C1244438A088B09A808A958
:1069400009851882851983E0687003A3E0696012E5
:10695000126AAA901A621260137A627B1A794B1239
:106960003C279019DCE060046401707312443D8A96
:10697000088B09A808A909EE24111276E2687003B1
:10698000A3E069605A7402122E61AA82AB83123DA1
:10699000838A088B09A808A909E8496026888289A2
:1069A00083A3A3A3A3E06401600D88828983A3A3CA
:1069B000A3A3E06402700C7402122E61AA82AB835E
:1069C000123D8F901AFC126ABA60149019D0E064DC
:1069D00001700C1270D5901AFD125A9112277A7913
:1069E000001270D5123FB1901A6C126AA5FD127098
:1069F000D51245C3740B122E61E4126AC0740C12D6
:106A00002E61126013740B122BE3123D1DE9603FDF
:106A10007C087D0079007418122BE3123363740E26
:106A2000122E61AC82AD837418122BE312352BE960
:106A3000601D7402122E61AC82AD83740E122E6141
:106A4000AA82AB83123CF3740B122BE3123D2F741A
:106A500002122E61AC82AD83740E122E61AA82AB3B
:106A600083123CF3740B122BE3123D23E9602A746A
:106A70000C122E61126AB0851882851983E0687045
:106A800003A3E0696013126AAA740C122E611260EB
:106A900013740B122BE3123D2F7420025532EAF8C7
:106AA000EBF9901936E0FCA3E02285188285198362
:106AB000126ACB22F582E438F583126ACBE84922C8
:106AC000F0851882851983126ACB22E0F8A3E0F9D9
:106AD0002274E812259474F7122C0B8A168B177FF8
:106AE000008F088F091239B78A128B13EA45137089
:106AF00003026CB57E00800DEE75F00CA4F8126CEC
:106B0000BA123D8F0E851282851383E0F8EEC3988A
:106B10004003026BEC750CFF750DFF750EFF750FD2
:106B2000FFEE75F00CA4F8A9F0126CBA123D83EADE
:106B30004B60D18A828B83A3A3A3A3E06401600D81
:106B40008A828B83A3A3A3A3E0640270B7126D9221
:106B5000700C126DBA122DD4126D9F122BF3EE75BC
:106B6000F00CA4F8A9F0E51228F582E513126DAB3C
:106B7000122AFD40837A0E7B0012341D8A0A8B0B89
:106B8000EE75F00CA4F8A9F0E51228F582E51339AA
:106B9000F583A3AC82AD83123531850A82850B83E0
:106BA000A3A3A3A3A3A3A3A3780C122DF2E50A2405
:106BB0000C125C76E4F0A3F0E5084509700E850A36
:106BC00010850B11851008851109801CE510240C17
:106BD000F8E43511F988828983E50AF0A3E50B1200
:106BE00079AFF510A3E0F5110F026B04EF7003020B
:106BF0006CAE7408122E617402126CD785188285EF
:106C000019831260137E00EF75F00CA4FAABF0123A
:106C1000341D8A0C8B0DEA450D7003026CAE805852
:106C2000850810850911EE75F00CA4F8A9F0E50CA3
:106C300028F50AE50D39F50BAC08AD09AA0AFB12D7
:106C40003531850882850983A3A3A3A3A3A3A3A3A6
:106C5000122E0E850A82850B83A3A3A3A3A3A3A34D
:106C6000A3122E4A0EE510240CF582E43511126CA5
:106C7000CDAA10AB11123423E508450970A275089E
:106C8000007808122B7E75081F7509807808122B72
:106C90007A780C122B7AEFF97405122BEBE5162497
:106CA0000FFAE43517FB1239FF7405122B8DAA1267
:106CB000AB131234237409025A67E51228F582E5F2
:106CC0001339F583A3AA82AB8322127A48F583E0B5
:106CD000F508A3E0F50922F0851682851783A3A3A2
:106CE000126ACB2274F01225941239B78A088B09E4
:106CF000AE08AF09EE4F7003026D8F750800807902
:106D0000750CFF750DFF750EFF750FFFE50875F02B
:106D10000CA4F8A9F0EE28F582EF126CC1123D83A5
:106D2000EA4B60538A828B83A3A3A3A3E064016030
:106D30000D8A828B83A3A3A3A3E064027039126D32
:106D400092700C126DBA122DD4126D9F122BF3E5B6
:106D50000875F00CA4F8A9F0EE28F582EF126DABDF
:106D6000122AFD5012E50875F00CA4F8EE28F58201
:106D7000EF126CC1123D8F05088E828F83E0F8E51B
:106D800008C3985003026D00EEFAEFFB12342302A1
:106D9000541AEA241BF582E43BF583E0640122EAFD
:106DA0002417F582E43BF583780C2239F583A3A3FD
:106DB000A3A3A3A3A3A3A3780C22127A97780C22EF
:106DC00074F112259474F6122C0BEAFEEBFF750891
:106DD00000901936126ABA70527A377B0012341D4D
:106DE000901936125CFF901936126ABA60197C3716
:106DF0007D007900123363EEFCEFFD9019361270BE
:106E0000DB123981E9700B85188285198374880239
:106E10006F6B1278A712700C7401F07C8D7D399025
:106E20001A0B1270DB124047027002E0C812700C9D
:106E30007402F0EEFCEFFD1274C7123981E9700C98
:106E40008518828519837488F0750801750A0075A4
:106E50000B19780A122B7A1270EB1229A51278A757
:106E600024281274AEFC12711D1278A72414127417
:106E7000AEF91238DF7404122B8D12701912703CA7
:106E800024311274AE604312756CFAE433FB123491
:106E90001D126A9ECC243212702E6022750C007571
:106EA0000D19750E00780C122B7612756CFCE433FC
:106EB000FD1271091233577403122B8D800C851843
:106EC000828519837488F0750801780A122B7A126A
:106ED00070DF1229A51278A724111274AEFC12716A
:106EE000001278A7242B1274AEF91238DF74041242
:106EF0002B8DE9F81278A7243412703C24341274D4
:106F0000AE6035127563FAE433FB12341D126A9ECB
:106F1000CC243512702E6042750C00750D19750E5B
:106F200000780C122B76127563FCE433FD1270F7B7
:106F30001233577403122B8DE508A2E0402512701E
:106F4000191274AE700890193612752F60157B00F7
:106F50007A007900123987027002851882851983B8
:106F60007488F08518828519837486F07409122E4E
:106F7000617402127A25F8A3E0F97401122E61E817
:106F80001278D4A31274F8122B7E7401122BDB88B2
:106F90000889097808122B7A750820750980780805
:106FA000122B7A79017406122BEBEEFAEFFB1239F1
:106FB000C97405122B8D12751E70447409122E614E
:106FC0007402127582127022122E61127586122BB3
:106FD0007E7401122BDB880889097808122B7A75D8
:106FE00008207509807808122B7A79017406122B13
:106FF000EB9019361270DB1239C97405122B8D1201
:10700000397B740A122B8D7F070228191270102207
:10701000242EF582E438F583229019361274E32485
:107020003122F5838882A3A3126ACB740122F582F0
:10703000E43CF583E8F0A3E9F0EA4B22F582E4387A
:10704000F583127047C822E9F0901936E0F8A3E002
:1070500022C082C083901936126ABA6075E0C824D3
:1070600035126AB460061270F71234231278A7241E
:1070700032126AB460061271091234231278A724FE
:1070800012126AB460091270DF1270DB123423121C
:1070900078A72415126AB4600612711D12342312E7
:1070A00078A72429126AB460091270EB1270DB12FF
:1070B00034231278A7242C126AB4600612710012CD
:1070C00034239019361270DB123423901936E4F011
:1070D000A3F00266AB8518828519831271182212FB
:1070E00074E02412F582E438F583221274E0242936
:1070F000F582E438F583221274E0243512711222ED
:107100001274E0242C127112221274E024321271D3
:107110001222F582E438F5831279CFFB221274E053
:1071200024151271122274F1122594EAFEEBFF8CE1
:10713000088D09750A018C0C8D0D750E00780C12E6
:107140002B767C177D001233577403122B8D127728
:1071500009E5082411127214E06037127A9F123484
:107160001D8A0C8B0DA80CA90D1272336021E50845
:107170002412127227122B76E508241112721C12A7
:107180005FE01270DB1233577403122B8D8003758E
:107190000A00E5082414127214E06035127A9F1276
:1071A000341D8A0C8B0DA80CA90DEE241512723615
:1071B0006055E5082415127227122B76E508241471
:1071C00012721C12720C1270DB1233577403122BE2
:1071D0008DE50AA2E0402BEE2412F582E43F126A0C
:1071E000B86009125FDF1270DB123423EE2415F54C
:1071F00082E43F126AB8600AEE12720C1270DB125F
:107200003423A90A027007750A0080CB12771E2268
:10721000E508240BF582E43509F583221274BE25B6
:10722000E0FCE433FDEE221274BEF50CA3E0F50D94
:10723000780C22EE2412F582E43FF583E8F0A3E90E
:10724000F0E8492274EE12259474ED122C0B890B90
:107250008A0E8B0F750C00750D00750AFF7510FFF7
:107260007511FF750800750900851882851983E47A
:10727000127582F9E84960177403650B60067402A1
:10728000650B7010E0C824301274AE650F6005798C
:10729000000274A97C8D7D397A007B00124047740E
:1072A00001650B700A8518828519837485803DE518
:1072B0000B60067403650B70199019361274FEF09A
:1072C0007403650B7029E50E602985188285198382
:1072D000801A7402650B701BE50E9019367005124A
:1072E00074FE80081278AA1275157402F08004E505
:1072F0000B601E1275047019127528600512701C3F
:10730000800A12752F600A1278A724341274AE1402
:10731000F01275286018126CCF12756C1279C8CAF9
:107320002432127540241D1274D42425802612752F
:107330002F6026901936E02417F508A3E03400F5F5
:10734000091275631279C8CA2435127540240612D1
:1073500074D4240E1274AEF50A7409122E617402EC
:1073600012689CE06003027410E50845097003028E
:10737000741012750470047E2280027E21850882BA
:10738000850983127026122E6112601390193AE05B
:10739000C0E01278A72430F582E438F583D0E0F01D
:1073A0007412122E617403F0AC0CAD0D740A122B22
:1073B000E3123531850882850983A3E0F50C780C4A
:1073C000122B7E780A122B7E740C122BDB880C8910
:1073D0000D780C122B7A7810122B7AE5082406F51A
:1073E0000CE43509F50D780C122B7A1274B6F97489
:1073F00009122BEBEEFA7B00123A3B7408122B8D2C
:107400007C8D7D39901A0B1270DB1240470274A7F5
:10741000901936E0F8A3E0127022122E61127586E0
:10742000122B7E7401122BDB880889097808122B35
:107430007A7508207509807808122B7A790174060C
:10744000122BEB9019361270DB1239C97405122B0E
:107450008D12751E704E1278A72419F582E438F546
:1074600083127028122E61E8F0A31270422418F5DE
:1074700082E4381274F6122B7E7401122BDB88081A
:1074800089097808122B7A75082075098078081206
:107490002B7A79017406122BEB1274C71239C97456
:1074A00005122B8D12397B790174130264C4F582A5
:1074B000E438F583E022E508240E1274BE22F5823A
:1074C000E43509F583E022901936E02417FAA3E0A9
:1074D0003400FB22F50CA3E03400F50D1274E02219
:1074E0009019361274E722E0F8A3E0C822E51624CA
:1074F0000EF582E43517F583E0F508780822127559
:107500000E74012290193612750EE0640122127475
:10751000E712751522242FF582E438F583221274C0
:10752000E0127010E0640222127572901936221275
:107530007533221274E72434F582E438F583E022AF
:10754000F582E43AF583E028F8A3E039F9E824FE6F
:10755000F582E934FFF583E0F510A3E0F511901909
:1075600036E02290193612753325E0221275722505
:10757000E0229019361274E72431F582E438F5835D
:10758000E02212704822E8F0A3127047F583888247
:10759000A3E0F508780822C082C0837B007A857951
:1075A000011239870266AB74F4122594ECFEEDFFEC
:1075B000EA1276CE3BF583127A7C127A041276EECA
:1075C000A3A3126013EA1279ED3BF5831276E9F07A
:1075D000126CCA850882F5831279BE8E828F83A3CE
:1075E000A3A3A3126014E5082402F50850020509BC
:1075F000FCAD09EE2406FAE43FFB12353185088222
:10760000850983A3A3A3A3A3A3A3A3E0C0E0127946
:10761000EC3FF583D0E0F0E5082409F508500205B9
:1076200009F5828509831279BEF8EE240F12600DE8
:10763000127709850882850983A3A3E0F8EE241157
:107640001277AF50020509E86028127A9E12341DA5
:107650008A0A8B0BA80AA90B1272336015EE24124A
:107660001276FC24111276E2F91239038A088B098A
:107670008007EE24111276D7F0850882850983E011
:10768000F81276C4E8127957858208858309602D3F
:10769000EE24141276E2127A9E12341D8A0A8B0BA3
:1076A000A80AA90BEE24151272366011EE241512E9
:1076B00076FC24141276E2F912390380041276D48F
:1076C000F002547FEE2414F582E43FF58322240F68
:1076D000F582E422EE2414F582E43FF583E422EE01
:1076E000240EF582E4125CC222127A7CA322127666
:1076F000F222E0F8A3E0F98E828F8322125CBFFCB5
:10770000A3E0FDAA08AB09EE22EE125FE4E4F0A3C9
:10771000127718E4F0A3F022F0EE12771E2224155F
:10772000F582E43FF5832274F6122594ECFEEDFF1A
:10773000126CCAAC08FDEEFAEFFB123531850882F7
:10774000850983127A67E5082409F50850020509BE
:10775000F582850983127A82F0A3E91277BEF8EEEA
:1077600024131277AF500205097403687022AC0825
:10777000AD091277A7123531850882850983A3A345
:10778000A3A3A3A3A3A3E0C0E01276C4D0E0801318
:10779000850882850983127A5FF582E43FF583E8E4
:1077A000F0A3E9F0025535EE240BFAE43FFB22F595
:1077B00082E43FF583E8F0E5082403F50822127916
:1077C0005BA3E02274F2122594EAFEEBFF750A0037
:1077D000EE24101276E2C3940C400D127A3E127819
:1077E000AA240B1274AEF50AA80AE828F8E433F9C3
:1077F000E8240DFAE439FB12341D8A088B09EA45A6
:10780000097003027894EE125FFD3F1279F3F88A53
:10781000828B83127AB6707CEEFCEFFDEA2403FAC9
:10782000E43509FB123531EE2408FE50010F1279C0
:10783000BA850882850983A3126014127210E4F0DD
:10784000E50A6050E508240DF8E43509F98E828FC9
:1078500083A3A3E0C0E0127210D0E01279E5C0E08B
:1078600012789BD0E0F0EE2404FE50010F850A0B45
:107870008E828F83126AA5FBEC88828983125D0059
:10788000E82402F8500109EE2402FE50010F150B06
:10789000E50B70DCAA08AB09027A39E508240CF57F
:1078A00082E43509F583229019361274E322FCEF45
:1078B000FDE5082402FAE4221278BC221278C022E4
:1078C0001278DDA3A3A322E0FEA3E0221271168AA0
:1078D000828B8322F0A3E9F08E828F8322F088824C
:1078E00089832274F1122594127A93E0F508A3E0BB
:1078F000850882F583E0F50BA3858208858309A3BB
:10790000A3E0F50A127A203400FB12341D8A0C8B96
:107910000DAE0CAF0DEE4F60378E828F83E50BF00E
:10792000850882850983E0FA127964E50A1279579D
:10793000A3A3A982AA83890C8A0D880E780C122B26
:1079400076AC0A127A1D3FFB1233577403122B8D4B
:10795000EEFAEFFB02700712795B22F08508828550
:107960000983A322A3E0F8E4C8F9EA8E828F83A3F7
:10797000127AC4A32274F7122594EA2413F8E43B84
:10798000F9888289831279CFF5838A82127AA612C6
:1079900079A788828983A3E0FA88828983A3127AEF
:1079A000AC12601402539C1279AFF8A3E0F92212D2
:1079B00078DDE022EA240AFAE4228E828F831279AB
:1079C000C2221279CFF9EA22F8E433F9901936E0AD
:1079D000FAA3E0221279D822127A2FA3A3A32212AB
:1079E00079D8A3E022127A2BA3A3E022EE240EF58D
:1079F00082E4221279F722F583E0FEA3E0FF8E8273
:107A00008F83E022127A09A322F08A828B83A32239
:107A1000127A1422F08A828B83A3A3A3227D00EE24
:107A20002404FAE422127A2BA3E022127A2F22F005
:107A30008E828F83A322122B8D7F06022819126754
:107A400074F58322127A4822127A4D3B22EA2413DB
:107A5000F582E422E0F50FA385820A85830B2212CA
:107A600079C2F8EE240B22A3A3A3A3A3A3A3A3127A
:107A70007A7CA3A3A3A3A3A3A3A3F022E08E828F67
:107A800083221279C28E828F83A3A3A3A3A3A3A36D
:107A9000A3A322127A9722127A4D3BF58322F8256E
:107AA000E0FAE433FB22E08C828D8322A3E0F9EA42
:107AB0008C828D83A322127A2BAE82AF8322F0EECA
:107AC0002402FE22F0A3E9127A2FA32274F61225D3
:107AD000948C088D09127A93127B011279BA8C82E8
:107AE0008D83F0A3E9127ABE50010F1278AE3509EA
:107AF000FB1235318E828F83A3A3A3127B0902551B
:107B000035126ACBE8FEE9FF22127C5AA3A3A3A395
:107B1000A3F02274F2122594127B9E75F00CA4A996
:107B2000F02401FAE439FB12341D8A0C8B0DEA456E
:107B30000D60648A828B83A38582088583098A828B
:107B40008B83E50BF0750A008046EEFCEFFDAA087A
:107B5000AB09123531EE2408FE50010F7904FAEF1B
:107B6000FB12336FEAF8EBF9ECFAEDFB850882853E
:107B70000983A3A3A3A3A3A3A3A3122E4AEE2404C1
:107B8000FE50010FE508240CF50850020509050A0E
:107B9000E50AC3950B40B3AA0CAB0D027A39127AF1
:107BA000481279F7F50BA3AE82AF8322127BB02285
:107BB0001279CFF8E4C8F9EA2822127A14A3A3A311
:107BC000A32274F61225948C088D09127A44127C33
:107BD0004512336FEAF8EBF9ECFAEDFB8508828584
:107BE0000983122E4A8E828F83A3A3A3A3E0F88574
:107BF0000882850983A3A3A3A3F0C39406500512AA
:107C00007C52803D850882850983A3A3A3A3E064F9
:107C1000FE600E850882850983A3A3A3A3E0F47008
:107C200021127C52A3F0EE2406FE50010F8508823B
:107C3000850983A3A3A3A3E0F47007127C6CF0A3CF
:107C4000E9F0025535F5831278C7FF7904EEFAEFB3
:107C5000FB228E828F83127C5A22A3A3A3A3A3E0CC
:107C6000850882850983A3A3A3A3A3228E828F8381
:107C70001279C2850882850983A3A3A3A3A3A3A322
:107C80002274F7122594E99005E4F07A107B001233
:107C900033BD7F0102281974F4122594EAFEEBFF2C
:107CA00054807054EF54107003027D99127E0D6061
:107CB00003027D437AE77B191233A58A088B09A852
:107CC00008A9099019ECE8F0A3E9F09019EEE8F0A2
:107CD000A3E9F0E849606CE0F5838882A3E07900CD
:107CE00024055001099019EAF0A3E9F0805A1231F5
:107CF000B9AA08AB091233819005E4E0F912339375
:107D00008A088B09EA450960358A828B83E0146012
:107D10001224E7601A2449601B24FE601C24D660EC
:107D2000CD80CEA3A3E0FAA3E0FB12318F80C21274
:107D300031BF80BD1232D980B812330F80B3748046
:107D4000027DCF127E0D604D9019EAE0FCA3E0FDAC
:107D50009019EEE0FAA3E0FB7900122EAD9019EA3B
:107D6000C3E09AF0A3E09BF09019EA127E10701322
:107D70009019ECE0FAA3E0FB1233819019ECE4F0E7
:107D8000A380119019EEE02AF8A3E03BF99019EED8
:107D9000E8F0A3E9F074108036EF54086009790028
:107DA00012323774088028EF5404600979011232C6
:107DB000377404801AEF5402600979021232377462
:107DC00002800CEF5401600B790312323774016F9B
:107DD000FF8031EE5480600E7A009005E4E0F912E5
:107DE00034BF74808016EE54106007123CB77410D4
:107DF000800AEE540860091231A174086EFE8004F6
:107E00007E007F00EEFAEFFB7F040228199019EC48
:107E1000E0F8A3E0F9E8492274F6122594EA240573
:107E2000FAE43400FB12337B8A828B83E58245833C
:107E30006007A3AA82AB8380047A007B007F0202E2
:107E4000281974F7122594EAFEEBFF8E828F83E0E7
:107E50002403F508F9123243A808EE28F582E43F1E
:107E6000F583E9F0EE24FFF582EF34FFF58374FE2D
:107E7000F0AC82AD837AE77B1912339F7A007B10D6
:107E80009005E4E0F9027C8F74F612259474E312F5
:107E90002C0B9019E9E0705E8518828519837401B6
:107EA000F0122E617404F07402122E617401F074E9
:107EB00003122E61E4F0A3F0740A122E61E4F0A321
:107EC000F07412122E61E4F0A3F07405122E61E436
:107ED000F07416122E617401F0741B122E6174BDC1
:107EE000F0A3743CF0AA18AB197900122EA19005EA
:107EF000E4E0F912323DE4F508F5097808122B7A2E
:107F00007C027D007A017B0F1234957402122B8D56
:107F10007808122B7A7C027D007A027B0F1234954E
:107F20007402122B8D7808122B7A7C027D007A0362
:107F30007B0F1234957402122B8D7808122B7A7CE9
:107F4000027D007A047B0F1234957402122B8D7817
:107F500008122B7A7C107D007A057B0F1234957401
:107F600002122B8D7808122B7A7C107D007A067B0A
:107F70000F1234957402122B8D12328B1232317A19
:107F8000019005E4E0F91234BF741D122B8D027EBE
:107F90003D74F7122594EA14600D14600A24FE6003
:107FA0000624F4600C80169005E4E0FA1232498051
:107FB0000C7A007B109005E4E0F91233BD027C924C
:107FC000C082C083851882851983E0F8A3E0F9E8B0
:107FD0004960128A828B83ECF0A3E824FF18E9340D
:107FE000FFF94870F2D083D082022B22022B22FFAD
:107FF000FFFFFFFFFFFFFFFF851A87C2AF022B22A3
:108000000000000000000000000000000000000070
:108010000000000000000000000000000000000060
:108020000000000000002403540049002000430029
:10803000430032003500330031002000550053006A
:108040004200200043004400430024035400650024
:10805000780061007300200049006E007300740016
:10806000720075006D0065006E0074007300A53C21
:10807000A548DB424140D740B73691389D357F3522
:10808000E9490000000000000000000000000000BE
:1080900000000000000000000000000000000000E0
:1080A00000000000000000303132333435363738FC
:1080B00039414243444546000000000000000000F2
:1080C000FFFFFFFFFFFFFFFFFFFFFFFFFFFFFFFFC0
:1080D000FFFFFFFFFFFFFFFF0000000000000000A8
:1080E0000008000400020001020502000801748279
:1080F000003A003B0000000000000000000000000B
:10810000000200020603E803000000000000000077
:10811000FF00FFFFFFFF03000000E9FFFFFF00007B
:1081200000FF09433886965118000400000019E04A
:10813000FCFFF8FF0000E71F0300805101003C0036
:108140000000100E00009F0200006AAEE7FF08006A
:108150000000FA000000040309041F000000FEFFF5
:10816000FFFF9751180060EA0000E2040000580287
:108170000000BC0200003200000000F8FF076400AD
:108180000000E90300000B0000000A0000001027B7
:108190000000000000000048000001000000300066
:1081A0000000000000000A74F7122594E9901AB943
:1081B000F0901A6EE4F0123327901AD1E4F0A3F095
:1081C000901ABAF0A3F01245AB9019DCE060046499
:1081D000017006123D53123F1B12332D9019F5E426
:1081E000F0A3F0123C5D02B40074EC12259474D735
:1081F000122C0BEAFEEBFF54806068901AB9E0F98C
:108200001233938A088B09EA4509604F7C0080018C
:108210000CEC75F003A4F8A9F0745028F5827450A2
:1082200039F583E493F4602CE493F88508828B831A
:10823000E06870DCAA08EC75F003A4F8745128F526
:1082400082745039F583E493C0E0740193F583D0D0
:108250008212277AAA08AB09123381EEFAEF648002
:1082600002872DEF5420601E1243F58A088B09EA1D
:108270004509600A124311AA08AB09123381EEFACC
:10828000EF642002872D9019DCE06402705FEEA29B
:10829000E0501F901A73E0640F701179001242E1F0
:1082A000E96009901C99122E321242F9EE64010223
:1082B0008644EF54406036901870E064067028746D
:1082C0000BF0901CB1E0F9750801750900750A0002
:1082D000750B00901A61E07808122ADEAA08AB0933
:1082E000AC0AAD0B123E3D9019CC0286EBEE542049
:1082F00070030286157A207B00901AB9E0F91234D7
:10830000F5EA4B4C4D701A901ACD122E0EE8494AE0
:108310004B700E750C01750D00750E00750F008009
:1083200061750C00750D00750E00750F0012350794
:108330008A088B098C0A8D0B901ACD122E0EE849F3
:108340004A4B602A901ACD7808122AFD400E750C0F
:10835000FF750DFF750EFF750FFF801285080C85E8
:10836000090D8C0E8D0F901ACD780C122BF3740121
:10837000780C122BC2E50C450D450E450F7003021B
:10838000853C7C0079047A007B001243BF8A088B0D
:108390000902846985188285198374FFF0740112BB
:1083A0002E6174FFF07402122E6174FF12A320FA82
:1083B000A3E0FB7403122BEB12D1B812441FE96443
:1083C00001600302844BE508240D12B0034480F8D9
:1083D000A3E0F97424122E61E8F0A3E912C511A3F9
:1083E000A3A3E0C0E07426122E61D0E012CFC0A398
:1083F000E0540860167424122E61A3E04401128731
:1084000050C0E07428122E61D0E0F0E50812ED5C57
:10841000350912CF99601CE508240F12CC88A3E01F
:10842000C812C4D938F583E0F87412122E61E8F04E
:10843000A3E4F090810A12299D7404122BEB7407B7
:10844000122BE3123E7F7404122B8D85088285095E
:1084500083A3A3A3A3A3A3A3A3A37406128750F982
:108460001243A1850A08850B09E508450970030236
:10847000853C7C007904AA08AB091243BF8A0A8BA9
:108480000B850882850983A3A3A3A3E0F510A3E0CD
:10849000F511E4F512F513780C7910122DB4402380
:1084A000E5082404F8E43509F9850C10850D1188D8
:1084B000828983C3E09510F0A3E0951112F1DF707B
:1084C000A2800E850882850983A3A3A3A3E4F0A359
:1084D000F0850882850983A3A3A3A3A3A3A3A3A3D1
:1084E000A3E06401850882850983A3A3A3A3A3A3B2
:1084F000702BE0540460030283948508828509830D
:10850000A3A3A3A3A3A3A3A3A37406F07AB7850888
:10851000828509831289331242F3028463A3A3A3E1
:10852000A3E06003028394850882850983A3A3A343
:10853000A3A3A3A3A3A37401F002846312438F7CBB
:108540000079017A007B001243BF8B09EA4509607C
:108550000C7A207B00901AB9E0F91233BD850C0A21
:10856000850D0B7C0079047A007B001243BFEA4B37
:10857000701580558A828B83A3A3A3A312E69BE583
:108580000898E5099940098A828B83A3A312874240
:108590007C0079041243BF8B0DA90DEA4970D5C345
:1085A000E50A9508E50B95095013C3E508950AF50A
:1085B00008E509950BF509E508450970147A207B53
:1085C00000901AB9E0F91233BD901ACD129B4C807D
:1085D0003FE50825E0F508E50933F509E4F50AF576
:1085E0000B7808122B727A207B00901AB9E0F912EE
:1085F00034E37404122B8D123507EAC0E0EBC0E0BF
:10860000ED901ACDFBECFAD0E0F9D0E0F8122E4A4A
:10861000EE6420802FE0600764016003028706EEAD
:1086200054106008123F57EE64108018EE544060FA
:1086300008123FCFEE6440800BEE5480600B123E78
:1086400025EE6480FAEF02872DEF5401600B12458E
:1086500081EEFAEF640102872DEF54086047123F64
:10866000279019C6E0640170349019C7E0602EF5B8
:1086700008E4F509F50AF50B908106780C122DD463
:108680007808790C12242F7808122B727A007B0854
:10869000901AB9E0F91234E97404122B8DEEFAEF56
:1086A000640802872DEF54106012901ACBE0600529
:1086B000E4F0123F27EEFAEF64108071EF5440604F
:1086C00045901AF212CF9B60369019D0E064017089
:1086D0002E901AF312C8BD12277A901AF812CF9B67
:1086E000600612C8BD12277A90810612299D7A0071
:1086F0007B40901AB9E0F91234E97404122B8DEE24
:10870000FAEF64408027EF5402600A12457BEEFACC
:10871000EF64028018EF5404601612CE6F79019056
:108720001A6C12CC9C123E9DEEFAEF6404FB80049E
:108730007A007B007429122B8D7F0C0228198E82FF
:108740008F83A3A312874822E0F508A3E0F509224E
:1087500012C515A3E022C082C08374EA122C0B7CE0
:10876000167D007900AA18AB191233637408122E13
:10877000617402F0901A62129B1F1287967409129C
:108780002E6112CCAB7413122E61E412CFD2123CC4
:108790004B741602D58BE8F0A3E9F0901A6C12D551
:1087A0004E2274F712259474DA122C0BEAFEEBFFBA
:1087B000EE4F602DAC18AD1912441F7406122E61D5
:1087C000E0601E7417122E61E0FD7401122E61E04C
:1087D000FCEEFAEFFB79001242B7E9600479A4805D
:1087E000027900742602B3FD74F4122594EAFEEBBC
:1087F000FF8E828F83A3A3A3A3A3A3E05440601999
:1088000012E2FD12CC9C1244D9E960077AFF7BFF8B
:108810000288DD12E2FD0288D09019DCE060076476
:108820000160030288C5901A59E0A2E14003028862
:10883000C512B44312CD9BA3A3A3A3E0FA888289F7
:1088400083A3A312D91A8E828F83A3A3A3A3A3A366
:10885000A3E054106004794080027900750AFE7527
:108860000BFF780A122B7A1289211229A5AC08ADC8
:108870000912E2FD12CC9C123F2D7404122B8DE5DF
:10888000086A7003E5096B600B12BF5A6A7003A394
:10889000E06B703F750A00780A122B7E79028E8297
:1088A0008F8312B504FCA3E0FDAA08AB0912451B97
:1088B0007401122B8D7508CDAA0812892F1242F36C
:1088C000E9604C80579019DCE0640270E8901A620D
:1088D00012CC9C74FE6A700374FF6B60D812E2FDC8
:1088E00012E16D1244D9E98E828F83600B12BC783D
:1088F00012F4B1E4F0A3800312F49FF07CE77D4210
:108900008E828F8312CC9C123C51E9F50870A9EE3F
:108910004F60097901EEFAEFFB12439BA908028F21
:10892000D1EE128926222411F582E43FF583228EAE
:10893000828F8312F488E0F92274F6122594E9FEFE
:10894000EAFF7A0F7B0012337BEA4B601F8A828B2F
:1089500083740CF0EEA3A3F0EF8A828B8312B1B97B
:10896000901AB9E0F91233877900802FEEF912439B
:10897000C58A088B09A808A909E849601C8882896A
:1089800083A3A3A3A3A3A3A3A3A3740612ED62E0EE
:10899000F9123FE1EEF91243A1791002C91A74F4F9
:1089A0001225948A088B098C0A8D0B901A73E06447
:1089B0000F702CEA4509450A450B6023901A6EE0BA
:1089C00064086005E0640470167808122B727A015E
:1089D0007B00901AB9E0F91234E37404122B8D0273
:1089E0008FD174F2122594EAFEEBFF8C0A8D0B896D
:1089F00008740E122E6112E6A0850C82F583E4F055
:108A0000A312CE64F5838882E0F91244B5E96026AA
:108A100012CC8F1244D9E96402701B8E828F83A31B
:108A2000A3A3A3A3A3A3A3A312BAE5850C82850DD8
:108A30008312CCAB800375080012B4FB14602E14B3
:108A4000604314606414606C146048147003028AFC
:108A5000D424FE7003028AEE147003028AF71470A5
:108A600003028B0A147003028B18028B2E780C12EF
:108A70002B7AAC0AAD0BEEFAEFFB123F3F740212F9
:108A80002B8D028B13AC0AAD0BEEFAEFFB123F45B8
:108A9000028B3812CC8F1244D9E96003028B2EEE80
:108AA000FAEFFB123F93028B38A908EEFAEFFB12A4
:108AB0004521805F12B97964027073E508700A126B
:108AC000E2237003A3E069706FEEFAEFFBA90812CE
:108AD00044A9803F12E2237003A3E069705012B9E9
:108AE0007964027049EEFAEFFB124491804AEEFA83
:108AF000EFFB12459F804112E2237003A3E06970EF
:108B00002DEEFAEFFB12452D802EEEFAEFFBA908B1
:108B1000124539E9F50880209019D0E06401700908
:108B2000EEFAEFFB124545800F750800800A7508C4
:108B3000007AD37B00123873A9088007A90A74034E
:108B4000122B8D7F0602281974F412259474D61204
:108B50002C0B8A088B098A828B83A3A3E0F912432A
:108B6000C58A0A8B0BAE0AAF0BEE4F7003028C7AEC
:108B7000850882850983A3A882A983E0C0E012CC7E
:108B800076D0E012E6ADE064F160338508828509B5
:108B900083A3E064CD6027850882850983A3E06410
:108BA0001A601B850882850983A3E064E9600F854C
:108BB0000882850983A3E064E16003028D72901945
:108BC000DCE0600764016003028C9B8E828F83A3CC
:108BD000A3A3A3A3A3A3E054087003028C9B8E82DB
:108BE0008F83A3A3A3A3A3A3A3A3A37405F09019A6
:108BF000DCE0600464017053850882850983A3E08A
:108C000064E96047901AEE12CF9B600612C8BD124D
:108C1000277A901AF012CF9B6031901A59E0A2E1A6
:108C2000502912D18EA3A3A312B9B78882898312C7
:108C3000CC9C1245DBEA4B6012850882850983A330
:108C4000E0F9901AF012E30112277A8E828F83A343
:108C5000A3A3A3A3A3A3A3A3E0640270108E828F97
:108C600083A3A3A3A3A3A3A3A3A37406F08508824D
:108C7000850983A3A3E0F91243A112438F9019DC65
:108C8000E064027011901C9FE0F508A3E0AA08FBC5
:108C9000E4FCFD1242F9742A028FCE790012439B44
:108CA000E97003028D729019DCE0600764016003D3
:108CB000028D47901A59E0A2E14003028D4712CF7E
:108CC000967003028D478E828F8312CC9C7404129F
:108CD0002BEB12D1B812441F850882850983A3E0CB
:108CE00064E97023128E7C122B7E850882850983AD
:108CF000A3E0F50A780A122B7E128E8912CC9C1200
:108D000044557402122B8D740D122E6112CF8C12E9
:108D1000F10A12CCAB7409122E61E0600479408034
:108D2000027900740F122E6112B9B7740D122E6100
:108D300012CC9C123F39E9600E8E828F83A3A3A3CD
:108D4000A3A3A3E04420F0EE2404F50AE43FF50BCE
:108D50008E828F8312B010E0F9850A82850B831210
:108D6000CC9C123339850A82850B83EAF0A3EB028F
:108D70008BED850882850983A3E0C0E07402122E82
:108D800061D0E012A80012E109E508240B12B0033B
:108D9000C0E07403122E61D0E012E970E0AA18ABB3
:108DA000197031123E799019DCE06004640170277B
:108DB0007402122E61E0701F12E2FD12CC9C12446C
:108DC000D9E97039901AEE12CF9B603112C8BD12EA
:108DD000277A80031244AF7402122E61E064E970B6
:108DE0001C128E7C122B7E750AE9780A122B7E12D9
:108DF0008E8912CC9C1244557402122B8D9019DC72
:108E0000E0600764016003028C4B901A59E0A2E114
:108E10004003028C4B8E828F83A3A3A3A3A3A3A39F
:108E2000A3A3E06402703C8E828F83A3A3A3A3A3B9
:108E3000A3E05404602D12E2FD12CC9C1244D9E947
:108E40008E828F83700F12E30174FFF0A312A9B01A
:108E50007405028C6CA3A3A3A3A3A3A3A3A374036D
:108E6000028C6C850882850983A3E064E9600302B3
:108E70008C4BEEFAEFFB124557028C4B8E828F83A0
:108E800012DA50750A01780A22E508240C12BF791B
:108E9000E0F98A828B83A3A3A3A3A3A3A3A3A31212
:108EA000D9122274F4122594EAFEEBFF75080075BE
:108EB00009008E828F83A3A3A3A3A3E0603B750860
:108EC0000812CC8F79FF1240E38B0BEA450B601040
:108ED00075082C8E828F83A3A3A3A3A3E0D2E0F016
:108EE0008E828F83A3A3A3A3A3E054036401600332
:108EF000028FAD430811028FADEE241812B97C60C9
:108F000049EE241A12B97C6003F4701D12E223703A
:108F100003A3E0697006750822028FAD901A6EE017
:108F200064046003028FAD801CEE241BF582E43FD5
:108F300012B9C5241A12B97CFAEE2419129BDC125C
:108F40003FA5E97068750901806312CC8F1244D97E
:108F5000E96402700375080112E2237003A3E0695B
:108F60007006E508D2E1F508E50860158E828F836A
:108F7000A3A3E07006E508D2E58004E508D2E6F593
:108F80000812CC8F1244D9E964017006E508D2E0DA
:108F9000F5088E828F83A3A3E0601212B4FBF9124E
:108FA00044B5E964016006E508C2E0F5089019DC03
:108FB000E0600464017012E508A2E1400CE509A23A
:108FC000E04006E508D2E7F50802891C7418122B68
:108FD0008D7F0402281974EC12259474C3122C0B93
:108FE000EAFEEBFF85188285198374FEF0A304F076
:108FF0007510007511007509009019DCE0640270AD
:10900000248E828F83A3A3A3A3E06019901C9D12DA
:10901000CF9B6011901C9DE0F50AA3E0AA0AFBE437
:10902000FCFD1242F97405122BEB8E828F83A3A3F1
:10903000A312CF8E12CC9A12441FE970030294122D
:1090400078017407122E61E0C39402400278007424
:1090500009122E61E0C3940240027800740E122EB1
:1090600061E064F87003A3E0F47003029412740EDC
:10907000122E61E064F97003A3E0F470030294120D
:10908000740E122E61E064FA7003A3E0F470030220
:109090009412740E122E61E064FB7003A3E0F4706E
:1090A000030294127408122E61E0F9901A5CE069D0
:1090B0006003029412E8A2E040030294129019DCCB
:1090C000E06402700B7429122E61E06003029412B6
:1090D00012BADC7424122E6112B9E6241C12BADF13
:1090E0007412122E6112CCAB740B122E61E0601D53
:1090F000741C122E61E0FD7406122E61E0FC8E825B
:109100008F8312CC9A79011242B7E9703D7405122F
:109110002BE312430BE9F508740B122E61E0702F5C
:10912000901A56E060297422550864226021744226
:109130005508644270147422122E61129AF8600F5E
:109140007422122E61129AFE60057ACF029414E9FD
:10915000A2E6506C9019DCE060046401701B901A68
:1091600059E0A2E150137422122E6112B504122AA2
:109170002A01010B97910012947422122E6112B5EC
:109180000424FD601214600F24FD600B24FD6007B1
:1091900024FE60030294127422122E61129B377017
:1091A0000F7422122E61A312C8BDA3E0640D6010DB
:1091B0007405122BE3124515E964017003029AE16C
:1091C000EE242DF582E43FF58312A3137003A3E090
:1091D000697021750A00780A122B7E780A122B7E9C
:1091E000EE242F129BDC129B0412CC9C124455746B
:1091F00002122B8D740B122E61E070030292A312E7
:109200009B0412CC9C1245DB8A0A8B0BEA450B703F
:109210000302933A7406122E61E0F88E828F83A3C4
:10922000A3E028F8A3E03400F9E8240D129AE6F848
:109230008A828B83A3A3A3E068600EE88A828B8373
:10924000A3A3A312B1A7129B4C79047406122E613A
:1092500012A663E02AF8A3E034008882F583A3AA6B
:1092600082AB8312336F8A0C8B0D8C0E8D0F850AA7
:1092700082850B83A3A3A3A3780C122AFD400302CB
:109280009AE190819A780C122D4D850A82850B8384
:10929000A3A3A3A3E50CF0A3E50DF0A3E50EF0A3B3
:1092A000E50FF09019DCE0640260030293E7901A86
:1092B0006EE064046008E064096003029AE1E50876
:1092C000A2E54003029375EE242F12B97CC0E0742E
:1092D00002122E61D0E0129B5DC0E07403122E6179
:1092E000D0E0129B55C0E07404122E61D0E0F074FF
:1092F00016122E61E0640170267410122E61129B0A
:10930000147003A3E0697017740E122E6112CC9CC6
:109310001244D9E9640270077416122E61E4F01247
:109320009B4212299D7406122BEB7409122BE31237
:109330003E7F7404122B8D029AE1901AB3E064010F
:1093400060030292A37422122E61129AF87009E54A
:1093500008A2E650030292A37412122E61E0F47088
:1093600003A3E0F4600CEEFCEFFD7405122BE31296
:109370004317029AE1A2E64003029AE17422122EF8
:109380006112D19B7016741C122E61E0640270543D
:109390007405122BE379001244A980487422122E1E
:1093A00061129AFE7014741C122E61E06404703411
:1093B0007405122BE312449D802A7422122E61122E
:1093C0009B37700C79007405122BE3124521801431
:1093D0007422122E6112B506640C70087405122BEB
:1093E000E3124551029AE1E0600764016003029ACA
:1093F000E1901A59E0A2E14003029AE17429122E89
:1094000061E060267410122E6112CC9C123D71E94D
:10941000700A7AD37B00123873029AE18E828F83AE
:10942000A3A312E301A3E0C2E5F07416122E61E0DB
:10943000601DEE2402F8E43FF9E8FAE9FB12D1A13D
:1094400014F012D1A1F87416122E61E8F07006E53E
:1094500008C2E7F508E508A2E35061751110A2E221
:109460005018740A122E61E054E3F0740A122E614F
:10947000E0131313541FF8E0802CA2E4502A740A5E
:10948000122E61E01313543F5407F8600974076803
:10949000600B18E87007C3E508C2E7F508E8333346
:1094A00054FCF8E054E348F0740A122E61E0C0E086
:1094B0008E828F83A3A312B0EED0E0F0901A6EE0FC
:1094C00064046008E064096003029598740E122E2B
:1094D0006112E2307003A3E069601F740E122E6106
:1094E00012CC9C1244D9E96402600F740A122E61F6
:1094F000E0540364016003029AE17407122E61E0F4
:109500007041EE242F12B97CC0E07402122E61D09B
:10951000E0129B5DC0E07403122E61D0E0129B55F7
:10952000C0E07404122E61D0E0129B3D12299D749C
:1095300006122BEB7409122BE3123E7F7404122BDC
:109540008D80527422122E6112D19B7016741C12DF
:109550002E61E06402703E7405122BE37900124420
:10956000A980327422122E61129AFE7014741C1299
:109570002E61E06404701E7405122BE312449D807A
:10958000147422122E61129B37700A79007405122E
:109590002BE3124521029AE174615508700302968B
:1095A0009FE508A2E0506D12B9AE7405122BE312CC
:1095B0003FD5E9705C12444FE9F5097416122E612B
:1095C000E0700F7410122E61129B147003A3E069F7
:1095D0006042A90912B9AE7405122BE3123FDBE910
:1095E0006024E508A2E3500C85188285198374FF76
:1095F000F0A3800C740E122E61129B1FE8F0A3E9F9
:10960000F0751004800EE508C2E5F50875090080C4
:109610000353089FE508A2E5503FEE242F12B97CC2
:10962000C0E07402122E61D0E0129B5DC0E07403B2
:10963000122E61D0E0129B55C0E07404122E61D04E
:10964000E0129B3D12299D7406122BEB7409122B1C
:10965000E3123E7F7404122B8DE508A2E64003025C
:109660009974A818A919880A890B780A122B7AA963
:1096700009129AEF122BE31242FF7402122B8DE9AA
:10968000F50970030299747422122E6112B50464F4
:1096900001600302997474104510F51002997474F6
:1096A00007122E61E06401705D7422122E6112B502
:1096B000046405701EA818A9198808890978081279
:1096C0002B7A129AED122BE31242FF7402122B8DA9
:1096D000029AE17422122E61129B377029740E12C5
:1096E0002E6112CC9C123D71E9601BA818A9198843
:1096F0000A890B780A122B7A129AED122BE3124286
:10970000FF7402122B8D7416122E61E070257407FF
:10971000122E61E06401700C7422122E61E0F812C6
:109720009B37600CEEFCEFFD7405122BE312431720
:10973000029AE1124395E96003029AE1741D122E28
:1097400061E070030297ED7420122E6112B9B774B4
:109750001F122E61E0FA741E122E61E0F9123FA56D
:10976000E9607D741F122E61E0701E740E122E616E
:10977000129B1F12F4C1FAA3E0FB123D7D8B0BEA92
:10978000450B600302996E80517420122E6112CC39
:109790009C741F122E61E0F9123F9F851882851973
:1097A0008312E16D7808740D122E61E0600278106A
:1097B000740C122E61E06004740828F8740A122EEA
:1097C00061E0600108088E828F83A3A3E028FAA3DA
:1097D000E034008A82F583E014F075104002996E3F
:1097E0007508007808122B7E790B029927740E12E7
:1097F0002E6112CCA07409122E61E060030299421E
:10980000E508A2E350030299427407122E61E06456
:1098100001607A790085188285198312CC9C123FE9
:10982000F98A0A8B0BA80AA90BE849601C8882896F
:1098300083A3A3A3A3A3E06401605288828983A3C6
:10984000A3A3A3A3E064026044EE242D12B9B18562
:10985000188285198312CC9C1245DB8A828B83E5A2
:10986000824583600FA3A3E0F91245F9E96005C3BF
:10987000940840197410122E6112CC9C123D71E9AB
:10988000700302991D7409122E617404F07800E8C7
:10989000F5097809122B7E741E122E61AC82AD83FD
:1098A000740F122E6112CC9C740A122E61E0F91210
:1098B000400B7401122B8DE9600F7510208E828F82
:1098C00083A3A312B504543FF0741D122E61E0600F
:1098D00023740E122E6112B9B7741E122E61AA8261
:1098E000AB8312441985188285198312E16D744087
:1098F0004510F5107407122E61E0640160157900BF
:109900007410122E6112B9B7740E122E6112CC9C13
:10991000123FABE508A2E350377940803575080067
:109920007808122B7E7902740F122E6112B9B77467
:1099300011122E6112CC9C12451B7401122B8D0248
:109940009AE1E508A2E3400302988D784002988FDF
:1099500079007410122E6112B9B7740E122E6112B2
:10996000CC9C123F39E9600674204510F510124472
:109970004FE9F509851882851983E064FE7003A319
:10998000E0F470037509009019C9E06401600302F6
:109990009A27EE241312B97CF47003A3E0F4700349
:1099A000029A27740E122E61C3E094F9A3E094FF8B
:1099B000507512BADC7410122E61E0687003A3E0D7
:1099C0006960647410122E6112CC9C123D7D8A0A6B
:1099D0008B0BA80AA90BE849604D88828983A3A351
:1099E000A3A3E06401600D88828983A3A3A3A3E0FD
:1099F000640270337430122E61740112E6B7F8A35A
:109A0000E0F9743B122E6112CCAB7430122BE312CE
:109A10003D29E960127433122E61AA82AB83123D94
:109A20008FE960031237FBE508A2E74003029AE1E1
:109A3000E5097003029AE18E828F83A3A3A3A3E0BA
:109A4000FA7B0012341D8A0A8B0BEA450B70030265
:109A50009AE1EE2404F512E43FF5138E828F83A37E
:109A6000129B29122B76851282851383E0FC7D00E0
:109A70001233577403122B8D7407122E61E0C0E06D
:109A8000742B122E61D0E0F0742E122E61E4F0A33C
:109A9000F0742B122BDB880C890D780C122B7A7545
:109AA00008007808122B7E7810122B7AE509F50849
:109AB0007808122B7E12B9701229A585128285139F
:109AC00083E0F97408122E6112B9B7AA0AAB0B121F
:109AD000440D7408122B8DE96007AA0AAB0B1234EF
:109AE00023743D028736F582E412EEF522790012E6
:109AF000B97412B9BB74072212B51E64062212B5DE
:109B000020640722EE242BF582E43FF58312B9CBC3
:109B100012B9752212D54EEE241312BF61682212BB
:109B2000D54E85188285198322A3E0F50CA3E0F5B4
:109B30000D750E00780C2212B520640322F0129BE2
:109B40004222EE2425F582E43FF58322E4F0A3F0DF
:109B5000A3F0A3F022F0EE243112BF6122F0EE2434
:109B60003012BF612274F4122594EAFEEBFF8C08D8
:109B70008D099019C6E0600F12E2237003A3E0691B
:109B80007005123F278052790012CC8F123FF98A5C
:109B9000828B83E58245836035A3A3A3A3A3A3E0BF
:109BA0005418602AE508241C12CC881229A5E5085F
:109BB000241312CC881229A5EE2418129BDC129BC8
:109BC000E112CC9C1240117404122B8D800B790091
:109BD000129BE112CC9C123F51028FD112BF61F94E
:109BE000228E828F83A3A3A3A3A3A3A3A3A312B9AB
:109BF000CB12CC7B2274F012259474EA122C0B8ABF
:109C00000A8B0BEA2402F50EE4350BF50F0A0AFB6A
:109C1000123D838A088B09AE08AF09750801850AD1
:109C200082850B83A3E0F509750C01AC0EAD0F74B2
:109C30000B122E61AA82AB831235317413122E617E
:109C400074FEF0A304F07415122E617402F074080F
:109C5000122E61E4F0901CD7E0700EEE4F700AE512
:109C60000970067508C3029E31901A6EE0640860A0
:109C7000067508C2029E2D850A82850B83A3A3A3C5
:109C8000A3A3A3A3A3A3A3E0A2E1500EA2E35005C4
:109C9000750C04800C750C038007A2E35003750C4F
:109CA00002EE4F7003029D408E828F83A3A3A3A375
:109CB000E06404600D8E828F83A3A3A3A3E06403FA
:109CC000700C7404650C602C7403650C60268E8225
:109CD0008F83A3A3A3A3E06402600D8E828F83A36E
:109CE000A3A3A3E0640170317402650C60067401E3
:109CF000650C70188E828F8312CC9C1244F7E97029
:109D00003F12A9A6122E6112CCAB80348E828F83B3
:109D1000A3A3A3A3E06402600D8E828F83A3A3A3F9
:109D2000A3E06401700A8E828F8312CC9C123F6F75
:109D3000E50A2402FAE4350BFB123D8F7E007F001A
:109D40007413122E61E064FE7003A3E0F4704612F7
:109D50003D35E97040E509601B901CE012CC9C1277
:109D600044F7E9700F901CE012A9AA122E61E8F0E6
:109D7000A3E98020850A82850B83A3A3A3A3A3A3C1
:109D8000A3A3A3A3E05402F9123F637413122E613C
:109D9000EAF0A3EBF07413122E61E064FE7003A3EB
:109DA000E0F470067508C7029E2DE509F50D780DE3
:109DB000122B7E850A82850B83A3A3A3A3A3A3A34F
:109DC000A3A3A3E0F9E50A2402FCE4350BFD741417
:109DD000122E6112CC9C123EA37401122B8DE970DD
:109DE0004CA90CE50A2402FCE4350BFD7413122E79
:109DF0006112CC9C123D5F8A0E8B0FAE0EAF0FEE40
:109E00004F601F74026509700D8E828F83A3A3A318
:109E1000A3A3E0D2E3F07415122E61E4F0750800FC
:109E2000800B7413122E6174FEF0A304F0E5097028
:109E300009AA18AB19123C33800AFCA90CAA18AB6A
:109E400019124497E9FCEE4F6053E50960208E82B9
:109E50008F83A3A3A3A3A3E0D2E6F07402650970E5
:109E60000D8E828F83A3A3A3A3A3E0D2E5F0850A7E
:109E700082850B83A3A3A3A3A3A3A3A3A3A3E0A26D
:109E8000E6500D8E828F83A3A3A3A3A3E0D2E7F0B5
:109E90008E828F83A3A3A3A3A3A3E004F0E508709D
:109EA0003BEC60337D007A017B10123333EE4F6060
:109EB0000CE50A2402FAE4350BFB123D8F741312F1
:109EC0002E61E064FE7003A3E0F4600B7413122EA5
:109ED0006112CC9C123F6F741602D93CFC80C57491
:109EE000F712259474F7122C0BEAFEEBFF901A6E12
:109EF000E06403600DE064016008E064096003024F
:109F0000A02E8E828F83A3E06003029FEC7C007DF5
:109F1000007A027B0012333312A0338A828B8312C1
:109F2000BAE5901A5F12CCAB7953123C27901A6EA7
:109F3000E064096009901A6C12CC9C1245D5851812
:109F400082851983740112CFD27942123C27901A6C
:109F50006E7404F07401122BE3794A123C217401EF
:109F6000122BEB7A647B1A123531901870E0640B77
:109F700070057406F0800B7900901A6C12CC9C125C
:109F80003E9D9019DCE060046401701F901A62E04D
:109F900064FE7003A3E0F4602A79007401122BEBD5
:109FA000901A6212CC9C123D5F8018E0640270131C
:109FB000901A5F12B9B77A037B0012333312A8925A
:109FC000123333901A59E0A2E35004D2F08002C257
:109FD000F012CFC87952123C279019DCE06402706D
:109FE0004A901C99122E321242F9803FFC7D007A71
:109FF000037B101233339019DCE06402701B90185D
:10A0000070E0640B7003740AF09019CAE4F0FA7BF4
:10A0100040901AB9E0F91234EF8E828F8312A03D7E
:10A0200012CC9C123E9D901A6EE4F01243657409A6
:10A0300002B3FDEE2402FAE43FFB22E0F8A3E0F9CC
:10A04000901A6C22C082C0839019F512CF9B701FAA
:10A05000901A6EE014600924FC600A14600C800FF2
:10A06000901A0080349019FC802F9019FE802AE805
:10A070004960089019F612A674700C8A828B83A32B
:10A08000E0F9123E85801D9019F512D1A564027089
:10A090000512456F800E901AEC12CF9B600612C815
:10A0A000BD12277A02C58874F412259474FE122C0E
:10A0B0000B8A088B097A007B04901AB9E0F91234F4
:10A0C000EFAA18AB197950123C217A0F7B0012339A
:10A0D0007B8A0A8B0BAE0AAF0BEE4F60208508829D
:10A0E000850983A3E07016901A6CE0F47003A3E076
:10A0F000F4603B12A30D7003A3E069603185088210
:10A10000850983A374EA12A7F8123C277A627B1AA6
:10A11000794B123C277A6C7B1A7950123C277A6172
:10A120007B1A79E1123C27EE4F700302A1B78E82B1
:10A130008F837402F0901A6CE0F47003A3E0F46073
:10A140000A12A30D7003A3E069704F851882851968
:10A150008312A03BE8F0A3E912A7F8123C21901A61
:10A160005F12B02112CCAB7A627B1A794B123C2180
:10A170007A617B1A79E1123C21750A00780A122B68
:10A180007E780A122B7E901C4D12A03E12AD571203
:10A19000CC9C1244557402122B8D8508828509834C
:10A1A00012A1BCA3F0901A6E7403F0EEFAEFFB90CC
:10A1B0001AB9E0F91233877402028FCEA3E08E82BF
:10A1C0008F832274F412259474E8122C0BEAFCEBB2
:10A1D000FD8C828D83A3A3A3A37808122DD47808C5
:10A1E000122D94901A6F7808122D277F7F7E7F7929
:10A1F00000901A6F7808122DD4E97808122BC2E566
:10A2000008A2E050297800901ABA80148508828547
:10A210000983A3A3E069700108E508241412CC881F
:10A2200012AA4170E7E8C39F5004E8FFE9FE09E97C
:10A23000C3941B40BC8C828D83A3A3A3A3122E0EB8
:10A24000E8494A4B6079EC2404F508E43DF50985BA
:10A250000882F583122E0E901A6F122E4A7C187DFA
:10A26000007900AA18AB1912336385088285098327
:10A27000122E0E851882851983122E4A7404122E0E
:10A28000617401F0901A75E0C0E07405122E61D07F
:10A29000E0F07407122E61E412CFD2123C3F806AC4
:10A2A000901A6C12CC9C123ED38A0A8B0BA80AA976
:10A2B0000B901A6C12A31C687003A3E069602D90C8
:10A2C0001ABA12AA41602585088285098312A31350
:10A2D0007003A3E069700C850882850983A3A3E05D
:10A2E0006E60BDE508241412CC8880D6EE901A6109
:10A2F000F0124347E96013901A6EE4F0901A0212CC
:10A30000CF9B600612C8BB12277A028FCC851882B9
:10A3100085198312D54E901A6CE06822E8F0A3E903
:10A3200012A32422F0850882850983E02274F412A6
:10A33000259474E8122C0B8A828B83A3A3A3A3A376
:10A34000A3A3A3A312DA4C7C00901A6F7808122DF5
:10A35000D4EC7808122BC2E508A2E0502FECF8EA02
:10A360002812BAD4F8901CDFE0C398501F7508017A
:10A37000750900750A00750B00EC7808122ADE7862
:10A3800008122D94901A6F7808122D270CECC394A4
:10A390001B40B6901A6F122E0EE8494A4B604E7C55
:10A3A000187D007900AA18AB19123363901A6F1246
:10A3B0002E0E851882851983122E4A7404122E617E
:10A3C0007401F07407122E617401F0901A75E0C0E8
:10A3D000E07405122E61D0E0F07407122E61E412D1
:10A3E000CFD2123C3F901A6E7406F0801C901A6E09
:10A3F000E4F0FCFD7A047B10123333901A0212CF82
:10A400009B600612C8BB12277A028FCC74F5122506
:10A410009474D1122C0B8A088B098A828B8312BC0C
:10A4200070741C122BEB8A828B83A3A3A3A3A3A318
:10A43000A312A66C12CC93124377741C122E61E007
:10A44000702C850882850983A3A3A3A3A3A3A3A338
:10A45000E0C3940B40188E828F83A3A3A3A3A3A36E
:10A46000A3A3E06402700712CC76E0F4600302A6B6
:10A470005E901A6EE06402700302A543E064067009
:10A480000302A5439019F512CF9B600812A67470C1
:10A490000302A577901A6EE064086008E064046027
:10A4A0000302A65E741E122E6112A663A3A3A3A3C9
:10A4B00012BC709019F5E0F849600712D1AB640244
:10A4C0006077901A6CE06E7003A3E06F600302A6E1
:10A4D0005E74016A60167423122E61AC82AD837AB9
:10A4E000807B1A12352BE9600302A65E7A007B029C
:10A4F000901AB9E0F91234F5EA4B4C4D600302A60C
:10A500005E901A6F122E0E851882851983122E4ABC
:10A51000901A75E0C0E07404122E61D0E0F074056A
:10A52000122E617401F07406122E61740212CFD2E1
:10A53000123E0DE9600302A65BEEFAEFFB124569DD
:10A5400002A65E9019F512CF9B702C750800780852
:10A55000122B7E7808122B7EEE2410F582E43FF554
:10A560008312CF8FA3A3A3A3A312B9D412CC9C129E
:10A5700044557402122B8D8E828F8312BAE57407B4
:10A58000122E61E8F0A3E912A9B012BAE57409121B
:10A590002E6112B9E612BF6BC0E0740B122E61D0AF
:10A5A000E0F012CC76128744740F7808122DE37411
:10A5B0000C122E61E508F07420122E61E0C0E074E8
:10A5C0000D122E61D0E0F07422122E61E0C0E07412
:10A5D0000E122E61D0E0F0741D122E61E0C0E07406
:10A5E00010122E61D0E0F0741E122E61E0C0E074F3
:10A5F0000F122E61D0E0F0EE241012B97CC0E0748E
:10A6000011122E61D0E0F07421122E61E0C0E074CE
:10A6100012122E61D0E0F0742E122E61E0C0E074B0
:10A6200013122E61D0E0F07423122E61A982AA8346
:10A6300089088A09750A007808122B767C087D0043
:10A640007417122E61AA82AB831233577403122B34
:10A650008D7407122BE3123E978003123E13742F62
:10A6600002B66DE0FA8E828F83A3A322A3E0F98A5B
:10A67000828B832212D1AC64012274F71225947468
:10A68000C9122C0B124587901A6EE06408601F9067
:10A690005157E493901A50F0905157E493901A4E0A
:10A6A000F0901A77740112A7EFA30412A7EF7C238E
:10A6B0007D0079007414122BE3123363901A7FE04B
:10A6C0007009741E122E6174018006741E122E61B0
:10A6D000E412A800740FF0901CDE12CFD27946125B
:10A6E0003C277401122E61E4F0901CB2E0C0E074CB
:10A6F00002122E61D0E0F0901A5CE0C0E074031208
:10A700002E61D0E0F07404122E61E4F07405122E74
:10A7100061E4F07407122E61E4F0901A7FE0C394B4
:10A720000F500CE0C0E07406122E61D0E080077478
:10A7300006122E61740FF07C807D1A7408122E614F
:10A74000AA82AB831235317C037D0079FF7410122D
:10A750002E61AA82AB83123363901AB8E0C0E07412
:10A7600013122E61D0E012CBDC7401122BE31243E2
:10A77000717ABC7B1A7945123C27124485901A7372
:10A78000E0C0E0741C122E61D0E0F0901A74E0C0BA
:10A79000E0741D122E61D0E0F0901A61E0C0E07408
:10A7A0001A122E61D0E012879A7418122E6112CC00
:10A7B000AB7420122E61E4F0901A76E0C0E0741FB2
:10A7C000122E61D0E0F07434122E61E4F07429127C
:10A7D0002E61E412A7F8123C277A627B1A794B1299
:10A7E0003C277414122BE3123C45743702B3FDF07E
:10A7F000A3E4F0A3F0A3F022F07A5F7B1A7953224E
:10A8000012A80422F085188285198322C082C08391
:10A810008A828B83A3E0901A6E6004E4F0807074E7
:10A8200008F0901A7FE07028901A0212CF9B6008FF
:10A83000790012C8BD12277A901A6C12B9B77A053E
:10A840007B00123333901A6C12CC9C1245D58018C1
:10A850007900123E91901A5F12B9B77A067B001206
:10A86000333312A892123333901AF212CF9B601F27
:10A870009019D0E06401701790810612299D7A002A
:10A880007B40901AB9E0F91234E97404122B8D025E
:10A89000C588901A6212B9BB7A047B002274F41244
:10A8A000259474EA122C0B8A088B09EA2402FAE434
:10A8B0003509FB123D838A0A8B0BAE0AAF0BEE4FB4
:10A8C000700302A9A18E828F83A3A3A3A3E06401D6
:10A8D000602A8E828F83A3A3A3A3E06402601D8EEF
:10A8E000828F83A3A3A3A3E0640360108E828F836F
:10A8F000A3A3A3A3E06404600302A9A1E5082402C2
:10A90000FCE43509FD740B122E61AA82AB8312356B
:10A910003112A9A6122E6112CCAB7415122E6174DD
:10A9200001F07408122E61E412CFD2123C39E9FC16
:10A930007D007A077B001233338E828F83A3A3A31B
:10A94000A3A3E0C2E012A9B0740112E97F5001098B
:10A950007A027B00122337E88E828F83A3A3A3A3FE
:10A96000A3A3A3A3F09019D0E0640170349019CA96
:10A97000E06402702C8E828F83A3A3A3A3E0640102
:10A98000600D8E828F83A3A3A3A3E06402701212D2
:10A99000B970122E0E12C25F122E4AEE241B12CF75
:10A9A000827416028FCE8E828F8312D54E7413223C
:10A9B00012A9B42212C295A3A3A3A32274F2122552
:10A9C0009474F8122C0BEAFEEBFF8C0A8D0B890DA8
:10A9D0009080C8AC18AD197408122A9E750C00EE50
:10A9E000FCEFFDAA18AB1912352BE97003750C01A9
:10A9F000901ABA801AEEFCEFFDE508240BFAE43554
:10AA000009FB12352BE97023E508241412CC8812B7
:10AA1000AA416024E50CA2E040DB85088285098319
:10AA2000E0650A7004A3E0650B70DD850882850986
:10AA300083A3A3E0650D70D0AA08AB097408028B4C
:10AA400040128748E508450922C082C083901ABA9F
:10AA500002C58574F7122594901ABA12F105800C7C
:10AA600012D7B412BC73123423EEFAEFFBEA4B7028
:10AA7000EF901ABAE4F0A3F002B40074F412259433
:10AA8000EAFEEBFFEE241312B97C6403700CEE2493
:10AA90000BFAE43FFB123D83800EE06402707C12EF
:10AAA000CC7612CC9C123D7D8A088B09E5084509BD
:10AAB00060698E828F83A3E0700F85088285098389
:10AAC000A3A3A3A3A3A3E4805164F1600A8E828FA1
:10AAD00083A3E064E17027850882850983A3A3A38B
:10AAE000A3A3A3E06401701685088285098312CCB4
:10AAF0009C123F6FEE240BFAE43FFB123D8F85085A
:10AB000082850983A3A3A3A3A3A3E0600E85088283
:10AB1000850983A3A3A3A3A3A314F0028FD174F187
:10AB20001225948A088B09ECFEEDFF890A8A828B34
:10AB30008312DBEF8A828B8312A1BC12ABF08A8274
:10AB40008B83A3A3E0C454F0FA88828983E04A127D
:10AB5000AC0012A1BC12ABFAE0333354FCF88E8285
:10AB60008F83E04812ABFAA3E033333354F8F88E06
:10AB7000828F83E04812ABF08508828B83A3A3A366
:10AB8000A3A3A3E0A2E0E4331313FA88828983E04D
:10AB90004AF0E5082407F50CE43509F50D750E00BB
:10ABA000780C122B767C087D00EEFAEFFB123357FF
:10ABB0007403122B8DEE2408FE50010FE508240FBC
:10ABC000F50CE43509F50D780C122B767C037D002D
:10ABD000EEFAEFFB1233577403122B8DE50AC39480
:10ABE0000F400A12CC8412A1BDA3A3A3F002E95125
:10ABF000F0EEF8EFF9A30EAF832212AC00A3A3226C
:10AC0000F08508828B83A3A32274F1122594EAFEB7
:10AC1000EBFF890A8C088D098E828F83E08C828DF0
:10AC20008312BF9CAE82AF83E012C34B12C535C402
:10AC300012C34B12ACC8E012C35212C533A2E2E4F5
:10AC4000338C828D8312C532131313541F12C34BDE
:10AC500012C531A2E7E4338C828D83A3A3A3A31290
:10AC6000ACC88E0C8F0D750E00780C122B767C08FC
:10AC70007D00E5082407FAE43509FB123357740315
:10AC8000122B8DEE2408FE50010F8E0C8F0D780CC8
:10AC9000122B767C037D00E508240FFAE43509FBCE
:10ACA0001233577403122B8DE50AC3940F40118E93
:10ACB000828F83A3A3A3E0C0E012CC84D0E0800401
:10ACC00012CC84E4F002E951A3A312BFA00EAF831B
:10ACD0002274F51225948A088B098A828B83A3AE8D
:10ACE00082AF83E0F9123EBB8E828F83E064EB601B
:10ACF00024850882850983A3E064E16018850882C1
:10AD0000850983A3E064F1600C850882850983A32B
:10AD1000E0641A7009850882850983A3E4F0901C19
:10AD200099122E321242F9750A01780A122B7E8589
:10AD30000882850983A3E0F5087808122B7E790044
:10AD4000901A6C12AD5712CC9C1244557402122BFF
:10AD50008D12438F02B67012B9BB901A6222C08264
:10AD6000C083E9901ACC7003E480027401801EE075
:10AD7000F902C588C082C0837CE77D428A828B83CA
:10AD800012CC9C123C5102C588EAF0A3EBF002C53C
:10AD90008874F6122594901ACCE0701B7C0079011F
:10ADA0007A007B001243BFEA4B600C8A828B8312CD
:10ADB000CF9B60031242ED02C91AC082C08379049E
:10ADC0001243B9E9F8905155E493C398401079FFC4
:10ADD0001243B9E9F8905154E493C39850047901AF
:10ADE0008002790002C58874F01225948A088B09C4
:10ADF000890B750C008A828B83A3A3A3A3A3A3A3AF
:10AE0000A3E0F91243C58A0E8B0FAE0EAF0F750A81
:10AE100001EE4F600302AED285088285098312B02D
:10AE200010A3A3A3A3A3A312C05912CC9C1243AD99
:10AE30008A0C8B0DAE0CAF0DEE4F700302AFFB8E84
:10AE4000828F83A3A3A3A3E4F0A3F0E508240CFA64
:10AE5000E43509FB8A828B83E0C0E012E975D0E01B
:10AE6000F0E508240D12B00812DBBD12CCAB124481
:10AE7000E5EE240F12E167E508241112B0081289EB
:10AE80002212CCABE508241312B003C0E012B97053
:10AE9000D0E0F0750C01EE240612BF51E0547FF0B3
:10AEA000A3E054FC12E6ADE05404600302AF499005
:10AEB0001CABE0F50875090074077808122D148E94
:10AEC000828F83A3A3A3A3A3A3E04508F0A3E04537
:10AED00009F08E828F83A3A3A3A3128742740778FD
:10AEE00008122DE3E5085407FCE50B606C8E828F99
:10AEF00083A3A3A3A3A3A3A3A3A3740212C536127F
:10AF0000B2D7600B901A5A12B021A3A312CCABECAB
:10AF1000700302AFC4EE240612F453547FF508A365
:10AF2000E054FCF509EC24FFF50EE434FFF50F7452
:10AF300007780E122D14E508450EF8E509450FF9BE
:10AF40008A828B8312CCAB807B8E828F83A3A3A358
:10AF5000A3A3A3E0448002AED1EC7005750A008083
:10AF6000638E828F83A3A3A3A3A3A3E05420600CCA
:10AF7000123375EA547F7900245F80198E828F83A3
:10AF8000A3A3A3A3A3A3E05410601A123375EA5439
:10AF90000F7900240A5001098E828F83A3A3A3A3F3
:10AFA000F0A3E9800D8E828F83A3A3A3A37401F085
:10AFB000A3E412A9B07404F07A207B00901AB9E0DF
:10AFC000F91233BDE50CA2E0503412B9D0A3A3A30B
:10AFD000A3A3A3A3A3A3E0F9EEFAEFFB1243B3E903
:10AFE000601C12ED5B3F12CF99600912B52E12CC96
:10AFF0009C123423EEFAEFFB123423750A00A90ADF
:10B0000002D93F12BF79E02212BF7912D54EEE224B
:10B01000A3A3A3A3A3A312B9BB850882850983A315
:10B020002212D54E8E828F83A3A32274F41225940C
:10B0300074F7122C0B7E001243C5EA4B700302B06A
:10B04000E78A828B83A3A3A3A3A3A3A3A3A3E06400
:10B0500006600302B0E78A828B83A3A3A3A3A3A302
:10B06000A3E0FF8A828B8312B0EEE0C0E074081286
:10B070002E61D0E012B51512CCA11243E3EF5408B3
:10B08000606385188285198312B9B77A007B001234
:10B0900043A78B0BEA450B704C12F5AD123C697C53
:10B0A000007D007A007B0080288E828F8312B50499
:10B0B000F47003A3E0F4602D901A6C12B9D812CC8E
:10B0C0009C123C63E9641A601C7C007D00EEFAEF80
:10B0D000FB1243A78A0A8B0BAE0AAF0BEE4F70C967
:10B0E0007900123C6F7E01EEF97409028FCE12BC1A
:10B0F0007C12B0F5222408F582E438F58322C08260
:10B10000C083EA4B7005901AD180068A828B83A394
:10B11000A312B30B60258A828B83A3A3A3A3A3A34B
:10B12000A3E0540860E5EC4D60158A828B8312B56C
:10B13000046C7003A3E06D70D280047A007B00027F
:10B14000C58874F2122594EAFEEBFF890A8C088DFB
:10B15000097A147B0012341DEA4B603F8A828B838C
:10B16000A3A3A3A3A3A3A3A3A3E412B50AA3E50ADD
:10B1700012B1A7A3A312DD2A8A828B83A3A3A3A360
:10B18000E4F0A312B52812B1B912E105EA12ED5CA0
:10B190003BF583E4F012B19EF0A3F0028B43A3F0E1
:10B1A0008A828B83A3A32212B1AB2212B1AF22F009
:10B1B0008A828B83A3A3A3A322A3F012F4743BF58A
:10B1C00083E4F02274F4122594EAFEEBFF89088CE4
:10B1D0000A8D0BEE4F700302B260740165087012A5
:10B1E00079011243B9E9F8905156E493C39850227B
:10B1F000801674046508701479041243B9E9F89054
:10B200005155E493C398500A791180567402650829
:10B21000704E8E828F83A3A3A3A3A3A3A3A3A3E5AE
:10B220000812B9E012DBCAE4F0A3F0901AD112CFF1
:10B230009B60178003E0F8A312CDA2A3A312B30B67
:10B2400088828983A3A370ED8003901AD112E1094B
:10B250007A207B00901AB9E0F91233BD79008002A0
:10B2600079C1028FD1C082C083E9F87900901AD1E8
:10B27000801D8A828B83A3A3A3A3A3A3A3A3A3E07C
:10B2800068600574FF687001098A828B83A3A3122A
:10B29000B30B70DE02C58874F7122594EA4B700573
:10B2A000901AD180068A828B83A3A312B30B6020ED
:10B2B0008A828B83A3A3A3A3A3A3A3A3A3E0697000
:10B2C000E4EC60108A828B83E012B2D770D78004DE
:10B2D0007A007B0002B40012F4A9E0540422C08278
:10B2E000C083901AD180068A828B83A3A312B30BEA
:10B2F00060128A828B83A3A3A3A3A3A3A3A3E06961
:10B3000070E580047A007B0002C58812D1D0EA4B38
:10B310002274F7122594EAFCEBFD901AD180068A7C
:10B32000828B83A3A312B30B60248A828B8312B512
:10B33000046C7003A3E06D70E68A828B83A3E0C87F
:10B3400012BC6912D92BA2E0E43370D380047A00D6
:10B350007B0002B40074F21225948A0A8B0B8C0CC9
:10B360008D0D750800750900EA450B6030901AD103
:10B3700080068E828F83A3A312BC73EE4F601EAC37
:10B380000CAD0DEEFAEFFB850A82850B8312277A4E
:10B39000E9640170DDEEF8EFF988088909AA08ABC5
:10B3A00009028B437900022B2274F7122594901A1C
:10B3B000D112BAE57C007D00800DE8FCE9FD8882B1
:10B3C0008983A3A312BAE5E8496030EA687002EB0A
:10B3D0006970E7901AD112CC9CE86A7002E96B8818
:10B3E000828983A3A3700812BAE5901AD18009124A
:10B3F000BAE58C828D83A3A312CCAB8003122B8D74
:10B400007F0102281974F7122594EAFEEBFFEE4F34
:10B41000602F1243DD12B44312CC9C1234238E826F
:10B420008F8312CC9C12342312ED5B3F12CF9960B4
:10B430000912B52E12CC9C123423EEFAEFFB123413
:10B440002380BD12CFA1F5832274F61225948A823F
:10B450008B8312B504F508A3E0F509901AD112BA4E
:10B46000E57D007C00802F88828983A3A3A3A3A30A
:10B47000A3A3A3A3E0640570140C12DBE6F5838E8E
:10B4800082E065087004A3E0650970010D88828977
:10B4900083A3A312BAE5E84970CD905152E493F822
:10B4A000EDC398500890515112EEE3400F8A828B01
:10B4B00083A3A3A3A37401F0A3E48010901A5AE01D
:10B4C000F812A66CA3A3A3A3E8F0A3E912B528740D
:10B4D0000512B50AE0440812B515F47003A3E0F4B0
:10B4E0006011901A6C12D90E12CC9C123C63E96464
:10B4F0001A70057901123C6F02C91AEE241DF582FB
:10B50000E43FF583E0F812B5202212B50E2212B105
:10B51000AFA3A3A322F08A828B8312B51E22E0F888
:10B52000A3E0F5838882E02212B50EA3A322EE12D7
:10B53000CD8722C082C083EAFCEBFDEC4D6017ECA6
:10B5400024FBF582ED34FF12CF99700712B58DE020
:10B55000F4600712338179058030901AB9E0C0E0B9
:10B5600012B58DD0E0F0905148E493F97AD37B1A6C
:10B570001233B7E9640170107A007B20901AB9E0A9
:10B58000F91233BD79008002790402C588EC24FFEA
:10B59000F582ED34FFF5832274F4122594A2AFE412
:10B5A00033F508C2AF901AD312BC73EE4F603AEE77
:10B5B00024FBF582EF34FF12CF997A007B20901A9A
:10B5C000B96007E0F91233BD8005E0F91233C3E436
:10B5D000F50AF50B780A122B7AEEFCEFFD7AD37B95
:10B5E0001A1233B17402122B8DE508A2E092AFEE6D
:10B5F000FAEFFB028FD174F51225948A088B097536
:10B600000A00901AD112DBEA805A8E828F8312B51B
:10B610000465087004A3E06509703D8E828F83A3E2
:10B62000A3A3A3E4F0A312C2A6540460118E828FD8
:10B6300083A3A3A3A3A3A3A3A3E0F9123FE18E8254
:10B640008F83A3A3A3A3A3A3A3A3A37406F07AF059
:10B6500012892F1242F3050A8E828F83A3A312BA96
:10B66000E5E8FEE9FFEE4F70A1A90A8003122B8DD9
:10B670007F0302281974F012259474D4122C0BEA5B
:10B68000FEEBFF750B00750A007508FE7509FF12C9
:10B690004395E9600302B963EE241512B97C604456
:10B6A000901CC8E0C43354E0F8E0333354FC48C085
:10B6B000E012D73DD0E012B9E012CC9C79FF1240E5
:10B6C000E38B0DEA450D600F750B017508FF12CF76
:10B6D0008612CE5CD2E0F09019DCE0600464017068
:10B6E00003750A408E828F8312CC9A1244D9E96086
:10B6F0000312B988EE241312B97C700D90513FE407
:10B7000093C0E012B970D0E0F08E828F83E0A2E7A0
:10B71000500454038019EE241412B97C7012901A4C
:10B720004BE0C0E012F449D0E0F0901A4BE004F096
:10B7300012F4657016901CB4E0600D901A56E0701B
:10B740000A8E828F83E0700312CD779019DCE0605F
:10B75000046401704B901A59E0A2E15043E50BA23A
:10B76000E040218E828F8312CC9A1244D9E9603056
:10B770008E828F83E0600DEE240B12B4FEF912442A
:10B78000B5E9601C12B994700302B915EE241312C6
:10B79000B97C6401600302B91512B52EE054FBF0C8
:10B7A0008E828F83E06401700DEE240B12B4FE6470
:10B7B00002700312B9A112B994600302B87BE50BC1
:10B7C000A2E0500302B87B9019DCE06007640160DE
:10B7D0000302B87B901A59E0A2E1400302B87BE56E
:10B7E0000AF50B780B122B7EEE2406FCE43FFD8E4F
:10B7F000828F8312CC9AEE2412129BDC12400B74BF
:10B8000001122B8DE9600612B98812B99A8E828FC7
:10B8100083A3A3A3A3A3A3E0603CEE2402F50CE45E
:10B820003FF50D850C8212B9C52407FAE43FFB12DF
:10B8300044198A088B09850C82850D83E0650870A0
:10B8400004A3E06509700C8E828F83A3A3A3A3A336
:10B85000A3E4F012B9A18E828F83E06401600BA98A
:10B860000A12B9D412CC9A123FABA90A12B9D0125B
:10B87000CC9A123F39E9600312B99AAC18AD19EEAF
:10B88000FAEFFB1244138A0A8B0B74FE65087004EE
:10B8900074FF6509700312873EEA450B700302B915
:10B8A000678E828F83E0C0E07401122E61D0E0F0D9
:10B8B0007404122E6112E109EE241E12BADF740222
:10B8C000122E6112CCAB7401122BDB880C890D781F
:10B8D0000C122B7AEE242012B980122B7E12B52E78
:10B8E0001229A5EE240E12B980122B7E901A5F1237
:10B8F00029A57408122E61E0F9AC08AD0912440DB7
:10B900007408122B8DE9FE74106E705DAA0AAB0BE1
:10B910001234238054EE241312B97CC0E074171241
:10B920002E61D0E012F4BA740F122E6112B9E6241F
:10B930000412F45812BAE57411122E61E8F0A3E96A
:10B9400012BFC1C0E07418122E61D0E012E96B1270
:10B95000A66D12B9B77406122BE3123FDBE9600340
:10B9600002B7A0791180047E10EEF9742C02D93C44
:10B9700012B97422EE12CDBF22EE241712BF61223B
:10B9800012BF61F50C780C22EE2412F582E43FF52B
:10B9900083E4F02212B9A854402212B9A84420F03E
:10B9A0002212B9A84440F022EE12CD8BE022EE2400
:10B9B00013F582E43FF58312B9BB2212B9BF22E02E
:10B9C000FCA3E0FD22F58312B9CB2212B9BFEE220F
:10B9D0008E828F83A3A3A3A312B9BB8E828F8322EF
:10B9E00012DBD622A3A3E8F0A3E9F0EE22C082C0C6
:10B9F0008374D7122C0B9080007403122BEB7426E7
:10BA0000122A9E8A828B83A3A3A3A312BAE5740E83
:10BA1000122E61E8F0A3E912D547740C122E6112C0
:10BA2000BAE9240D12BAD4C0E0741A122E61D0E023
:10BA3000F012D7BE12BAE37420122E6112BAE924B2
:10BA40001512BAD4C0E07408122E61D0E0F0EA24D6
:10BA50001CF582E43B12BAE37412122E6112BAE9A9
:10BA6000241112BAD4C0E07409122E61D0E0F0EAB9
:10BA7000241212BAD4C0E07407122E61D0E0F0EAAA
:10BA8000241EF582E43B12BAE37424122E6112BA2A
:10BA9000E9242012BAD4C0E07426122E61D0E0123C
:10BAA000A80074FFF07401122E6174FFF07402128A
:10BAB0002E6174FFF090810A12299D7404122BEB01
:10BAC0007407122BE3123E7F7404122B8D790074DD
:10BAD0002902D58BF582E43BF583E022EE2413F5B1
:10BAE00082E43FF58312D54E22E8F0A3E9F0EA2282
:10BAF00074EE12259474EC122C0B8A0E8B0F8C08AA
:10BB00008D09890C750A107A217B0012341D12D51B
:10BB100091E849700302BC62750B007C217D0079BD
:10BB200000851882851983E0FA1233637429122E76
:10BB30006112BC739019DCE060046401703EAA08D5
:10BB4000AB09123D7D8A108B11A810A911E849603C
:10BB50002388828983A3A3A3A3E06401600D888264
:10BB60008983A3A3A3A3E064037009EE5440700487
:10BB700074044FFFEF54046003750B01901A6C12AC
:10BB8000CC9C85188285198312BC782409F582E43F
:10BB90003812E16B7426122E6112BAE57411122E5E
:10BBA00061E8F0A3E912BC8112F46B12BC8112B0FF
:10BBB000F5740212F4C5F8A312C8BD12DE9412BCCB
:10BBC0008112F47BE50CF07428122E61E0F50885F3
:10BBD000188285198312F484E50812BC8112BC69AD
:10BBE000F583E50EF0A3E50FF07406122E6112E165
:10BBF000097408122E61E508F0742C122E6112E30C
:10BC000001C082C083740C122E61AC82AD83D083DC
:10BC1000D0827405122A9E742B122E61E0C0E0744B
:10BC200013122E61D0E0F0A90BAA18AB1912439B96
:10BC3000E9640170219019DCE0600464017012E590
:10BC40000BA2E0500CA9081243C5EA4B6003124353
:10BC5000E9750A00800C85188285198312CC9C1224
:10BC60003423A90A741402C2AC241FF582E43822DA
:10BC7000A3A3A312DBEAFF2212BC7C2212D5ABC81D
:10BC80002212D5A0C82274EE122594EAFEEBFF8C96
:10BC9000088D098E828F83A37408F0EE241612B9E2
:10BCA0007C60088E828F83A37410F012B9796009CA
:10BCB0008E828F83A3E02408F0EE241512B97C60F5
:10BCC000088E828F83A3E004F08E828F83A3A3A3C8
:10BCD000A3A3A3E060198E828F83A3A3A3A3A3A32E
:10BCE000A3E0C3332402F88E828F83A3E028F012EE
:10BCF000BF5A6005750B0E8003750B009019DCE0D0
:10BD00006402701E9019D0E0640170168E828F83D9
:10BD1000E06401600D9019CAE0600712BF4774012A
:10BD2000800412BF47E412BF9CE012BF6928250BB4
:10BD30008C828D83F012BF5A6013901A57E0F9126B
:10BD400042BDE9F8850882850983E029F0850882EB
:10BD5000850983E0C39475400975080075090002E0
:10BD6000BF40E0FA7B0012341D8A088B09EA4509BE
:10BD7000700302BF408E828F83E0FA901A5C12BF7C
:10BD8000957402780C122D14EA450CFAAB0DEE24D2
:10BD90001212B97C5403F50C750D007406780C1260
:10BDA0002D14EA450CFCEBFDEE241512B97C600461
:10BDB000780180027800EE2416FAE43FFBE8F9ED02
:10BDC00049FD12BF5AF50C7409780C122D14ED457B
:10BDD0000DFD8A828B8312BF95740B780C122D1483
:10BDE000ED450DFDEE241712BF8F740C780C122D4B
:10BDF00014ED450DFD8E828F83A3A3A3A3A3A312ED
:10BE0000BF95740A780C122D14ED450DFDEE242318
:10BE100012BF8F740D780C122D14ECF8ED450DF94E
:10BE2000E8850882850983F0E9A3F0EE240212BFB9
:10BE30005112C06312BFB7F0EE240412BF5112BFFB
:10BE40008112BFB7A3A312CDB512BF81A3A3A3A331
:10BE500012BFC1850882850983A3A3A3A3A3A3A3BB
:10BE6000F0750A088A828B83E06015EE241812B9F7
:10BE7000B1E5082408FAE43509FB123531750A10DA
:10BE800012B9796019EE241A12B9B1A80AE5082886
:10BE9000FAE43509FB1235317408250AF50A8E8259
:10BEA0008F83A3A3A3A3A3A3E06057EE2407F510F9
:10BEB000E43FF511851082F583E0C0E012BF70D039
:10BEC000E012BFA7E0C0E00812BF72D0E012BFA727
:10BED000129B29122B76851082851183E025E0FCC8
:10BEE000E433FDA80AE50828FAE43509FB123357C4
:10BEF0007403122B8D851082851183E0C333250ACC
:10BF0000F50AEE241512B97C6008C0E012BF70D0AB
:10BF1000E0F012CC76129B2A122B7612BF6AFC7DBF
:10BF200000A80B8E828F83A3E0FAE5082AFAE43595
:10BF300009FBEA28FAE43BFB1233577403122B8DFA
:10BF4000AA08AB0902C2AFEE2423F582E43FF583D1
:10BF500022F8E43FF9888289832212BF5E22EE2410
:10BF600011F582E43FF583E022F8EE12DBC1E02216
:10BF7000A80AE5082812BF7922F582E43509F5837D
:10BF80002212BF8522E0850882850983A3A322F5BA
:10BF900082E43FF583E0F50C750D002212BFA0226C
:10BFA000F08E828F83A322F0050A8E828F83A3A353
:10BFB000A3A3A3A3A3A322A3A312E6BD12BF85A399
:10BFC00022F0EE241412BF612274F412259474FD41
:10BFD000122C0B8A088B09ECFEEDFF7401122BDB8F
:10BFE000880A890B780A122B7A7402122BEBEEFA6C
:10BFF000EFFB123F877402122B8DE9705385188274
:10C0000085198312C063F07401122E61E0F812C02A
:10C0100059A3A312F4C1602914850882850983A35A
:10C0200012F4C512DA457401122E61E028F8A3E07B
:10C0300039F9E824FEF582E934FFF58312F1058031
:10C040000C850882850983A3E4F0EEFAEFFB8004F7
:10C050007AFE7BFF7403028FCEA3E0F98508828508
:10C06000098322E08508828509832274EE122594D3
:10C070008A0A8B0B8910ECFEEDFF750F017C267D83
:10C08000007900EEFAEFFB123363E510C394085019
:10C090000302C1F88E828F83E510F0EEFCEFFD8580
:10C0A0000A82850B8312C503124425E96003750FCC
:10C0B0000012C4E58E828F8312C53DEE12C4D93FB3
:10C0C00012C527C0E0128921D0E012C51FC0E0EEE2
:10C0D0002412F582E43FF583D0E012BF9C7408126D
:10C0E000C28DA3A3E06018E50A2408F8E4350BF933
:10C0F00012B97012CCAB8E828F83A3E02408F08E2D
:10C10000828F83A3A3A3A3A3A3A3A3E060178E821C
:10C110008F83A385820885830912C4F812D73D1244
:10C12000A31C2408F0EE241912B98BEE241B12B9BB
:10C130008BA312C28DE0600F12C2748E828F83A314
:10C14000A3A3A3A312C2A0EE241812B97C70030209
:10C15000C1E812C274FAEE2419F582E43FF583EACD
:10C1600012C2A0F8E50A28F582E412F5A7F812DC5D
:10C17000FEE812C2A0E8C39AEE5068241912B97CF6
:10C18000F8905149E493C398500575110C8008EE5E
:10C19000241912B97CF5118E828F83A3E0F8E50A89
:10C1A00028F50CE4350BF50D750E00780C122B7686
:10C1B000AC11EC2CFCE433FD7A1F7B0E1233577468
:10C1C00003122B8DEE241BF582E43FF583741FF0E0
:10C1D000A3740EF0E511C333F8850882850983E066
:10C1E00028800412CD6EE4F08E828F83A3E0F88E57
:10C1F000828F83E0C398500479008061A3E0FAE560
:10C200000A28F8E4350B12C269E8F0A3E912C53632
:10C21000C39AC0E012C25FD0E012C2A6603DEE2415
:10C2200017F8E43FF9880889098882F583E024F249
:10C23000F0EE241D12BF51E0240EFAA3E03400FBFF
:10C240008882898312E16D901A57E0F91242BDE9A4
:10C25000F8850882850983E0C398F0A90F8050EE25
:10C260002417F582E43FF58322F9EE241DF582E4DC
:10C270003FF583228E828F83A3858208858309E020
:10C28000F8E50A28F582E4350BF583E02212C29125
:10C290002212C29522F08E828F83A3A3A3A3A3228E
:10C2A00012A32404F02212C291A3E022122B8D7F4C
:10C2B0000A02281974F41225948A088B09EA12C319
:10C2C00052A3A3F0EA1313543F12C34BA3A3A3F04A
:10C2D000EAC4131312C35212C3657409780A122DEB
:10C2E000E312C359A3A3A3A3A3A3F0EB12C35B124E
:10C2F000C364740A780A122DE3E50A5401C0E0EC25
:10C300002418F582E43DF583D0E012C369740B78FC
:10C310000A122DE312C35912C362740C780A122D4B
:10C32000E312C359A312C362740D780A122DE3E518
:10C330000A5401C0E0EC2424F582E43DF583D0E00A
:10C34000F0740E7808122DE302891C540F8C828D34
:10C35000832254038C828D8322E50A54018C828DC2
:10C360008322A3A3A3A3A3A3A3F08A0A8B0B22C0B7
:10C3700082C08379008A828B83A3A3A3A3A3A3E0B3
:10C38000901A56600EE070238A828B83A3A3E0701C
:10C390001A8016E060158A828B8312CC93901A5F04
:10C3A000E06A7003A3E06B6002790102C58874F251
:10C3B0001225948A0A8B0B890C8C088D098A828B32
:10C3C0008312C50312442512C4E5850882850983BA
:10C3D00012C53DE50812C4D9350912C527C0E0E5EC
:10C3E00008241112CC88D0E012C51FC0E012CC8402
:10C3F000D0E012CFAF740812C511E06017E50A242F
:10C4000008F8E4350BF9E508241312C4DD12CFAFA8
:10C41000E02408F0850882850983A3A3A3A3A3A32E
:10C42000A3A3E06017850882850983A312C4F4E5FD
:10C4300008241512C4DD12C5362408F0850882854B
:10C440000983A3A3A3A3A3E06019850882850983B8
:10C45000A3AE82AF8312C27F85088285098312C58D
:10C460003104F0AA08AB0912442BE9F50D7064857C
:10C470000882850983A3A3A3A3A3A312C063A37007
:10C480001AE0FAE50A2AF8E4350BF9E508241D124A
:10C49000CC8812CCABE50CC39A802C12C4F4E824EF
:10C4A0000EF8500109E508241D12CC8812CCAB907F
:10C4B0001A57E0F91242BDE9F88E828F83E0F9E560
:10C4C0000CC39924F2C398C0E0E508241712CC8865
:10C4D000D0E0F0A90D028B43EA12F4752212BF7965
:10C4E000E8F0A3E922850A82850B83A3A312C55332
:10C4F000E0F9EA22AE82AF83E0F8E50A28F8E435F5
:10C500000BF922E0FAA3E0F8E4C8F9EA28E439FBE1
:10C510002212C5152212CFB7A3A3A3A3A3A322124D
:10C52000C566A3A3A3E022F583E812C55FA3A3E039
:10C5300022A3A3A3A3A3F08E828F83E022A3A3A3AD
:10C54000A3A3A3A3A3A312C55F12C553A3A3E0F99A
:10C55000EAF822E0FA850A82850B83A3A3A322F0DE
:10C56000A3E912C56622F0850A82850B83A3A3A3E3
:10C57000A322C082C0837AE17B1A79E2123C217A3D
:10C58000E17B1A800312CC9CD083D082022B22C084
:10C5900082C083901A5F80EDC082C083901A62804F
:10C5A000E4C082C083794A123C2180DC74F61225F3
:10C5B00094901AE9E0FE04F0EEF91243C58B09EA03
:10C5C000450970EDEE60EAF902C91A74EE1225947D
:10C5D000EAFEEBFF8C0E8D0F890C750A00750B00BF
:10C5E0001245DB8A088B097412122E61E0F50D7476
:10C5F00013122E61E0F510EA45097017E51060038B
:10C6000002C6EDA90CAC0EAD0FEEFAEFFB1245FF22
:10C6100002C7ECE510700302C6B89019DCE06004B4
:10C620006401700E901AEE12CF9B600612C8BD1204
:10C63000277AE50D700E850882850983E4F0750B75
:10C640000102C7109019DCE060076401600302C7B3
:10C6500010901A59E0A2E1400302C710901AF0129C
:10C66000CF9B600CA90DAA08AB0912C8BD12277A8E
:10C67000850882850983E0FA12E960500109C3EA5E
:10C6800098E499A2D265D033500985088285098340
:10C69000E004F0850882850983E0F8905142E49334
:10C6A00068706D750A01EEFAEFFB1240178508827B
:10C6B000850983A3E4F08058E50D701CEA2402127A
:10C6C000B003A80C28F8E4340013E813F070098ACA
:10C6D000828B83A3A37401F08A828B83A3A3E0F8E7
:10C6E000901C4DE0C3985052750B01804D7401654C
:10C6F00010701DE50D60199019DCE0600464017094
:10C700000F901A59E0A2E15007EEFAEFFB12401722
:10C710009019DCE06402702274016510701CE50D54
:10C72000901B006013E004F0901CACE0F8901B003C
:10C73000E0C3984005750A01E4F0E50BA2E092F031
:10C74000E50AA2E072F0400302C7EC9019DCE06059
:10C750000464017041901A59E0A2E15039EEFAEFF9
:10C76000FB123D7D8A088B09A808A909E8496026C3
:10C77000E50BA2E0500D88828983A3A3A3A3A3E0C5
:10C78000C2E0F0E50AA2E0506388828983A3A3A3F4
:10C79000A3A3E0D2E0F0E50AA2E050509019DCE05B
:10C7A00060046401701D901A59E0A2E15015EEFA80
:10C7B000EFFB123D6BE9600BEEFAEFFB7900123EE6
:10C7C000B58029901A62E06E7003A3E06F701DEED1
:10C7D000FAEFFB7901123EB59019DCE06402700CAF
:10C7E0007A017B00901AB9E0F91234EF02C2AF74FB
:10C7F000F41225948A088B098C0A8D0B90819A7803
:10C8000008122C62700E7A017B00901AB9E0F912BE
:10C8100033BD8035901C997808122DF2EA45094500
:10C820000A450B60187808122B727A017B00901A67
:10C83000B9E0F91234E37404122B8D800C7A017B79
:10C8400000901AB9E0F91234EF028FD1C082C08390
:10C85000901C9D02AD89C082C083901C9F02AD894F
:10C8600074F612259475084B75091A7808122B7AFC
:10C870007C6E7D007A217B001234957402122B8D20
:10C88000E9F508123D47E942089019DCE0600464CC
:10C89000017006123DC5E942089004DA12CF9B6090
:10C8A0000912C8BD12277AE94208124107E9FE12AF
:10C8B0003B91E9F8E5084E48F9805F79C4E0F583DB
:10C8C00088822274F612259412332D75084B75094F
:10C8D0001A7808122B7A75086E7509007808122BE1
:10C8E0007A7C007D007A217B001234A17404122B23
:10C8F0008D123D4D9019DCE0600464017003123D1F
:10C90000CB9004DC12CF9B600612C8BD12277A12AE
:10C91000410D123BA38003122B8D7F020228197454
:10C92000F612259474FF122C0B7E0075084B7509C6
:10C930001A7808122B7A7C6E7D007A217B001234E3
:10C94000957402122B8DE9600302CA047808122B39
:10C950007A75086E8E097808122B7A7C007D007A31
:10C96000217B001234A77404122B8DE9600302CAE4
:10C9700004901A5FE064FE7003A3E0F4700302CA3F
:10C98000047E01901A6EE064086005E06404706F34
:10C99000851882851983EE12CFD27942123C277A0C
:10C9A000767B1A7943123C277A737B1A7947123CBB
:10C9B000277A647B1A794A123C277A627B1A794B70
:10C9C000123C277A6C7B1A7950123C277A5F7B1ACB
:10C9D0007953123C277A747B1A7954123C277A6176
:10C9E0007B1A79E1123C27901A59E0A2E35004D255
:10C9F000F08002C2F012CFC87952123C2780051293
:10CA0000332D7E00123D3B9019DCE0600464017020
:10CA100003123DDD9004DE12CF9B600612C8BD12EA
:10CA2000277A124119EEF9740102C91774F612251A
:10CA300094E9FEA2E0502675084B75091A78081291
:10CA40002B7A75086E7509007808122B7A7C007DA8
:10CA5000007A217B001234A17404122B8DEEA2E324
:10CA60005003123D419019DCE0600464017008EE4F
:10CA7000A2E15003123DE3EEA2E2500E9004E01258
:10CA8000CF9B600612C8BD12277A02C91A74F6122B
:10CA9000259474EC122C0B7401122BEB901CDEE02D
:10CAA000F97ABC7B1A1243777405122E61E4F07494
:10CAB00007122E61E4F07A04F9123D59905157E4BF
:10CAC00093F8C3EA98EB94005058123D35E9705240
:10CAD00090513B12CB7E60197A047903123D598A3A
:10CAE000088B09905157E493F890513B12CB885032
:10CAF000087405122E617401F090513512CB7E60DE
:10CB0000197A027901123D598A088B09905157E42C
:10CB100093F890513512CB8850087407122E617427
:10CB200001F0901CDEE0F97CBC7D1A7401122BE34D
:10CB30001243717ABC7B1A7945123C277407122E76
:10CB400061E070117405122E61E07009851882850C
:10CB50001983E480088518828519837401F0901C7C
:10CB6000D8E0F8901CD7E058F8851882851983E042
:10CB70005812CFD27941123C27741402C917E4939A
:10CB8000F8740193F9E84922E493FA740193FBE8FD
:10CB9000C39AF8E49BF9C3E50898E509992274F76C
:10CBA00012259474ED122C0BE9FE901AB8F0AC1813
:10CBB000AD19901CDEE0F97ABC7B1A12437774122F
:10CBC000122E61EE12CBDCAA18AB191243717ABC9B
:10CBD0007B1A7945123C27741302B3FDF0901CDEDA
:10CBE000E0F97CBC7D1A2274F4122594EAFEEBFF76
:10CBF000901CE0E064FE7003A3E0F470767A167B8C
:10CC00000012337B8A088B09EA450960668A828BA9
:10CC100083740112C2A68A828B83A360047402808B
:10CC2000027401F0EA240AF8E4350912C26912F12B
:10CC30000AA312DD08F0A2E3400912CC7612CC9CC4
:10CC40001243FBEE241512B9B1E5082402FAE435CB
:10CC500009FB123531E508241312CC88E4F0AA0848
:10CC6000AB09901AB9E0F912338712CC7612D5408D
:10CC700012CCAB028FD112CC7A22EE240BF582E4D7
:10CC80003FF58322E5082412F582E412BF7C228E50
:10CC9000828F83A3A3A3A3A3A3A3A3A312D1D02270
:10CCA000E0F8A3E0F9851882851983E8F0A3E9F09C
:10CCB0002274F212259474FD122C0B8A088B0989B8
:10CCC0000A8C0B7401122E61740412CFD21244BB71
:10CCD0008A0C8B0DAE0CAF0DEE4F700302CD5F12C0
:10CCE000CD94740712DD0EE5082413FAE43509FB30
:10CCF0008A828B8312CDAA8A828B8312CDA9E50802
:10CD0000241512CC8812DD0812DD15E508240BF875
:10CD1000E43509F912CD6DE8F0A3E912DEA812445A
:10CD20003712DCF612CDB57401F07403650A6006A3
:10CD30007401650A700712CD7E7404800412CD7EE2
:10CD4000E4F0901CE012B02112CCAB7401650B70C2
:10CD50000312CD77EEFAEFFB123DFBE9F980027981
:10CD600010901CE074FEF0A304F0028B3EEE241839
:10CD7000F582E43FF58322EE128926E4F02212CDFB
:10CD8000867440F0A322EE12CD8B22240FF582E4AC
:10CD90003FF58322EE12F4753FF58312CD9F22E01A
:10CDA000F8A3E0F98882898322A3E088828983F04E
:10CDB000A308A9832212CDB922F0EE12CDBF2224FE
:10CDC00013F582E43FF5832274F4122594EAFEEB16
:10CDD000FF7A007B04901AB9E0F91234EF12CE6F9B
:10CDE000901A6E7409F01244378A088B09AC08ADAA
:10CDF0000912B97012CC9C12352BE96401705A7A71
:10CE00000F7B0012337B8A088B09EA4509604A8A46
:10CE1000828B83740212CE64F988828983A3E0FC3A
:10CE200088828983A3A3E0FBEC8A82850983A3A37C
:10CE300012E16E88828983A3A3A3E08A8285098395
:10CE4000A312CE5CFAA3E0FB794A123C27AA08ABF6
:10CE500009901AB9E0F9123387028FD1F0EE241548
:10CE600012BF6122F0EE241D12BF61F8A3E02290F0
:10CE700019F712D54E901C9FE8F0A3E9F09019F92C
:10CE800012D54E901C9DE8F0A3E9F02274F412250F
:10CE90009474FD122C0B8A088B097401122E617494
:10CEA0000212CFD21244BB8A0A8B0BAE0AAF0BEE32
:10CEB0004F700302CF7A12F494E412CFAFA3A3A36E
:10CEC000E06401700888828983A37420F085088259
:10CED000850983A3A3A3A3A3E064017009888289C1
:10CEE00083A3E0D2E6F0850882850983A3A3A3A3E8
:10CEF000A3A3E06401700A88828983A3E0D2E7805B
:10CF00000512B970740112CFC0E064017021850868
:10CF100082850983A3A312CF9B600312CF7F85086C
:10CF200082850983A3A312B00B12CD6E12CCAB8500
:10CF30000882850983A3A3A3A3A3A3A3E06401702C
:10CF40000712F005F0A3E4F085088285098312CC6E
:10CF50009C1244D9E9600412CF86F0EE241712CF58
:10CF60008212443712DCF612A32012CF8D12B9E4DC
:10CF7000FAEFFB123DFBE9F98002791002C054EE92
:10CF8000241612DD1D2212B9A8440422E0F8A3E001
:10CF9000F98E828F832212CFA1F58312D54EE849F4
:10CFA000228E828F8312BC7C241FF582E4382212E9
:10CFB000CFB32212CFB722F0850882850983A3223E
:10CFC00012CFB3A3A3A3A322A2F0E43385188285D2
:10CFD0001983F0AA18AB192274F512259474F31270
:10CFE0002C0B890AEAFEEBFF7508007509007C0D21
:10CFF0007D007900AA18AB1912336312C26A12D1EC
:10D0000087741F58600C7AD37B0012387379000242
:10D01000D0D7E8A2E55008740C122E617401F0E834
:10D02000A2E75008740B122E617401F0E8A2E674B6
:10D030000A5008122E617401F08008122E61E0641B
:10D040000170138E828F83A3A3A3A3A3A3A3E06085
:10D0500032EE241380128E828F83A3A3A3A3A3A3F3
:10D06000A3A3E0601EEE2415F582E43FF58312AA27
:10D07000416010AC08AD097402122E61AA82AB8324
:10D0800012353112CC7612CCA0740A122E61E064F3
:10D0900001703B12CC8F1244D9E97039EE240B1287
:10D0A000BADF901A62E0687003A3E0697027E508B0
:10D0B0004509601A1244378A088B09AC08AD097417
:10D0C00002122E61AA82AB8312352BE96007AA18DF
:10D0D000AB19123EAFA90A740D02B66D74F7122592
:10D0E0009474CD122C0BEAFEEBFF8E828F8312D14B
:10D0F000A5A2E0400302D18212D18EE054FE12EDCF
:10D100006D740D122BEB12D1B8124431E9707374A7
:10D110002A122E6112D19B70697C0D7D007900AAC4
:10D1200018AB191233637416122E6112CCA0742A34
:10D13000122E6112D187A2E55008740B122E617471
:10D1400001F0E8A2E75008740A122E617401F0E8B9
:10D15000A2E65004742080027422122E6112B9B724
:10D160007402122E61AA82AB831235318E828F83B4
:10D17000A3A3E0C0E0740C122E61D0E012CFD21253
:10D180003EA9743302B3FD12E305A3E0F8228E82B8
:10D190008F8312D932A3A3A3A3A32212B51E6404C2
:10D1A000228A828B83E0F812D1AB22A3E0C8240646
:10D1B000F582E438F583E022EA241EF582E43BF5AB
:10D1C00083E0F9EA241FF582E43BF58312D1D022F3
:10D1D00012F105FB22E9F87900740468600A740A08
:10D1E00068600574036870027901022B2274F612DC
:10D1F00025948A828B837424F0A3A37401F0123ED9
:10D20000018A088B09AE08AF09EE4F60108E828F3D
:10D210008312DEA6124437EE241A12E167EEFAEF0B
:10D22000FB02C91AC082C083901A5C02AD6FC08233
:10D23000C083901CDF02AD6FC082C083E9901CDF09
:10D2400002AD8DC082C083901AD57401F0E9A2E3CB
:10D2500050037403F0E9A2E15004E0D2E2F002C509
:10D260008874F612259479007C008A088B09780866
:10D2700012285FF8FF0796D294D294D294D294D217
:10D280008CD290D296D288D27C01800A7C0480060F
:10D290007C0280027C08901AD5E05C6004790280F0
:10D2A00005EC6002790102C91A74F4122594EAFEB1
:10D2B000EBFF8908123D838A0A8B0BA80AA90BE8A9
:10D2C00049604188828983A3A3A3A3E06036C39405
:10D2D00005503174016508601A88828983A3A3A36D
:10D2E000A3E06401600D88828983A3A3A3A3E06403
:10D2F00002700A8882898312CC9C123F6FEEFAEF8B
:10D30000FB123D8F028FD174F61225948A828B8393
:10D31000E07014A3A3A312CF9B600C8A828B8312AC
:10D32000CC9912416780047A007B0002C91AC0823E
:10D33000C083901A6EE0640870031244FD02C58831
:10D34000C082C0837C00EC75F003A4F8ADF0EDF969
:10D3500012D4167003A3E06B7018905146E493C08A
:10D36000E074D828F582741A3DF583D0E0F079C5D1
:10D3700080620CECC3940340CD7C00EC75F003A4F8
:10D38000F8A9F074D928F582741A129AE964FE702B
:10D3900003A3E0F4600F0CECC3940340DE7C00ECCC
:10D3A00012D3D77026EC75F003A4FCADF074D82C22
:10D3B000F8741A3DF988828983A312E16D90514671
:10D3C000E49388828983F0790080090CECC394038C
:10D3D00040CD79C702C58875F003A4F8A9F074D8C8
:10D3E00028F582741A12EEF522C082C0837C00EC0C
:10D3F00075F003A4F8A9F012D4167003A3E06B70C3
:10D400000912D3DE6004790180090CECC394034057
:10D41000DE790002C58874D928F582741A12EEF5F7
:10D420006A2274F212259474DD122C0BEAFEEBFFD3
:10D430007508009019DCE060076401600302D539CB
:10D44000901A5FE06E7003A3E06F7010EE4F7003F0
:10D4500002D52D75080112450302D539123D7D8A8A
:10D460000A8B0BEA450B700302D52D8A828B83A3AE
:10D47000A3A3A3E0640160108A828B83A3A3A3A368
:10D48000E06402600302D52D851882851983E412B9
:10D49000D547740B122E61E8F0A3E912CFD2123DEA
:10D4A00029E9700302D52D850A82850B8312D540A8
:10D4B00012CCAB7900123F63850A82850B8312DAA6
:10D4C0005B122E61AC82AD837418122E61AA82ABFE
:10D4D00083123531850A82850B8312BAE5742012D6
:10D4E0002E6112CCAB7422122E61E4F07C02850A0C
:10D4F00082850B83A3A3A3A3E0F9740D122BE3127F
:10D500004497850A82850B8312BAE57401122E6155
:10D51000E8F0A3E912CFD2123D2F750801E50A24E5
:10D520000CF582E4350BF583129B4C800C901A6C41
:10D5300012B9C7FAEFFB1245C3A9087423028B4046
:10D5400012D54E901CE02212B19F12D54E2212D558
:10D55000ABF922C082C08374FE122C0B9019DCE060
:10D560006004640170237901123F6912D591901A09
:10D570005FE8F0A3E912CFD27953123C27851882D5
:10D5800085198312CC9C12378F7402122B8D02C521
:10D5900088851882851983EAF0A3EB12D5A0F922B9
:10D5A000F085188285198312D5AB22E0F8A3E0221A
:10D5B00074F412259474F3122C0B8A088B09ECFE78
:10D5C000EDFF750A12EA45097005790002D69C90B4
:10D5D0001A5FE065087004A3E06509701D12443706
:10D5E0008A0A8B0BAC0AAD0BEEFAEFFB12352BE976
:10D5F0007005750A018003750A00851882851983F4
:10D60000E4F004122E6112DE9412CFD2123D1DE915
:10D61000602A7403122E61AA82AB83123CF9E9647A
:10D62000017019750A017403122E61AC82AD83EE8C
:10D63000FAEFFB12352BE96003750A009019DCE064
:10D640006004640170177412650A7011EEFCEFFD3E
:10D65000AA08AB09123D65E96003750A00EEFCEF0C
:10D66000FDAA08AB091245E1E9F8740A687005756E
:10D670000A01801D74A0687012EEFCEFFDAA08ABD1
:10D68000091245F3AA08AB091246057401650A7030
:10D69000097900AA08AB0912450FA90A740D028F77
:10D6A000CE74F6122594EAFEEBFF89089019DCE0AF
:10D6B00060046401701E1244FDE508F50978091242
:10D6C0002B7E790DEEFCEFFD7AFC7BFF12451B747F
:10D6D00001122B8D02C91A74F7122594EAFEEBFF92
:10D6E0008E828F83A3A3A3A3A3A3A3A3E060161298
:10D6F000D73D129BEE12CC9C124509E964017005DE
:10D7000012CC7680298E828F83A3A3A3A3A3A3A385
:10D71000E0602512B9AE12CC8F124509E9640170A0
:10D72000178E828F83A3A3A3A3A3A3A3A3A312CC27
:10D730009C1244F179018002790002B400EE2415B4
:10D74000F582E43FF5832274F212259474FD122CC5
:10D750000B8A088B09ECFEEDFF890B750A01740139
:10D76000122E61740412CFD21244BBEA4B60427491
:10D7700011122E61E0601412DE0DE412E30D8A82B4
:10D780008B83E0D2E7F012D7B4E4F012D7BE12CD0B
:10D7900099740312DA65EE88828983A3A3F0EF8877
:10D7A000828983A3A312B19E12DD2A123DFBE9F503
:10D7B0000A028B3CEA2414F582E43BF5832212F43E
:10D7C000743B2274F0122594EAFEEBFF890A750B74
:10D7D00001EE12DB273F12D92BF50C88828983A337
:10D7E000A3E0FA8882898312D91A12B97964046095
:10D7F0000A7AD37B0012387302D90AE50C122A2A5E
:10D8000002000215D8030BC2D8030CA8D80D80D88B
:10D810000EC2D8BFD89019DCE06007640160030233
:10D82000D8C2901A59E0A2E1400302D8C27900ABF5
:10D8300009123FF9EA4B603D8A828B83A3A3A3A31D
:10D84000A3A3E05418602E12CC761229A58A828BED
:10D8500083A3A31229A579008E828F83A3A3A3A3F8
:10D86000A3A3A3A3A312D90E12CC9C12401174043B
:10D87000122B8D802E7901AA08AB09123EC180427D
:10D880009019DCE0600464017038901A59E0A2E15C
:10D890005030AB091244EBAA08AB091244F1E96419
:10D8A000C5701F750B00801A9019DCE060046401DC
:10D8B0007010901A59E0A2E150081237B380037536
:10D8C0000A00EE2409F50EE43FF50FAC08AD09A9F6
:10D8D0000C850E82F58312CC9C123ED9850E828572
:10D8E0000F8312CC9C1244D9E9601F12BF5AC39413
:10D8F00002401712CC7612E2307003A3E069600A8E
:10D90000E50BA2E05004A90A80027900803112D907
:10D91000122212B9BF8A828B8322A3A3A3E0F8E468
:10D92000C8F9EA28F508E439F50922F58312D93255
:10D93000E02212D5ABF988828983A322122B8D7F36
:10D940000802281974EE12259474F5122C0B8A0A19
:10D950008B0B890D8C0E8D0F7E01EE122E61740AD9
:10D96000F0741D122E61E0F50CE9700FE50CC33365
:10D97000240AC0E0EE122E61D0E0F0AA18AB191212
:10D9800044BB8A088B09EA4509700302DA3D12C4D8
:10D99000D8350912DBDB7409F0A3E50DC43354E07C
:10D9A000450C12DBF4AC0EAD0FEEFAEFFB12353185
:10D9B000EE2408FE50010FE50D702F7C00741E123E
:10D9C0002E6112DA4C801D12DA44EA28F8EB39F99C
:10D9D0008882898312DBEF8882898312A1BCF0A33D
:10D9E0000EAF830CECC3950C40DDE508241712CC78
:10D9F000887401F0124437E508241AF582E43509E9
:10DA000012DA59122BEBAA0AAB0B123D05E9601989
:10DA1000E508241612CC887401F07403122BDBE5A0
:10DA200008241812CC8812CCAB850882850983A300
:10DA3000A312DA63AA08AB09123DFBE9FEEEF97402
:10DA40000B02C2ACEC25E0F8E433F92212DA5022E2
:10DA500012D5ABF9E8FAE9FB22F583EAF0A3EBF083
:10DA6000740322E50AF0A3E50BF02274F01225946A
:10DA700074F8122C0B8A088B0912DB26350912DC8C
:10DA80006FF8741F58F50A880BA3AE82AF83EEFCC3
:10DA9000EFFDAA18AB19123531EE2408FE50010F24
:10DAA000AC18AD197A807B1A12352BE9607374E0DB
:10DAB000550B7066AA0AEA2AFA7B0012341D8A0CFA
:10DAC0008B0DEA450D605A7C00801D8E828F83127B
:10DAD000C50312DA44E50C28F582E50D3912E16B35
:10DAE000EE2402FE50010F0CECC3950A40DD780CC9
:10DAF000122B7A780A122B7E7403122BEB7900E535
:10DB000008240B12CC8812CC9C1245337403122BC0
:10DB10008DAA0CAB0D12342380077AD37B00123808
:10DB200073740802D93CEA241DF582E42274F012D1
:10DB300025948A0A8B0B890D8C088D099018FC128C
:10DB4000CF9B60757410122E61E0F50C12DA45E877
:10DB5000240EFAE439FB12337B8A0E8B0FAE0EAF24
:10DB60000FEE4F60548E828F8374D4F012DBCAA301
:10DB7000A3E50DF0AC08AD09EE2405FAE43FFB1275
:10DB8000353112DBBCE50CF07411122E6112E2F695
:10DB90007808122B76AC0CEC2CFCE433FDEE240E52
:10DBA000FAE43FFB1233577403122B8DEEFAEFFBAE
:10DBB0009018FC12E30112277A02D93FEE12DBC162
:10DBC00022240DF582E43FF58322A3A3E50AF0A306
:10DBD000E50B12DBD62212BFA0A322F58312DBEAEB
:10DBE000FF8E828F832288828983E0FEA3E022E079
:10DBF0008E828F83F0A3AE82AF832274F6122594B7
:10DC000074F8122C0B890812DB263B12DC6FF974B6
:10DC10001F59F88909A3AE82AF837401687042EE80
:10DC2000FCEFFDAA18AB19123531EE2408FE5001A5
:10DC30000FAC18AD197A807B1A12352BE960297464
:10DC4000E05509701C8E828F83A3E0FA8E828F8349
:10DC5000A312C5058E828F83E0F9124563A908805F
:10DC6000097AD37B001238737900740802C917F55A
:10DC700083E02401FEA3E03400FF8E828F83E02244
:10DC800074F012259474FD122C0B8A0A8B0B8C08ED
:10DC90008D09890D750C017401122E61740312CF68
:10DCA000D21244BB8A0E8B0FAE0EAF0FEE4F603F09
:10DCB00012CD94740BF0A3E50D12DD0E7413122E29
:10DCC0006112DD0812DEA812443712DCF612DD15EF
:10DCD000EE2418F582E43F12DD288E828F83A3A301
:10DCE000E50AF0A3E50B12DE9B123DFBE9F50CA95A
:10DCF0000C740302D93C12DCFEEAF0A3EB22EE2402
:10DD00001AF582E43FF58322E08882898322F0A31A
:10DD1000A882A98322F0EE241612DD1D22F582E4EA
:10DD20003FF5837401F02239F58312DE94F02274FA
:10DD3000EF122594EAFEEBFF751000EE12DB273F91
:10DD400012DF7BF508A3E0F50912D73D12CC9C1237
:10DD50003D83EA4B700302DE088A828B83A3A3A370
:10DD6000A3E0700302DE08C39403400302DE08E56B
:10DD700008C3940F5004E50960057510018079EA25
:10DD80002412F582E43BF583E4F0E508702290501C
:10DD9000147808122D3A12DE0D7808122DF29050E8
:10DDA000147808122D3A12E7647808122DF280399F
:10DDB00075090074027808122D1474142508F58270
:10DDC000745012CC8B780C122D3A90813E78081248
:10DDD0002DD4780C790812242F12DE0D780C122D18
:10DDE000F212E764780C122DF2EA241BF582E43B70
:10DDF000F5837401F01237FB9019CAE0FCA91012E8
:10DE0000CC7612CC9C12454B7F09022819EA2417C4
:10DE1000F582E43BF5832274F012259474F5122CFC
:10DE20000B8A088B09890B8C0C750A017401122E60
:10DE300061740312CFD21244BB8A0E8B0FAE0EAFA9
:10DE40000FEE4F604812CD94740C12DA65A3E50C06
:10DE500012DEA8124437EE241AF582E43F12DA5992
:10DE6000122BEBAA08AB09123D05E9600E12CF7F19
:10DE70007403122BDB12CD6D12CCAB8E828F83A379
:10DE8000A312DE9412DE9B123DFBE9F50AA90A7487
:10DE90000B02D93CE508F0A3E5092212CDB97401C3
:10DEA000F0EEFAEFFB227401F0EE241712DD1D22D2
:10DEB00074F012259412DB263B12DF7BF8A3E0FE00
:10DEC000E8600302DF7874016E600874026E60031C
:10DED00002DF78EE9019CAF07508CA75091978083A
:10DEE000122B7A7508017509007808122B7A7C00CC
:10DEF0007D007A517B001234A17404122B8D7402C0
:10DF00006E7075901CC0E0700A9050147808122D45
:10DF10003A8028F50874027808122D147414250824
:10DF2000F582745012CC8B7808122D3A90813E788D
:10DF30000C122DD47808790C12242F908116780CAD
:10DF4000122DD47808790C122525908106780C12B0
:10DF50002DD47808790C12242F9019CC7808122D22
:10DF6000F29019CC12299D7A007B40901AB9E0F901
:10DF70001234E97404122B8D02D93FF583E0240199
:10DF8000F8A3E03400F988828983E02274F6122530
:10DF90009474DA122C0BEAFEEBFF12CF9660508ECF
:10DFA000828F8312CC9CAC18AD1912D1B812441FC9
:10DFB0007409122E6112E2307003A3E0696030121E
:10DFC000E2FD1229A57508FE7509FF7808122B7A63
:10DFD000741C122E61E0F9740D122E6112B9B7741F
:10DFE0000F122E6112CC9C1240117404122B8D74EE
:10DFF0002602C91774F7122594E9FD7A007B009078
:10E0000019DCE06004640170407C00800B12E0A029
:10E01000E02AFAA3E03BFB0C90515712EEE35029A3
:10E02000EC75F01CA4F8AEF0EEF912EF05F460E721
:10E03000740328F58274063912CF9960DAED60CD49
:10E0400012E0A0E4F0A3F080CE7C00800B12E08D03
:10E05000E02AFAA3E03BFB0C12EEE0502DEC75F049
:10E0600017A4F8AEF0EEF912F0847003A3E0F460A8
:10E07000E6746428F582740B3912CF9960D9ED608B
:10E08000CC12E08DE4F0A3F080CD02B400EC75F08A
:10E0900017A4F8EEF9746428F582740B39F583221D
:10E0A000EC75F01CA4F8EEF9740328F582740639B7
:10E0B000F5832274EC122594890CEAFEEBFF901A8A
:10E0C000B8E0C3950C503B12448B901AEA12E10958
:10E0D000901A52E0F508E4F509F50AF50B90817EF7
:10E0E0007810122DD47808791012242F7808122B6A
:10E0F000727A007B02901AB9E0F91234E3740412C8
:10E100002B8D0287398A828B83EEF0A3EFF0227485
:10E11000F6122594EAFEEBFF901AD68013888289C6
:10E1200083E06E7003A3E06F603A88828983A3A3C3
:10E1300012CF9B70E87A047B0012341D8A088B0989
:10E14000A808A909E849601C8882898312E109901E
:10E150001AD612CC9C88828983A3A312E16D901AEF
:10E16000D612CCAB02C91AF582E43FF583EAF0A3DC
:10E17000EBF02274F41225947E00901AD680070EDC
:10E180008A828B83A3A312B30B70F4EE25E0FAE42A
:10E1900033FB12341D8A088B09EA4509607F7C0035
:10E1A000901AD680228A828B83E0F50AA3E0F50BD1
:10E1B00012DA44E50828F582E50939F58312DA63B5
:10E1C0000C8A828B83A3A312B30B70D9901AB4125A
:10E1D000E2307003A3E0697808701C122B7AEEF528
:10E1E0000A780A122B7E7C807D1A7900901AB4126C
:10E1F000CC9C124533801A122B7AEEF50A780A125B
:10E200002B7E7C807D1A7900901AB412CC9C12452A
:10E21000277403122B8DAA08AB09123423123E1364
:10E22000028FD18E828F83A3A3A3A3A3A3A3A3A3AF
:10E2300012D54E901A5FE06822C082C08380128A95
:10E24000828B83A3A312BAE5901AD612CCAB1234F8
:10E2500023901AD612B30B70E602C58874F5122506
:10E2600094901A6C12BC73901AEA12A03B12CCABB9
:10E270007AEA7B1A7950123C27901AEA12E2F68069
:10E280001312EBAD7004A3E06509600612EBBA123D
:10E2900045CF050A90514AE493F8E50AC398502007
:10E2A000E50A75F017A4F8A9F012EA5B6E7003A3F3
:10E2B000E06F70CD745928F582740B12DD2780D27F
:10E2C000901AEA12BC739018FE12CF9B60257A0652
:10E2D0007B0012337BEA4B601A8A828B8374D5F001
:10E2E000A3A3E412E6A80412E30D9018FE12E301C2
:10E2F00012277A02B670128748750A00228E828F22
:10E300008312E3052212D5ABF58388822212B1ABCA
:10E31000EEF0A3EFF022C082C083901A5FE064FEAB
:10E320007003A3E0F4600E901A59E0A2E1500612C7
:10E3300045E712458D02C58874F0122594901AADF8
:10E34000E06053F50CE4F50DF50EF50F90810678BD
:10E3500008122DD4780C790812242F1233758A08EC
:10E360008B09A808A90990513DE49358F508A3E446
:10E370009359F509E4F50AF50B780C7908122CEE9F
:10E38000780C122B727A007B01901AB9E0F91234E2
:10E39000E97404122B8D02D93F74EE1225947E008D
:10E3A0007F008E0A8E0B123DAD750D00803BAA0DCD
:10E3B0007B00123DA78A088B09A808A909E84960D3
:10E3C0002688828983A3A3A3A3E060046404701752
:10E3D00088828983A3A3A3A3A3A3A3A3A3A3E0F9F0
:10E3E0001245F9E960010F050D905157E493F8E5E6
:10E3F0000DC39840B91245BD8A0E8B0F750C008075
:10E4000023AA0C7B001245C98A088B09A808A90910
:10E41000E849600EE8240F129AE6F91245F9E9601E
:10E42000010E050CC3E50C950EE4950F40D3EF2EBD
:10E43000FE700302E52F8E08750900740278081239
:10E440002D14AA08AB0912341D8A0A8B0BEA450B5E
:10E45000700302E52D750C008E08750900740278B2
:10E4600008122D14AC08AD0979FF123363750D0045
:10E47000805EAA0D7B00123DA78A088B09EA450938
:10E48000604C8A828B83A3A3A3A3E060046404701E
:10E490003D8A828B83A3A3A3A3A3A3A3A3A3A3E0E7
:10E4A000F91245F9E9F96026050C780A122B7AEE83
:10E4B000FD850882850983A3A3A3A3A3A3A3A3A384
:10E4C00012E5C012CC9C1245937402122B8D050DDF
:10E4D000905157E493F8E50DC3985006E50CC39F9F
:10E4E0004090750C00C3E50C950EE4950F5040AAC2
:10E4F0000C7B001245C98A088B09EA4509602AEAA3
:10E50000240F12B003F91245F9E9F9601C780A12D8
:10E510002B7AEEFDE508240E12CC8812E5C012CC51
:10E520009C1245937402122B8D050C80B87E007FDF
:10E5300062901A57E0600BF91242BDE9F87454C3B7
:10E5400098FF75F003EF84F50D94204003750D1FBF
:10E55000850A08850B09750C00EF6005750C207F96
:10E5600000E50DC39E5005850D0F80088E0FE50C4C
:10E57000D2E6F50CAC08AD09AA0CA90F124599E931
:10E58000F50EE50CA2E6401D150F7800800BE5089E
:10E590002404F5085002050908E8C3950F40EFE58B
:10E5A0000FCEC39EFEE97006E50CA2E650A8E50A70
:10E5B000450B6007AA0AAB0B123423A90E02C2AFA7
:10E5C000E0FC8508828509832274F2122594EAFE14
:10E5D000EBFF89088C098D0A7C007D00740E122ED9
:10E5E0006112CC9C750B00800DEAFCEBFDEA240463
:10E5F000FA50010B050BE50BC3950A400302E698A0
:10E600008A828B83E0F47003A3E0F4607AEC4D60BF
:10E610000C8C828D83C3E09EA3E09F50CC8A828BBA
:10E620008312E69BEE98EF9950BFEAF8EBF98882E7
:10E630008983E0F47003A3E0F46010E82404F85048
:10E640000109050BE50BC3950A40E3E8FCE9FDE889
:10E6500024FCF8E934FFF98882898312E6A08C82D1
:10E660008D83E50CF0A3E50D12E6B78C828D83A3B4
:10E67000A312E6ADA3A3A3E08C828D83A3A3A3F092
:10E68000C3EA98EB9940C412E1058A828B83A3A365
:10E69000E50912E6A8E508F0028B4312D54EC32225
:10E6A000E0F50CA3E0F50D2212B19FA32212E6B112
:10E6B00022F0888289832212E6BDA3E02212E6B10D
:10E6C000A32274F212259474FD122C0B89088A0976
:10E6D000ECFEEDFF750A0175F003E9A42402C0E029
:10E6E0007401122E61D0E012CFD21244BBEA4B600B
:10E6F0007012D7BE12CD997408F0741F55084509E1
:10E70000A3F0E82402F8500109750A0080338E82D4
:10E710008F8312DD0812DD0E8E828F8312CDA98EBB
:10E72000828F83A3A3E05407C4FC8E828F83A3A3AC
:10E73000A3E054074C12CDABEE2404FE50010F05AC
:10E740000AE50AC3950840C68A828B83A3A374FC9A
:10E75000F0A374FFF012E7647401F0123DFBE9F5D9
:10E760000A028B3CEA2413F582E43BF5832274F120
:10E770001225948A0A8B0B7508007AFE7BFF7CFEBB
:10E780007DFFE50A12DB27350B12D92BF509741F23
:10E790005509F50CE82402F8500109E509A2E74003
:10E7A00065E50A2417F582E412F5A7FE75F003E586
:10E7B0000CA424026E704FE50C600612DBE6FBEE43
:10E7C000FA750D00801DE05407F50EA3A882A983F9
:10E7D000EEFC901A5FE06E7003A3E06F7003850E8D
:10E7E00008050DE50DC3950C502612DBE6FCE4CCC4
:10E7F000FDEE2CE43DFFE82402F8500109888289EF
:10E8000083E0548860C07AD37B0012387302E951E8
:10E81000E508700BA9091245A5E9700302E9511238
:10E82000E95612CC9C123D7D8A0C8B0DAE0CAF0DBF
:10E83000EE4F605A8E828F83A3A3A3A3A3A3A3E466
:10E84000F090514293F88E828F83A3A3A3A3A3A336
:10E85000A3A3E0C398402412E9605001097A027B27
:10E8600000122337E88E828F83A3A3A3A3A3A3A3BD
:10E87000A3F0E508C39407500205088E828F83A396
:10E88000A3A3A3A3A3A3A3A3E508F002E9517CFFDC
:10E890007DFF12E95612CC9C1245B18A0C8B0DAE4D
:10E8A0000CAF0DEE4F704F1245B78A0C8B0DAE0CAE
:10E8B000AF0DEE4F700302E9517C177D0079001215
:10E8C000336312E95612CF8C1287968E828F83A300
:10E8D000A3A3A3A3A3A3A312B9E412B52F74AA12EE
:10E8E000E97F5001097A027B0012233712DBBCE872
:10E8F00012E96B7401F0905142E49312BF69C3981E
:10E90000401912E9605001097A027B001223371284
:10E91000F00BE508C394075002050812EFF7E5086D
:10E9200012E970E4F012A033123CF9E97023850A71
:10E9300082850B83A3A3A3A3A3A3A3A3E06012E5F3
:10E940000A2415F582E4350B12B9C512A03412352C
:10E95000317F07022819E50A12F475350BF5832279
:10E96000905142E49379002401F822F012EFFB2247
:10E97000F012E97522EE240CF582E43FF58322F0D3
:10E98000905142E49379002401F82274F7122594FF
:10E99000E9FE74FE6A700374FF6B603474605E6439
:10E9A00060602DEEA2E5401CA2E6901A5F500DC3F8
:10E9B000E09AA3E09B5019790002B400C3E09AA347
:10E9C000E09B40F3901A5F12E69BEC98ED9940E7CC
:10E9D000790180E574F71225947E008008EE12EB31
:10E9E000B31245CF0E12EA1540F37E00EE75F00328
:10E9F000A4F8A9F074D828F8741A39F988828983A0
:10EA0000A374FEF0A30412E6ADE4F00EEEC394038B
:10EA100040DA02B40090514AE493F8EEC3982274AD
:10EA2000F71225947E0080010E12EA155026EE1290
:10EA3000EA6B6A7003A3E06B70EE12EA5B6C700322
:10EA4000A3E06D600A74FF6C700374FF6D70D912DF
:10EA5000EBBA80047A007B0002B40012EA5F2274F1
:10EA60005928F582740B39F583E02275F017A4F864
:10EA7000A9F012EA762212EED5E02274F61225945D
:10EA80007CFF7DFF7AFE7BFF1245B1EA4B703C753F
:10EA900008008032E50875F017A4F8A9F0745E2824
:10EAA000F582740B129AE9600512EEFA7016744F33
:10EAB00028FE740B39FF8E828F8312CC9C12401774
:10EAC000EEFAEFFB050812EACE40C902C91A9051CE
:10EAD0004AE493F8E508C39822C082C0837A007B99
:10EAE000007C00801012F07C7003A3E0F460050A43
:10EAF000EA70010B0C12EEE040EB02C58874F412D0
:10EB000025948A088B09ECFEEDFF800B1245CFEEB1
:10EB1000FCEFFDAA08AB091245B1EA4B70EE028F7B
:10EB2000D174F71225947D007C0080020D0C12EE4A
:10EB3000E0501C12F07C7003A3E0F460F0EDF8EA02
:10EB4000684B70E8EC75F017A4F812EBBA80047A01
:10EB5000007B0002B40074F7122594EAFEEBFFEE8E
:10EB60004F60187C177D0079001233638E828F838B
:10EB700074FEF0A30412F012F0A3F002B40074F6D5
:10EB80001225948A088B097E00801AEE75F017A46E
:10EB9000F8A9F012EBAD7004A3E06509600612EB72
:10EBA000BA1245CF0E12EA1540E102C91A12EA5F05
:10EBB00065082275F017A4F8A9F0744F28FA740BB1
:10EBC00039FB2274F41225948A088B09ECFEEDFFC0
:10EBD0009019DCE0600464017020901A6CE06E70A3
:10EBE00003A3E06F7014123D7D8A0A8B0BA80AA95B
:10EBF0000BE8496005E82408801AEEFCEFFDAA083E
:10EC0000AB091245B18A088B09A808A909E849602F
:10EC100009E8240DFAE439FB80047A007B00028FB6
:10EC2000D174F41225948A088B09ECFEEDFF750A65
:10EC300000750B00802FE50B12F06C123CF9E960B7
:10EC400022E50B12EA6B65087004A3E06509700306
:10EC5000750A0AEEFCEFFD12F07312352BE9600322
:10EC6000430AA0050B90514AE493F8E50BC3985072
:10EC700004E50A60C1A90A028FD174F61225947EB8
:10EC800000805AEEFA7B00123DA78A088B09A8087B
:10EC9000A909E849604688828983A3A3A3A3E06405
:10ECA00001603988828983A3A3A3A3E06402602C56
:10ECB000E82407129AE6FA74012AF0901AAEE0C32B
:10ECC0009A501988828983A3A3A3A3A3A3A3A3A370
:10ECD000A3E412ED62A312ED6D1240170E9051578E
:10ECE00012EA18409E7E008059EE75F017A4F8AA2B
:10ECF000F0EAF912F0847003A3E0F46044744F2842
:10ED0000F8740B39F9E8240C129AE6F8740128F02B
:10ED1000901AAEE0C3985029EE75F017A4F8EAF9FE
:10ED2000744F28F8740B39F9E812ED5C39F583E477
:10ED3000F0E8240EF582E439F583E412ED6D12401B
:10ED4000170E12EA1540A27A00EA12D3D760021415
:10ED5000F00AEAC3940340F102C91AEE240FF582C7
:10ED6000E42212E6BDA3A3A3A3A3A3A32212E6B1A8
:10ED700012D1D02274F11225948A0A8B0BECFEED8D
:10ED8000FF750E007A007B017508FE7509FF740F90
:10ED9000122E6112E6A08011123375E50EF5F0EA2D
:10EDA00084E5F0FA750E007B007C00800712EED53A
:10EDB0001287440C12EEE0505CEC75F017A4F8AD2D
:10EDC000F0EDF912F0847003A3E0F460E612EA7249
:10EDD000650A7004A3E0650B60D912F0677003A3A5
:10EDE000E06F60CF12EA72650C7004A3E0650D60FD
:10EDF000C212EEFA60BDC3940850B8E0640760AD7B
:10EE0000EB050E70AEE50EC39A40A8744F28F5824C
:10EE1000740B02EE9F9019DCE0600764016003024E
:10EE2000EEA77C00800712EF151287440C90515713
:10EE300012EEE35072EC75F01CA4F8ADF0EDF9128F
:10EE4000EF1064FE7003A3E0F460E112EF10650AB6
:10EE50007004A3E0650B60D412EF106E7003A3E0A2
:10EE60006F60C912EF10650C7004A3E0650D60BC03
:10EE700012EEEA60B7C3940850B212EF0564016065
:10EE8000ABE0640260A612EEEA64076099EB050E3F
:10EE9000709AE50EC39A409474F328F58274053D88
:10EEA000F58312CC9C802BE50E6011EA700E740184
:10EEB000650E600302ED987A0102EDA474FE650808
:10EEC000700474FF65096006AA08AB0980047AFE25
:10EED0007BFF02E951744F28F582740B39F58322C8
:10EEE00090514AE493F8ECC3982274FC28F582749C
:10EEF0000512EEF52239F583E022745D28F582745F
:10EF00000B12EEF52274F728F582740512EEF52245
:10EF100012EF15E02274F328F582740539F5832287
:10EF200074F51225948A088B09ECFEEDFF750A0032
:10EF30008002050A90514AE493F8E50AC3985022EA
:10EF4000EEFCEFFDE50A12F06C12352BE960E3E50B
:10EF50000A75F017A4F8A9F0744F28F582740B1203
:10EF6000DD2702B670E9F87907C3940D40047901F2
:10EF70008019E8C3940740047903800FE8C3940321
:10EF8000400479058005E870027900022B2274F0B4
:10EF90001225948A088B098C0A8D0B890C1245B7AF
:10EFA0008A0E8B0FAE0EAF0FEE4F60487C177D00C0
:10EFB00079001233638E828F8312DE9412F0121264
:10EFC000DA63E50C600712B52EE50C800312F0053C
:10EFD000F0901AB3E06401700612EFF7E4800512B6
:10EFE000EFF7740712E97F5001097A027B001223C0
:10EFF0003712F00B02D93F12EFFB22EE240EF582FE
:10F00000E43FF5832212CD86740122EE12DBC1E8C3
:10F01000F02212A9B4A32274F7122594EAFEEBFFA2
:10F02000750800803AE50875F017A4F8A9F012F009
:10F03000677003A3E06F601474FF6E700374FF6F5A
:10F04000701B12F0847003A3E0F4601112F07312CD
:10F050003CF9E97008E50812EBB31245CF05081238
:10F06000EACE40C102B40012EA766E2275F017A40F
:10F07000F8A9F0745128FA740B39FB22EC75F017DB
:10F08000A4F8A9F012EA7664FE22C082C0837AFF57
:10F090007BFF12460502C588C082C083901AEC74BB
:10F0A00017F0A37446F0901AEE741DF0A37446F0A6
:10F0B000901AF07423F0A3744602AD8D74F71225F4
:10F0C00094EAF8EBF99019F512F105CA2406F582D5
:10F0D000E43AF583E0702B88828983A3A3A3A3A3DA
:10F0E000A3A3A3A31229A59019F512F10A122E3297
:10F0F00088828983A3E0F9123ECD7402122B8D120F
:10F100003E1302B400E0FAA3E02212F105F5838A6F
:10F110008222C082C083901AB612F1D6F0901AB63D
:10F1200012CF9B7005790112455D02C58874F612F5
:10F13000259474FC122C0BE9FE905144E493700862
:10F1400074E16E600302F1D1EA2408F8E43BF98827
:10F1500082898312F1D612F1DF700E901AB6E4F0B4
:10F16000A3F0790112455D8068901CD4E06062F8DC
:10F17000901AB612CC9CC3E89AE49B5054790012C2
:10F18000455D8A088B09AC08AD09ECF8EDF9E87526
:10F19000F064A4F8AAF075F064E9A42AF9901AB60C
:10F1A00012CC9C12233FE8941AE994004023901853
:10F1B000F612CF9B601B901AB612CCA07402122ECE
:10F1C00061ECF0A3ED12CFD29018F612E3011227F2
:10F1D0007A740402C917E02401F0A3E0340022127B
:10F1E000E6B112D54EE84922C082C08374F8122CD1
:10F1F0000B9080D8AC18AD197408122A9EAC18ADCB
:10F200001912352BE96401700479008002790174C8
:10F210000802D58B74F6122594740C122E6112BC60
:10F2200073743A6E7001EF6006743B6E4F70237416
:10F230000A122E611229A58C088D097808122B7AE2
:10F24000EAFCEBFDEEFAEFFB1234A77404122B8DEF
:10F250008002790A02C91AC082C083901AF274B37C
:10F26000F0A3743DF0901AF474B9F0A3743DF090DB
:10F2700019CAE064017032901AF67441F0A3744622
:10F28000F0901AF87447F0A37446F0901AFA744D8F
:10F29000F0A37446F0901AFC7453F0A37446F090F7
:10F2A0001AFE743BF0A37446F0901AF612CF9B60DE
:10F2B0000612C8BD12277A02C58874F41225947408
:10F2C000E6122C0B8A088B097404122E617402F06A
:10F2D00004122BE31244BB8A0A8B0BAE0AAF0BEE6F
:10F2E0004F700302F44412F494746012CDB512DE30
:10F2F000A612443712DCF612B9E012DE9412BFC136
:10F300007012901A4BE0C0E012F449D0E0F0901A6D
:10F310004BE004F012F4657016901CB4E0600D90A0
:10F320001A56E0700A8E828F83E0700312CD77AC9C
:10F3300018AD19EEFAEFFB1244138A088B09EA455F
:10F3400009700302F43D7A217B0012341D74061209
:10F350002E6112E16D7406122E6112CF9B700302B2
:10F36000F4367C217D0079007406122E61E0FA12D9
:10F3700033637401122BE37950123C217401122E75
:10F380006112BAE57406122E6112F105CA2409F55C
:10F3900082E43AF58312CCAB901A5F12BAE5741787
:10F3A000122E6112CCAB7406122E6112BC7812F4CC
:10F3B0006BF07406122E6112B0EE740212F4BA747D
:10F3C00006122E6112F10A12CCAB7406122E6112D3
:10F3D000F49F12F4C5C0E07406122E6112BC7812BC
:10F3E000F47BD0E0F0EE240E12F453C0E074061269
:10F3F0002E6112F484D0E0F07406122E6112BC78F3
:10F4000012BC6912DD28EE240F12BADF740C122E22
:10F410006112CCAB8A828B83E0C0E0740E122E6145
:10F42000D0E0F07406122BE31243897406122E61A9
:10F4300012CC9C123423AA08AB09123423EEFAEF43
:10F44000FB123423741A028FCEEE2414F582E43FAB
:10F45000F5832212F458E022F8E43FF9E8FAE9FBD8
:10F460008A828B832212BF5E64012212F47538F502
:10F4700083740222EA240BF582E422241EF582E43E
:10F4800038F5832212F4882212BC7C240CF582E425
:10F4900038F5832212CC7A12CD9F7404F0A322E0B7
:10F4A00012F4A97401F0A3E422F8A3E0C812F4B1A5
:10F4B00022240DF582E438F5832212DBD612D54ED4
:10F4C00022E8F0A3E912A804E02274F61225947E43
:10F4D0000080187C047D0079FF8E088D0974027805
:10F4E00008122D1412F7051233630E90514112EADF
:10F4F0001840E002C91A74F412259474F7122C0B08
:10F50000750800802285080A750B007402780A12BB
:10F510002D1474EE250AF582740E12F5A724FFF05F
:10F52000A3E034FFF0050890514112EAD1506D85F7
:10F53000080A750B007402780A122D1412F59FF454
:10F540007003A3E0F460DE85080A750B007402788E
:10F550000A122D1474EE250AF582740E350B12CFA3
:10F560009970A27408122E617402F085080A750B56
:10F5700000780A122D1474EC250AFE740E350BFF68
:10F580008E828F8312CCA012F5AD123C697C047D73
:10F590000079FFEEFAEFFB123363808902B0E97461
:10F5A000EC250AF582740E350BF583E02212F71E66
:10F5B0002274EE12259474F7122C0BEAFEEBFF7501
:10F5C0000CFF7408122E6112F710123C63E9641AE2
:10F5D000700302F683750E00741B122E61780812F8
:10F5E0002DD4800B74FF650C7003850E0C050E90F6
:10F5F0005141E493F8E50EC3985048850E107511FB
:10F600000074027810122D1412F687F47003A3E030
:10F61000F460D1850E1075110074027810122D144B
:10F6200012F6876E7003A3E06F70C2750F0074024C
:10F63000780E122D1474EE250EF582740E350FF52A
:10F64000838030E493650E702D74FF650C602E8509
:10F650000C0E750F007402780E122D1474EC250E2A
:10F66000F8740E350FF98882898312E1098882893E
:10F6700083A3A312DD2A7901740902C2AC12F5AD8D
:10F68000123C69790080F174EC2510F582740E3516
:10F6900011F583E02274F412259474F7122C0BEA0E
:10F6A000FEEBFF7408122E6112F710123C69750808
:10F6B000008002050890514112EAD1504585080AA0
:10F6C000750B007402780A122D1412F59FF4700362
:10F6D000A3E0F460DE85080A750B007402780A1254
:10F6E0002D1412F59F6E7003A3E06F70C67C047D2D
:10F6F0000079FF8D0974027808122D1412F7051293
:10F70000336302B0E974EC2508FA740E3509FB2264
:10F71000740212A804EEF0A3EFF012F71E22901A62
:10F720006C12B9BFAA18AB192274EE1225948A087C
:10F730008B09ECFEEDFF750A00EE65087003EF65BE
:10F7400009600C12349B8A0C8B0DEA450D7006750E
:10F750000A0102F7E5EEFAEFFB12349B8A0E8B0FDB
:10F76000AC0EAD0FEC4D6007EEFAEFFB1234ADE4DA
:10F77000F50EF50F780E122B7AAC0CAD0DEEFAEFFC
:10F78000FB1234957402122B8DE96059AA0CAB0D53
:10F7900012341D8A0E8B0FEA450F6046780E122B2D
:10F7A0007A780C122B7A7C007D00AA08AB091234FF
:10F7B000A77404122B8DE9701D780E122B7A780C29
:10F7C000122B7A7C007D00EEFAEFFB1234A1740458
:10F7D000122B8DE96003750A01AA0EAB0F123423B8
:10F7E0008003750A10A90A02C2AF122398022B22C5
:10F7F000C082C08374FF122C0BAC18AD197A01794A
:10F800008712355B851882851983E0C39403400F06
:10F810007402F07C007D00FA79E2123591800CE4EC
:10F82000F0901CD3E0FA7B001236C37401122B8DCA
:10F83000D083D082022B2274F012259474F5122CFE
:10F840000B851882851983EAF0A3EBF0ECFEEDFF3F
:10F85000750820E9700302F9F7901806E0F47003C8
:10F86000A3E0F47062EE4F6073740A122E617403A9
:10F87000F07402122BE31235319017FFE0F508788F
:10F8800008122B7E7403122BEB7401122E6112FEF0
:10F89000619017FFE0F91241437401122B8DE9F5D5
:10F8A0000870247D007C007900EEFAEFFB1239D558
:10F8B00090815212299D7A007B0190186DE0F91217
:10F8C00034E37404122B8D851882851983E0FCA320
:10F8D000E0FDAA0879E112359102FA207508027458
:10F8E0000A122E617402F0122E6174FFF0A3F0125E
:10F8F000FA2FA3A3A31229A588828983A3A3A3A374
:10F90000A3A3A3A3A3E0FC7402122BE37901123892
:10F91000E57402122B8DE9602F7508007808122B10
:10F920007EE4F50AF50B780A122B7A7808122B7E02
:10F930007404122BDB880A890B780A122B7A12FACC
:10F940002A1229A57901805712FA2F1229A5888237
:10F950008983A3A3A3A3A3A3E0FC7402122BE379DE
:10F96000011238E57402122B8DE9700302F8C77595
:10F9700008007808122B7E7401122BDB880A890B91
:10F98000780A122B7A7508017808122B7EE4F50AA2
:10F99000F50B780A122B7A12FA2A1229A579007C23
:10F9A000FF7DFF740A122BE31239E17408122B8DCC
:10F9B000E9F508E508600302F8C7901A0BE0F50CBA
:10F9C000A3E0F50DE4F50EF50F780C122B727A001A
:10F9D0007B20901805E0F91234E37404122B8D8516
:10F9E0001882851983E0F8A3E0F9901806E8F0A3DF
:10F9F000E9F0802C124ACD7C00851882851983128B
:10FA0000FF9C124A6DEA4B70EB90815212299D7A4D
:10FA1000007B0190186DE0F91234E37404122B8D11
:10FA2000740B122B8D7F0802281912FFABA32290B2
:10FA30001802E0F8A3E0F988828983A3A3A3A3A313
:10FA4000A3A32274F712259474F7122C0B740812D6
:10FA50002E617402F0851882851983EAF0A3EBF019
:10FA60007D007C00AA18AB19123A4D7409122B8D37
:10FA700002FCB874F4122594E9FE7A007B409018D9
:10FA800005E0F91234EFEE700A7A0012FFA1124B72
:10FA90001580477A0112FFA1124B1574FF6E603A70
:10FAA000EEC3944140027E40EEF50875F0E8A4C52F
:10FAB00008A8F075F003A428F8E428F5093395E0C8
:10FAC000F50AF50B7808122B727A007B4090180526
:10FAD000E0F91234E37404122B8D7F0402281974A8
:10FAE000F412259474F4122C0B8C088D09E9FF7420
:10FAF0001B122E61E0FE74FE6A700374FF6B7009C6
:10FB00007408122E61E4F0801D851882851983EA3D
:10FB1000F0A3EBF07408122E617402F01244D9E9DC
:10FB20006004EEC2E4FE740A122E61E4F0A3F01247
:10FB3000FFA6C0E07409122E61D0E0F0741C122EF2
:10FB400061E0F50A780A122B7E741B122BDB880AFF
:10FB5000890B780A122B7A741B122E611229A5EFD9
:10FB6000F50A750B00780A122B7A7808122B7AEEB8
:10FB7000F97CFF7D177409122BE3124B39740912BB
:10FB80002B8DE9FA600E741A122E61E0FC7D00796B
:10FB9000E0123591740C122B8D02FADA74F61225EC
:10FBA00094E9FEEAFF8C088D09EEFA7B0012349B83
:10FBB000EAF9EFC3995004790180207808122B7A72
:10FBC000E9F5087509007808122B7A7C007D00EEB3
:10FBD000FA7B001234A77404122B8D802D74F61258
:10FBE0002594E9FEEAFF8C088D097808122B7AEF3C
:10FBF000F5087509007808122B7A7C007D00EEFA72
:10FC00007B001234A17404122B8D7F020228197418
:10FC1000F5122594E9601714601C14602114602605
:10FC200014602B14603014603F14604E80667508B9
:10FC300070750918802675083875090F8042750897
:10FC40005F75091A802875086275091A8020750881
:10FC50006475091A802A75086175091A750A007891
:10FC600008122B767C01802275086C75091A750ABA
:10FC7000007808122B767C02801075088075091AAE
:10FC8000750A007808122B767C087D0012335774B1
:10FC900003122B8D7F0302281974F7122594E9FEB5
:10FCA00074016E70097D007C0079001239D58008DE
:10FCB00074F71225941231EF7F0102281974F7129C
:10FCC00025941231F580F174F212259474FF122CF0
:10FCD0000B890A8A088B09EB5480700302FDE180CE
:10FCE0000FA3E0F91231E9EEFAEFFB123381A90A12
:10FCF0001233938A0C8B0DAE0CAF0DEE4F700302D6
:10FD0000FDD98E828F83E024E6603D24496074141F
:10FD1000700302FDB614601624F3700302FDBF14D5
:10FD2000700302FDC91460B924E5600B80B9EEFAD6
:10FD3000EFFB12358580B0A3E0FA8E828F83A3A3F8
:10FD4000A3E0F9123573809FEE2422F582E43FF59B
:10FD5000831229A5EE2420F582E43FF5831229A51C
:10FD60008E828F83A3A3A3A3E0FCA3E0FD8E828FEA
:10FD700083A3A3A3A312FE5F1232077404122B8D78
:10FD800002FCE7A3E0640660148E828F83A3E06424
:10FD900007600A8E828F83A3E064097005790002F0
:10FDA000FCE48E828F83A3E060076401600302FCA1
:10FDB000E7792202FCE412FE5F1231FB02FCE7A3AA
:10FDC000E0FA8E828F8302FD3FA3E0F98E828F835B
:10FDD00012FE5F12357902FCE7AA08E5096480800B
:10FDE0006FEB544060107A0012FFA1124B15AA0865
:10FDF000E5096440805AEB5420601B792190180675
:10FE000012FE6112357990180674FFF0A3F0AA086B
:10FE1000E5096420803AEB54107A006036790812C4
:10FE20004A8BAC18AD197A01790312355B851882BB
:10FE3000851983E0A2E2500512353D800D7CF47DEA
:10FE4000017B327A007902124A85AA08E50964101A
:10FE5000FB80027B007401122B8D7F06022819A300
:10FE6000A3E0FAA3E0FB2274F612259474F7122C97
:10FE70000BEA240CF582E43BF583E0F508A3E0F5FA
:10FE80000978081227CD00000200008094FE068049
:10FE9000B1FE54FF12399F8A828B83E5822403FCD2
:10FEA000E43583FDA3AA82AB83790112320102FFFC
:10FEB000541239A58A088B09AE08AF09901806E0DC
:10FEC000F47003A3E0F4700302FF547408122E616F
:10FED0007402F08E828F83A3E0F8A3E0F985188284
:10FEE000851983E8F0A3E9F08E828F83A3A3A3A3EF
:10FEF000E0F5087808122B7E7401122BEB9018069F
:10FF000012FF9C1241437401122B8DE970467A0056
:10FF10007B20901805E0F91234EF90815212299D50
:10FF20007A007B0190186DE0F91234E37404122B0F
:10FF30008D7D007C0079008E828F8312FE601239E5
:10FF4000DB790090180612FE611231F590180674E4
:10FF5000FFF0A3F0740902FC0774F7122594E990EE
:10FF60001805F090180674FFF0A3F09018007405BF
:10FF7000F0A37418F09017FFE4F0FA12FFA1124BEF
:10FF8000157A007B80901805E0F9123A7D7A067B9D
:10FF900080901805E0F9123A7D02FCB8E0FAA3E07F
:10FFA000FB12FFA6F92212FFABE022901802E0F844
:10FFB000A3E0F58388822274F412259489088A09C3
:10FFC000ECFEEDFF7A047B0012337BEA4B601E8A65
:10FFD000828B83E508F0A3E509F08A828B83A3A3D3
:10FFE000EEF0A3EFF0901805E0F912338702FADA89
:10FFF000FFFFFFFFFFFFFFFFFFFFFFFFFFFFFFFF11
:020000040001F9
:10000000C082C083790012CFA2C082C0839019F150
:1000100012C856D083D082C3E09CA3E09D500DEA65
:10002000240B12804F12802F60027901029E4BEA4E
:1000300075F00BA4FAA8F075F00BEBA428FB90194F
:10004000F3E02AF8A3E03B8882F583E0540F22F521
:1000500082E43B12B98B2274F7122594890812B0FE
:10006000A41283B7ACF075F00BE9A42CF99019F346
:10007000E028F8A3E039F9E8FEE9FF7401650860BB
:10008000067402650870228A828B8312856D740261
:1000900065087021EA2403FA50010B123CF9E9705B
:1000A000148E828F83E4F0800CEA2403FCE43B127C
:1000B0008564123CF38E828F83E0D2E7F01237C55D
:1000C00002AC5A74F412259412863E79008E828F07
:1000D00083E06078890A890B8063E50A75F00BA4D8
:1000E000FAA8F075F00BE50B12803B7048E50A7535
:1000F000F00BA4F8AAF075F00BE50B1285818E8247
:100100008F83E085088285098312A5321284E2EE8E
:100110002403FCE43F1281FA123CF312AEA8E50A74
:10012000F0A3E50B129B68D2E7F01237C579019076
:1001300019F112943B050AE50A7002050B9019F1BA
:1001400012C08EC3E50A9AE50B9B408E029B727427
:10015000F5122594EAFEEBFF750A01740B122E616D
:1001600012CCB3EC4D6015EC12BD583D12864C79A3
:1001700001123CDBE508450960758023E508450967
:10018000604412BD56350912864C1281FB123CF9AF
:10019000E96401701BEEFAEFFB123CE1E9F50A8518
:1001A00008828509831284DA7902AA08AB098011D2
:1001B000128565123CF9E9640170347903EEFAEFB7
:1001C000FB123CDB80298E828F83A3E064FE7003E8
:1001D000A3E0F4700B128565123CF9E96401700C20
:1001E000EEFAEFFB123CE1E9F50A8003750A000222
:1001F0008CCBE50A2403FCE4350BFDE5082403FA67
:10020000E43509FB2274F71225949019F112AFD846
:10021000EA4B602FEA75F00BA4FAA8F075F00BEB2F
:10022000A428FBEAFEEBFF12341D9019F312AFD89D
:100230009019F312ADED6012EEFCEFFD7900123370
:100240006380079019F3E4F0A3F002AC5AC082C0B7
:1002500083EC4D600512353180097C087D00790002
:10026000123363029E4BC082C0837900EA4B601652
:100270007800E8FCEA2C12B0B06004790178080834
:10028000E8C3940840EC029E4BC082C0837901EC25
:100290006A7002ED6B6011EA4B600BEC4D60071267
:1002A000352BE9F980027900029E4B74F7122594F0
:1002B00074F3122C0BECFEEDFF851882851983E494
:1002C000F004122E61EAF0A3EB12C14E123D1D7430
:1002D00003122E61AC82AD83EEFAEFFB123CF3EE1B
:1002E000FAEFFB123CF902AC5574F712259474F343
:1002F000122C0BECFEEDFF851882851983E4F0EAE1
:10030000FCEBFD7403122E61AA82AB83123CF3AAAC
:1003100018AB19123D237401122E6112A5438E826F
:100320008F8312AF9474FE68700374FF6960047960
:10033000018002790002AC5574F7122594EAFEEBB5
:10034000FF123CD5E9F5087401650870111283A20B
:10035000F4FA88828983E05A4480F01237C5A908EC
:1003600002AC5A74F7122594EAFEEBFF7508008E72
:10037000828F83E0602A123CD5E9F5087401650894
:10038000701E1283A2FA88828983E05A70128E82CC
:100390008F83E04480FA88828983E04AF01237C56F
:1003A00080BC12AD1CF81283B7128759F8A3E0394C
:1003B000F98E828F83E022A3E0F9E875F00BA4F8B0
:1003C0002274F41225948A088B097C007D00EA12BD
:1003D00081FD123CF3E5081284FC790085088285D2
:1003E0000983A3E064FE7003A3E0F460787E007FDD
:1003F000008065EEFAEFFB12802F6057EEFAEFFBFC
:10040000EA75F00BA4FAA8F075F00BEBA428FB90AA
:1004100019F3E02AF50AA3E03BF50B85088285096C
:100420008312C08D850A82850B83A3E06A7003A3C3
:10043000E06B701FE50A2403FAE4350BFB123CF96C
:10044000E9640170061281F2123CF31284F1790121
:1004500012C9BD0EEE70010F9019F112C08EC3EEDD
:100460009AEF9B408E029B7274F31225948A088B3C
:10047000098A828B831284DAEA1284FC750C00EA02
:100480001281FD123CF9E9640170477E007F008013
:100490003C12874BFAA3E0398A82F583E0540F605F
:1004A0002712874BF50AA3E039F50B1281F21235BA
:1004B0002BE964017012850A82850B831284E21293
:1004C00084F1750C0112C9BD0EEE70010F12876820
:1004D00040BFA90C7F05022819A3A374FEF0A30452
:1004E000F022A312AC46850882850983A312A24B91
:1004F00022E508128506EEF0A3EFF02212850674BD
:10050000FEF0A304F022240BF582E43509F58322E2
:1005100074F5122594EAFEEBFF8E828F831284DA43
:100520007C007D00128565123CF3EEFAEFFB123C75
:10053000D5E9F50A7401650A702712AC3F1285757A
:10054000850882F58312856D1281FB123CF9E964FE
:1005500001700EE5082403FCE43509128564123CA1
:10056000F3028CCBFDEE2403FAE43FFB22A312C07E
:100570009C12A24B22E875F00BA4F8AAF075F00BC0
:10058000E912875FF508A3E039F5092274F2122514
:100590009474E6122C0B12863E750A0175080075DC
:1005A0000900750C00750D00851882851983E4F02B
:1005B000EE2403FCE43FFD7403122E61AA82AB8398
:1005C000123CF3AA18AB19123D23E96401701F74A1
:1005D0000B122E6112864E7401122E6112C096709B
:1005E00003A3E069604AA818A91988088909740D4D
:1005F000122E6112A531A312A543740E122E6112A0
:10060000AF94740D122BE3123D1DE964017009745F
:100610000D122BDB880C890D780C122B7AAC08ADEF
:1006200009EEFAEFFB123CE77402122B8DE9F50A92
:10063000EEFAEFFB123D17A90A741A02AEBAEAFEEF
:10064000EBFF12AEAC74FEF0A304F022F58312C0EF
:100650007CF912AEAC12A24B22C082C08378007922
:1006600000800508E87001099019F1129850E99B83
:100670005029E8FAE9FBEA75F00BA4FAACF075F042
:100680000BEBA42CFB9019F3E02AFCA3E03B8C823B
:10069000F583E0540F70CC790080027901029E4B03
:1006A00074F61225947E007F008039EEF8EFF9127F
:1006B00085757808122B7A75080B75090078081271
:1006C0002B7AEEFCEFFDEC75F00BA4FC75F00BED56
:1006D000A42AFD7A237B001234A77404122B8D0EFA
:1006E000EE70010F12876840C2028BE374F6122588
:1006F000947E007F00804C12874BF8A3E039F98884
:10070000828983E0A2E75036C2E7F08582088583BC
:10071000097808122B7A75080B7509007808122BD6
:100720007AEEFCEFFDEC75F00BA4FC75F00BEDA47C
:100730002AFD7A237B001234A17404122B8D0EEE55
:1007400070010F12876840AF028BE3EEF8EFF9E813
:1007500075F00BA4F812875922AAF075F00BE9A4E2
:100760002AF99019F3E028229019F112AC46C3EE51
:1007700098EF992274F6122594E4F508F5097808A3
:10078000122B7A9019F112943675F00BA4FCA8F094
:1007900075F00BEDA428FD7A237B001234957402CA
:1007A000122B8DE9FE6003123D4D02C6B274F612A3
:1007B000259474FF122C0B7E007F00803C851882EC
:1007C000851983E412919E122B7A75080175090030
:1007D0007808122B7AEEFCEFFDEC75F00BA4FCA868
:1007E000F075F00BEDA428FD7A237B001234A17480
:1007F00004122B8D0EEE70010F12876840BF74013A
:10080000028BE0C082C083905157E49375F01CA422
:10081000FCADF079FF7AF37B05123363029E4B74D3
:10082000F7122594E9FCEAFD7A007B008010EB12B8
:100830008E799C4008E0F8EDC39840010A0B905176
:1008400057E493F8EBC39840E57B0002AC5A74EC94
:1008500012259474F3122C0B8A0C8B0D8C088D09C5
:10086000890AEC45096016AA08AB09123D838A0E75
:100870008B0FAE0EAF0FEE4F600302894C7A0080F3
:10088000010A90515712BFD3500F128A4170F2746F
:10089000F328FE740539FF80047E007F00EE4F7060
:1008A000030289F590513B128A1260257403650A90
:1008B00060067404650A70197A047903123D598A36
:1008C0000E8B0F905157E493F890513B128A2B50A6
:1008D0002D905135128A12602C7401650A600674DD
:1008E00002650A70207A027901123D598A0E8B0F37
:1008F000905157E493F8905135128A2B40077A00B3
:100900007B00028A0D8518828519837401F0122EEE
:1009100061E50CF0A3E50DF0AC08AD097403122EEF
:1009200061AA82AB83123CF3AA18AB19123D2F7453
:100930000B122E6112A2448E828F83A3A3A3A3A3C2
:10094000A3E412C852AA0CAB0D1245C37800E50A05
:100950006007C39405500278048E828F83E50CF003
:10096000A3E50D128D3CA3A3E50AF0E88E828F83E8
:10097000A3A3A3A3A312C3635001097A027B0012AD
:10098000233712982BA3129CCA129857E50A605B72
:10099000C394035056901CBFE07018905014780C0C
:1009A000122D3A129802122DF2905014780C122D3A
:1009B0003A8027F50875090074027808122D141280
:1009C0008A1C122D3A90813E7810122DD4780C7921
:1009D0001012242F129802122DF2EE2413129805F1
:1009E000122DF2EE241B12C35A800912980E1284A3
:1009F000DDA3F0A3F07A047900123D59128D2D4049
:100A000005901CD8E4F0124485EEFAEFFB740D0259
:100A1000A051E493F8740193F9E84922741425086D
:100A2000F58274503509F583780C22E493FA740149
:100A300093FBE8C39AF8E49BF9C3E50E98E50F9998
:100A400022EA128A47F42275F01CA4F8A9F074F780
:100A500028F582740539F583E02274EE122594742A
:100A6000F3122C0BEAFEEBFF8C108D11750800AA17
:100A700010AB11123D83EA4B7003028B758A828B97
:100A800083E06E7003A3E06F7003028B758A828B24
:100A900083A3A3A3A3E0C394054003028B758A82BA
:100AA0008B8312C9ABE060728A828B83A3A3A3A35A
:100AB000E0C394035064901CBFE070219050147800
:100AC00008122D3A128B7C122DF2905014780812D5
:100AD0002D3AEA2413128B7F122DF28030F508751F
:100AE000090074027808122D14128A1C122D3A90F3
:100AF000813E7808122DD4780C790812242F129A8E
:100B00002C122DF2EA2413129A2F122DF2EA241B32
:100B1000F582E43BF583E4F0801B7508FE7509FF60
:100B2000750AFF750BFF128B7C122DF2EA2413124B
:100B30008B7F122DF2750800750900750A00750B80
:100B400000EA240C128B7F122DF2851882851983FE
:100B50007401F0122E61EEF0A3EFF0AC10AD117441
:100B600003122E61AA82AB83123CF3AA18AB1912AE
:100B70003D2F750801A908740D02C9A3EA2417F5D1
:100B800082E43BF58378082274F6122594123D7DA9
:100B90008A088B09A808A909E84960148882898312
:100BA000A3A3A3A3E06009C39405500479018002C4
:100BB0007900802F74F6122594123D7D8A088B09E6
:100BC000A808A909E849601488828983A3A3A3A37C
:100BD000E06009C394035004790180027900800326
:100BE000122B8D7F0202281974F6122594123D7D76
:100BF0008A828B83E5824583600BA3A3A3A3E07065
:100C00000479018002790080DAC082C083EAFCEBBB
:100C1000FD7A007B00029E48C082C0837C007D007C
:100C2000029E4874F512259474F3122C0BEAFEEB25
:100C3000FF8C088D09C3EC94F8ED94FF4004EE4F4F
:100C40006065750A00801974FF6508700474FF659B
:100C500009600B12CF9C7004A3E06509603B050A94
:100C6000905157E493F8E50AC398503BE50A128A7D
:100C70004260EBEE4F60D0128CB2122E6112C14A6C
:100C8000123D29E960D87403122E61AC82AD83EE67
:100C9000FAEFFB12352BE960C5E50A75F01CA4F8E4
:100CA000A9F0128E7080047A007B00740D122B8DD7
:100CB000801B8518828519837401F074F528F582EC
:100CC000740539F58312AC46740B22A90A7F03021E
:100CD000281974F412259474F3122C0B7508001261
:100CE0003D838A0A8B0BAE0AAF0BEE4F6025851849
:100CF00082851983128D3A128CC5122E6112C14A57
:100D0000123D117C1C7D0079FFEEFAEFFB1233637C
:100D10007508017A047900123D59128D2D50099001
:100D20001CD87401F0124485A908029B6D9051579C
:100D3000E493F8C3EA98EB940022740112A536A359
:100D4000A32274F7122594E9FE74FE6A700374FFFF
:100D50006B7C00700380240C128DA5501EEC128A4F
:100D60004260F4128F3F7003A3E06B70EA800BECDB
:100D7000128DBA6019E0640360140C128DA5501E28
:100D8000EE60ECEC128DAF60F1C3940550ECEC75A5
:100D9000F01CA4FCADF012D51212C08E80047AFEB5
:100DA0007BFF02AC5A905157E493F8ECC39822753C
:100DB000F01CA4F8A9F0128A4E2275F01CA4F8A920
:100DC000F0128A4E640122123D95029E4BC082C0F1
:100DD00083790180F274F01225948A0A8B0B7A04CD
:100DE0007901123D598A0C8B0DEA450D6040EA2AC3
:100DF000FAEB33FB12341D8A088B09AE08AF09EEFB
:100E00004F60267AFE7BFF123D9B74FE6A7003746E
:100E1000FF6B601E85088285098312AFD8E5082420
:100E200002F50850E2050980DE750C0080047E00A2
:100E30007F00850A82850B83E50CF0EEFAEFFB025A
:100E40009106C082C0837C008009EA24FF1AEB343B
:100E5000FFFB0C128DA55011EC128E79940550F207
:100E6000EA4B70E6128E7080047A007B00029E4B83
:100E700074F328FA740539FB22128A47C32274F7E7
:100E800012259474F3122C0B7E00807DEF75F01701
:100E9000A4F8A9F0128F3012C08EEE75F01CA4F8E1
:100EA000A9F0128F3F7003A3E06B603DEF75F01760
:100EB000A4F8AAF0EAF9128F3012A5437401122E99
:100EC00061E0687003A3E069601FEF75F017A4F894
:100ED000EAF9745128FC740B39FD7403122E61AACF
:100EE00082AB8312352BE96013EF75F017A4F8A9D4
:100EF000F0744F28FA740B39FB1245CF0F90514A0A
:100F0000E493F8EFC39840840E12D4FF501FEE1202
:100F1000DA7DF47003A3E0F460EE128CB2122E615D
:100F200012C14A123D29E960DF7F0080D002AC5532
:100F3000128F3422744F28F582740B39F5832212F4
:100F4000DA886A2274F412259474F3122C0B7E0052
:100F5000803890815E7808122DD4EE75F01CA4F8CC
:100F6000A9F0740628F582740639F5837808122CE6
:100F70006260169081127808122DD4EE75F01CA4D0
:100F8000F812900C7808122CC80E12D4FF507AEE8A
:100F9000128DAF60F4C3940350EF12900C122E0E1A
:100FA000E8494A4B70AC9019CAE06401702D901A60
:100FB000FA12ADED6025EE75F01CA4F8A9F074F3FB
:100FC00028F8740539F912906212299D8882898364
:100FD0001290F712277A7404122B8D8518828519C6
:100FE000837401F0EE75F01CA4F8A9F0128CBB120A
:100FF0002E6112C14A123D29E9608E7403122E61DE
:10100000AA82AB83123D8F8080029B6D740A28F503
:1010100082740639F5832274F6122594123D7D8A76
:10102000088B09A808A909E849603288828983A346
:10103000A3A3A3E06023C39403501E129062122E58
:101040001AE82417F582E439F583122E3EE8241BB2
:10105000F582E439F5837401F079018002790002A8
:101060008BE3E82413F582E439F5832274F012252A
:1010700094EAFEEBFF901AF412ADED6072901AFA4A
:1010800012ADED606A901AFE12ADED606212D38B64
:1010900012277AE97059901CBFE0700A90501478BA
:1010A00008122D3A8028F508750900740278081294
:1010B0002D1412D56D745012D36C7808122D3A90FD
:1010C000813E780C122DD47808790C12242F7808E0
:1010D000122B721290F112277A7404122B8DE9648C
:1010E00001700C8E828F83A3A312D37912277A808A
:1010F000158E828F83A3A312B98D901AFA12D3830F
:1011000022740D122B8D7F0802281974F612259473
:10111000E4F508F5097808122B7A905157E493F515
:101120000874037808122D1412942812349574024E
:10113000122B8DE9FE740A6E6025E4F508F5097836
:1011400008122B7A905157E49375F005A4FCADF08A
:101150007A3F7B001234957402122B8DEE600312DD
:101160003DCB02C6B274F612259474FE122C0B8588
:101170001882851983E4F0A312919E122B7A7508C8
:10118000027509007808122B7A7C007D007A227B98
:10119000001234A17404122B8D7402028BE0F0A8AB
:1011A00018A9198808890978082274EE1225947400
:1011B000DE122C0B8A0E8B0F8C088D09750C007AB1
:1011C000227B0012349B8A0A8B0B7A3F7B001234FD
:1011D0009B8A108B11AE10AF11E50A450B6017E525
:1011E00008650A7004E509650B600BAC0AAD0B7A63
:1011F000227B001234AD7436122E6112943BEE4FF6
:101200006015E50A6E7003E50B6F600BEEFCEFFDF9
:101210007A3F7B001234ADE4F510F5117810122BF3
:101220007AAC08AD097A227B001234957402122B35
:101230008DE9640A700302941EE4F508F509780844
:10124000122B7AAC0AAD0B7A3F7B001234957402F4
:10125000122B8DE9640A700302941E7404122BDBB6
:10126000880889097808122B7A75080275090078B0
:1012700008122B7A7C007D007A017B031234A7745C
:1012800004122B8DE9600302941E85188285198350
:10129000E4F0A3F07E000293957406122BDB88081D
:1012A00089097808122B7A750808750900780812E0
:1012B0002B7A8E0874037808122D14E5082402FC9A
:1012C000E43509FD7A017B031234A77404122B8DD7
:1012D000E9600302941E7408122E61E0F47003A307
:1012E000E0F470030293947406122BDB88088909DA
:1012F0007808122B7A7508087509007808122B7A7D
:101300007404122E6112CCB374037808122D1412D7
:1013100094281234A17404122B8DE9600302941EE8
:101320007402122BDB880889097808122B7A750859
:10133000057509007808122B7AEE75F005A4FCAD4E
:10134000F07A027B031234A77404122B8DE97041EA
:101350007402122BDB880889097808122B7A750829
:10136000057509007808122B7A7404122E61129404
:101370003675F005A4FCA8F075F005EDA428FD7AFB
:101380003F7B001234A17404122B8DE96003029498
:101390001E1299440E851882851983C082C08390DD
:1013A0005157E493F8D083D082C3E098A3E094002F
:1013B0005021851882851983C082C0837404122E3F
:1013C0006112A543D083D082C3E098A3E099500373
:1013D000029299A818A919880889097808122B7A05
:1013E0007508027509007808122B7A7C007D007A56
:1013F000227B001234A17404122B8DE97020AC0EF4
:10140000AD0F7A017B031234ADE970127434122EE1
:101410006112C8567A027B031234ADE96003750C81
:1014200001A90C742202C9A3E5082402FCE43509D1
:10143000FD7A227B002212C85AEC22E0F50AA3E0D2
:10144000F50B2274EC12259474FE122C0B750A0015
:10145000851882851983E4F0A3F090515793F50E17
:10146000F50875090074037808122D14E5082402A4
:10147000F50850020509E50E75F005A4F50EE5F036
:10148000F50F7A227B0012349B8A0C8B0DAE0CAFC9
:101490000D7A3F7B0012349B8A108B11A818A91972
:1014A000880C890D780C122B7A750C02750D00785A
:1014B0000C122B7A7C007D007A227B001234A774F8
:1014C00004122B8D7A017B0312349B8A0C8B0D7ACC
:1014D000027B0312349B8A128B13A812A913E50C0A
:1014E000450D700AE5086E7003E5096F7025E8493F
:1014F000700CE50E65107004E50F65117015E50CB4
:10150000450D607BEE4F604E85188285198312AFC2
:10151000DE60437C017D037A227B00124659E9F8A4
:10152000880A705B7C027D037A3F7B00124659E992
:10153000F8880A704AEEFCEFFD7A227B001234AD87
:10154000E9700EAC10AD117A3F7B001234ADE9604A
:1015500011750A018029AE0CAF0DE84960048810AE
:101560008911780E122B7A7810122B7AAC08AD09FB
:10157000EEFAEFFB123DD17404122B8DE9F50AA9A6
:101580000A740202A05174EC12259474D0122C0B30
:10159000851882851983E4F0A3F0123DD7E9600332
:1015A0000297EAA818A919880889097808122B7ADD
:1015B0007508027509007808122B7A7C007D007A84
:1015C000227B001234A77404122B8DE9600302976A
:1015D000EA905157E493F885188285198312985040
:1015E000E49B50030297EA750A00750B007508002A
:1015F000803D7403122E61122E0E129821122E4A73
:101600007403122E61122E0E12A868122E4AEE24B6
:101610001BF582E43FF583E4F07A047900123D592A
:10162000128D2D4005901CD8E4F012448505081257
:1016300097F740030297EA12A53DC3E50A98E50B28
:101640009940030297EA7414122BDB880C890D78F9
:101650000C122B7A750C08750D00780C122B7A85FC
:10166000080C7403780C122D14E50C2402FCE435EC
:101670000DFD7A227B001234A77404122B8DE970C1
:10168000AC7416122E61E0F47003A3E0F4609E05C2
:101690000AE50A7002050B7407122E617401F074DA
:1016A00016122E6112A5437412122E6112AF947499
:1016B00007122BE3123D29E9700302962D12C8533D
:1016C0007414122E6112C08E1245C3E50875F01C09
:1016D000A4F8A9F074F328FE740539FF7414122BD2
:1016E000DB880C890D750E00780C122B767C087D3A
:1016F00000EEFAEFFB1233577403122B8D12C368FE
:101700005001097A027B0012233712982B12985746
:101710007402122BDB880C890D780C122B7A750C55
:1017200005750D00780C122B7AE50875F005A4FC00
:10173000ADF07A3F7B001234A77404122B8DE96060
:1017400003029619908112780C122DD47403122E74
:1017500061780C122C6260030295F2E50875F01CAA
:10176000A4F8AAF0EAF9128DB66071C39403506C24
:10177000901CBFE07018905014780C122D3A1298FB
:1017800002122DF2905014780C122D3A8033F50C81
:10179000750D007402780C122D147414250CF5824A
:1017A000745012B95B780C122D3A90813E78101269
:1017B0002DD4780C791012242FEAF9129802122DE8
:1017C000F2EE2413129805122DF2E50875F01CA410
:1017D000F8740E28F58274063902961512980E04D4
:1017E000141284DDA3F0A30296188518828519834C
:1017F000E0F9743002A051905157E493F8E508C322
:101800009822EE2417F582E43FF583780C22129893
:101810002174FEF0A304F0A3F0A3F012A86C74FEF0
:1018200022EE2417F582E43FF58322E88E828F832F
:10183000A3A3A3A3A3A3A3A312AC1A740112AC1A6B
:10184000A374AAF0EE2410F582E43FF583E4F022BD
:1018500012B98DC3E89A22A3F012AEACE4F0EE24E4
:101860000CF582E43FF583E4F0A3F0A3F0A3F022AB
:1018700074F212259474FE122C0B8518828519833C
:10188000E4F0A3F075080002990FE50875F01CA4B8
:10189000F8A9F074F328F50C740539F50DAE087845
:1018A0000C122B7A750A08750B00780A122B7A8EA7
:1018B0000A7403780A122D14E50A2402FCE4350B9D
:1018C000FD7A227B001234A17404122B8DE50C24C6
:1018D00012F50AE4350DF50B780A122B7A750A0514
:1018E000750B00780A122B7AEE75F005A4FCADF0AA
:1018F0007A3F7B001234A17404122B8D850C8285F3
:101900000D83A3A3A3A3E0F4600312994405081276
:1019100097F7500302988AA818A9198808890978A6
:1019200008122B7A7508027509007808122B7A7C48
:10193000007D007A227B001234A17404122B8D7476
:101940000202AEBA851882851983E02401F0A3E073
:101950003400F02274F012259474F3122C0BEAFE7A
:10196000EBFF7A027901123D59EA8E828F83F07083
:1019700003029A1F75F00CA4FAABF012341D8A080A
:101980008B09EA45097003029A25AE08AF09750A6A
:1019900000801C90811212299DEEFAEFFB1233DBBE
:1019A0007404122B8D8A0C8B0DAE0CAF0D050A90B2
:1019B0005157E493F8E50AC398506AE50A128DBAC4
:1019C0006005E0640270E6128CB2122E6112C14A08
:1019D000123D29E960187403122E61AC82AD83EECA
:1019E000FAEFFB1235318A0C8B0DAE0CAF0DE50A08
:1019F00075F01CA4F8A9F0740E28F582740612D1B3
:101A0000EA6401708E128E70EA2413129A2F122D3E
:101A1000D4129A2C122BF3780C122B72029999750E
:101A20000800750900AA08AB09029101EA2417F51C
:101A300082E43BF583780C22C082C0839019FC7449
:101A40003BF0A37443F09019FE7435F0A37443F097
:101A5000901A02748BF0A3743EF0029E4BC082C0B9
:101A600083901A00742FF0A37443F0029E4B74F716
:101A7000122594EAFEEBFF901A6EE06408601FE006
:101A80006404601A8E828F83E054036401704412F0
:101A9000AD18F8A3E0F5838882E0640670358E8285
:101AA0008F83A3A3E064FE7003A3E0F460258E821D
:101AB0008F83A3A312C8637003A3E0697008EE24A8
:101AC0001512C84A60051244018003124407E9F563
:101AD0000880037508C2EEFAEFFB12342302835E1E
:101AE00074F41225948A088B098A828B83E0FAA306
:101AF000E0F8EA28FAE43400FB12341D8A0A8B0B62
:101B0000AE0AAF0BEE4F605A850882850983E0FC70
:101B10007D0079001233638E828F831284D9124440
:101B20003D8E828F83A3A3A3A3EAF0A3EB129B684D
:101B3000F8EE28F8E43F128651850882850983A3D0
:101B4000E0C0E012C34DD0E0F012444FEE240EF599
:101B500082E43FF583E912A4BEE0C0E012A216D0F1
:101B6000E0F0EEFAEFFB800A12A4B6E022740D1248
:101B70002B8D7F0402281974F412259474E8122C1A
:101B80000B8A088B098C0A8D0BE9FE901A6EE064B3
:101B9000046005E06408700479C2804BA3780812E1
:101BA0002DF2EE901A75129CCF1233638518828540
:101BB00019837808122DF27405122E61EEF0740468
:101BC000122E617401F07407122E61E4F0901A6E07
:101BD0007402F09019DCE0640270059019CAE4F018
:101BE000AA18AB19123C3F7418808474F41225941F
